:020000040800F2
:1000000000000110890E0708F5280008796F020822
:10001000290F0708290F0708290F0708000000000B
:100020000000000000000000000000006543000820
:1000300069430008000000006D4300088D0A0108B4
:10004000290F0708290F0708290F0708290F070894
:10005000290F0708290F07088DC2000891C2000860
:10006000290F070895C2000899C2000851300008FE
:1000700065300008793000088D300008A130000894
:10008000B5300008C9300008290F0708290F0708F4
:10009000290F0708290F0708290F07089DC2000824
:1000A000FD2E0008252F00084D2F0008E92E00081E
:1000B000752F0008892F00089D2F0008290F0708B9
:1000C000290F0708290F0708290F0708290F070814
:1000D000290F07085D2A0008692A0008290F070868
:1000E000A1C20008290F070871430008D92F000892
:1000F0000130000829300008C52F0008DD30000855
:10010000290F0708290F0708B12F0008290F070832
:10011000752A0008290F0708290F0708290F070863
:10012000F130000805310008193100082D310008B0
:1001300041310008290F0708290F0708290F070870
:10014000290F0708290F0708290F0708C5430008CA
:1001500055310008693100087D310008290F070872
:10016000290F0708290F0708290F0708290F070873
:10017000290F0708290F0708290F0708290F070863
:08018000290F0708290F0708E9
:10019000D0E907239A422FBFD01AC0688018C01A2E
:1001A000704700BFD0E9092300699A4238BF12188E
:1001B000D31A0138C01A7047D0E90902101AB0FAF0
:1001C00080F04009704700BF0246036A4069D16869
:1001D000C05C01338B4228BF00231362704700BF0D
:1001E000436A8269D154436A0169426B01338B428D
:1001F00028BF00234362D36843F08003D360704775
:10020000436B188810F0100002D01A889B880120D8
:10021000704700BF436B99891A88890610B5044658
:100220000AD592B2900607D5E26A002A29D09888AA
:10023000216B80B29047636B99891A88090692B244
:100240000FD510060DD5D4E909128A4214D0A16940
:100250002069895C99800132B2FBF0F100FB112228
:10026000A262998A1A88C90592B204D5D20744BFFE
:100270004FF6F7721A8010BDDA6822F08002DA6059
:10028000EFE79B88E2696169DBB28B54E269E16860
:10029000636B0132B2FBF1F001FB1022E261CBE7AC
:1002A000036942681F2B10B40AD95468A3F1200CCB
:1002B000202101FA0CF1214207D15DF8044B70476F
:1002C0001468202199402142F7D081690024C86830
:1002D0000C7480684C68016821F00101016020689D
:1002E00094F805C00C4C818934F81C4089B221EA8D
:1002F00004011F2B818107D9A3F1200120238B400A
:100300005DF8044BD3607047202101FA03F35DF8D8
:10031000044B9360704700BF5C8A070882B00922D3
:10032000274B8DF80720DA68D00319D4DA68D10694
:1003300040D4DA68D20541D4DA6812F0E00F3BD13C
:10034000DB6813F0020F14BF082309238DF8073070
:100350009DF80730012B0AD09DF8070002B07047C6
:1003600001238DF807309DF80730012BF4D1144A92
:1003700012E0D368DB0519D4D36813F0E00F17D16E
:10038000D36813F0020F14BF082309238DF8073038
:100390009DF80730012BDFD1D168C8034FF001036E
:1003A000F4D4D368D906E4D50623EFE70223EDE7BA
:1003B0000723EBE70623D4E70723D2E70223D0E79E
:1003C000003C0240704700BF704700BF01207047EB
:1003D000044BD3E90003984288BF03F50063181A61
:1003E000704700BFE01A0020054AD2E900318B4275
:1003F000FDD0D1180133C3F30A03087A13607047A4
:10040000E01A0020064BD3F8080800B97047D3F86B
:100410000808A0F10500B0FA80F04009704700BF5D
:10042000E01A0020012380F849307047064BD3F8CA
:100430000C08D3F81028431E90428CBF00200120E6
:100440009B1A03EBC0207047E01A002010B5D0F8CB
:10045000E83504461B699847032384F812310020CD
:1004600010BD00BF08B5042290F81211D0F8E8358D
:1004700080F8131180F81221DB689847002008BD2E
:1004800008B5D0F8E435DB6903B19847002008BD12
:1004900008B5D0F8E4351B6A9847002008BD00BFB6
:1004A00008B5D0F8E4355B6A9847002008BD00BF66
:1004B000037830B403B30446C0F1010C04EB0C0321
:1004C00014F8015FDBB2002DF8D101335B00DCB220
:1004D000138003230C704B7004785CB10223002559
:1004E0005A1CD2B2CC548D5410F8014F0233DBB2F7
:1004F000002CF5D130BC704702242346E8E700BF4A
:1005000010B5074C2068FF2808D00649D1F81428F8
:1005100001F6180100F080F8FF232360002010BDD1
:1005200000000020E01A0020432301480B807047A0
:1005300004000020122301480B807047480000206F
:10054000042301480B8070475C00002008B5044B71
:1005500004480A461946FFF7ABFF084608BD00BF2E
:10056000002300203829080808B5044B04480A462F
:100570001946FFF79DFF084608BD00BF0023002075
:100580004C29080808B5044B04480A461946FFF7E9
:100590008FFF084608BD00BF00230020542908082B
:1005A00008B5044B04480A461946FFF781FF084680
:1005B00008BD00BF002300206029080808B5044BCF
:1005C00004480A461946FFF773FF084608BD00BFF6
:1005D000002300206C290808704700BF704700BF47
:1005E000704700BF704700BF704700BF704700BF33
:1005F000044B00200522C3F80828C3F82009C3F8DB
:1006000024097047E01A0020024B0020C3F80808B4
:10061000704700BFE01A0020212838B50C4605D0ED
:1006200022282DD0202813D0002038BD0029FBD04F
:10063000072AF9D1194BD3F8280993F82C1993F804
:100640002D2993F82E39206021716271A371EBE797
:100650000029E9D0072AE7D1104DD5F8243913B184
:10066000096800209847206821796279A379C5F844
:10067000280985F82C1985F82D2985F82E39D3E716
:100680000029D1D0022ACFD1044BD3F82039002B36
:10069000CAD0098800209847C6E700BFE01A0020AA
:1006A00010B4144CD4E900239A4286BF03F5006CC1
:1006B000ACEB02029A1A0A44B2F5006F13D8B1B13A
:1006C00001444A1E013810F801CFE118824203F1BB
:1006D000010381F808C0C3F30A03F4D1636000206A
:1006E0005DF8044B704702205DF8044B70470846E4
:1006F000F6E700BFE01A00201D49D1F884391A79C5
:10070000022A00D0704710B41A4C93F9102002EB63
:10071000820204EB8202126E1089800708D51289CA
:10072000100605D49A6892070BD45DF8044B704705
:1007300000BFD1F884391A79022AE6D05DF8044B5B
:100740007047D1F888190C480C4A4FF4FA7404FB2E
:1007500001F1A2FB0121446889094268121B914200
:10076000FBD25B69002BE0D01A689B881383DCE71F
:10077000E01A002000000020001000E0D34D6210BD
:10078000034B93F85409003818BF0120704700BF8D
:10079000E01A00200E4BD3F8802942B110689188EE
:1007A0000269114203D1002283F85429704793F85B
:1007B00048290132D2B2072A83F84829F3D8D3F85E
:1007C0008C19C3F84419012283F85429704700BFDB
:1007D000E01A0020034B93F85409032894BF00202B
:1007E00001207047E01A002000487047382400209C
:1007F00030B4194B00209C7B14B11D688D4206D08B
:100800000130082803F11003F5D130BC70479AB1CC
:10081000124B03EB40218A4219D0114B93F8B421BB
:100820008AB1104B01225A7000F5817003EB001061
:100830000123837130BC70470A4B00F5817003EBD4
:1008400000108271E1E7012283F8B421E9E7022C6C
:10085000E3D1183BE8E700BF3057002030470020C5
:10086000185700201847002030B41D4C002384F88E
:10087000A03004F1180004E00133082B00F110004F
:100880001ED005688D42F7D190F80EC0BCF1030F61
:10089000F2D1BAB1134901EB4320824209D094F856
:1008A000B42112B9012284F8B4210F4901224A70FF
:1008B00000E0183903F5817301EB031301229A71EB
:1008C00030BC70470849D4F89C2003F5817301EBD4
:1008D0000313013204219971C4F89C20F0E700BF92
:1008E000185700203047002018470020A8B183681F
:1008F0001BB10E4B07229A7070470C4A1178D360D7
:1009000003294FF004000CBF80214FF48071C2E92D
:1009100001111361137590707047044A02F58051FC
:100920000123537081F8B431704700BF184700208D
:1009300010B5812104466FF01DF8204601216FF0AB
:1009400019F8204682216FF015F8FFF75DFE0020B0
:1009500010BD00BFC169026910B4002340F2011448
:10096000A0F844410B60D169846D21F002014FF081
:10097000010CD161A0F89CC32360D169044821F423
:10098000003180F890395DF8044BD161184670470A
:10099000E01A0020202301480B807047B00000209F
:1009A000122301480B807047D00000200423014827
:1009B0000B807047E40000200A4608B5054920B9BD
:1009C0000548FFF775FD034808BD0448FFF770FDB3
:1009D000004808BD742400207C29080894290808D0
:1009E00008B5044B04480A461946FFF761FD08465E
:1009F00008BD00BF74240020AC2908082048D0F8A6
:100A0000E837D0F8EC2730B59B184FF01A040C806B
:100A100001D11C4830BD1B4AD0F8EA174FF0000E38
:100A200010467546B3F1204F4FEA137C0CF13004A9
:100A30000EF1020E2ABF0CF1370C847080F802C050
:100A4000BEF1100FC5704FEA031300F10200E9D1A7
:100A500000200446B1F1204F4FEA117303F1300C2E
:100A600000F102002ABF373382F812C093740828BD
:100A7000D4744FEA011102F10202EBD1014830BDFA
:100A800000F0FF1FE800002008B5044B04480A46A8
:100A90001946FFF70DFD084608BD00BF742400206D
:100AA000C029080808B5044B04480A461946FFF750
:100AB000FFFC084608BD00BF74240020CC290808AC
:100AC00010B50F4C0F4BD4F86C1BB4F8700B0883A7
:100AD00003F58272C4F8E02CD3F80431984702E0A1
:100AE0001B69984720B9D4F8E03C002BF8D1FEE709
:100AF000D4F86C3BB4F8702B5A83002010BD00BFB3
:100B0000E01A00200000002038B5084BD3F8E03C84
:100B100053B1DB6914460D4698474FF400730268E1
:100B20002A600020236038BD1B68FFDEE01A002029
:100B300008B5074BD3F8E03C33B11B69984780F008
:100B40000100404240B208BD4FF0FF3008BD00BF79
:100B5000E01A0020002070472DE9F041164CD4F82F
:100B6000300B1646B4F8342B428303B30F4603EB25
:100B7000060806E000234D681A4639463046A84765
:100B800038B9D4F8E01C0029F4D1FEE71B69984776
:100B900020B9D4F8E03C002BF8D1FEE70136B0458F
:100BA00007F50077EDD1D4F8300BB4F8342B02837D
:100BB0000020BDE8F08100BFE01A00202DE9F041DF
:100BC000184CD4F8300B1646B4F8342B42832BB3B0
:100BD0000F4603EB060801E00B699847D4F8E01CC8
:100BE00051B10023CD681A4639463046A847D4F89B
:100BF000E01C08B10029EFD131B10B69984720B949
:100C0000D4F8E01C0029F8D1FEE70136B04507F51D
:100C10000077E3D1D4F8300BB4F8342B02830020F2
:100C2000BDE8F081E01A0020002070472DE9F04176
:100C3000204E96F8E43C002BFBD1B9B3014400F1FF
:100C4000FF384F1ED6F81018D6F80C3818F8010FD8
:100C50004A1CC2F30A029A4234BF002401249B1AA0
:100C6000314403EBC423012B81F8E80CC6F81028AB
:100C70001AD10FF057FF04460D460FF053FF031B28
:100C800061EB0501B3F57A7F71F10003F5D3D6F876
:100C90000C38D6F8102893428CBF002101219B1AF2
:100CA00003EBC123012BE4D0B845CBD10020BDE834
:100CB000F08100BFE01A002090F84820531C024445
:100CC000DBB280F8483082F8341090F849200AB13D
:100CD000132B03D9002280F8482003B9704710B5C0
:100CE000084CD4F8082802B910BDD4F80828052A01
:100CF000FAD119463430D4F88C39FFF797FFD4F87D
:100D00008C3910BDE01A002010B50A4CD4F8083810
:100D100003B910BDD4F80838052BFAD1002A0846CB
:100D2000D4F88C391146F4DDFFF780FFD4F88C3904
:100D300010BD00BFE01A002090F848100023A0F872
:100D4000483001B9704710B5084CD4F808381BB1C9
:100D5000D4F80838052B00D010BD3430D4F88C39C5
:100D6000FFF764FFD4F88C3910BD00BFE01A0020F3
:100D70002DE9F0475D4E1F4606EB80039C68002C72
:100D800000F0AD8004F13E03A36104F59F73E361BD
:100D90004FF48073C4E9043328362368666005463F
:100DA000E16094F83D00A36390460BF07BFA814626
:100DB00094F8440294F83CA0261D00284FD194F8E2
:100DC000450268BBD4F8403283BB390734D418F0ED
:100DD000020F60D118F0010F44D194F9472294F822
:100DE0004712D4F84832002A10DB41481B0184180E
:100DF000DBB284F800335209012301F01F0103FA2A
:100E000001F140F822103046BDE8F087394A01F080
:100E10000F010A441B01DBB213763046BDE8F087B0
:100E20006CF00EFAD4F84032002BCED0324A116B5F
:100E30000B4339071363CAD50135EDB2B9F1000F81
:100E4000CBD040F20673FA0689F80850A9F80630AC
:100E500036D4BB0694F8462245D4322133E06CF0F8
:100E6000EFF9ACE750460BF01DFA0135EDB2002862
:100E7000B3D040F206620572C28094F84622022185
:100E80000BF016FC94F9472294F84712D4F8483234
:100E9000002AAADABAE76B1CDBB2B9F1000F99D0CD
:100EA00089F8083040F20653A9F8063094F8462233
:100EB000484602210BF0FCFB18F0010F8DD0D1E762
:100EC00094F84622022148460BF0F2FB94F947229F
:100ED00094F84712D4F84832002A86DA96E7264674
:100EE0003046BDE8F0871221EDE700BF5C8A0708B5
:100EF00000E100E0FCEC00E0003802402DE9F047A2
:100F0000038A8489A4B21C4082B045D081468846B9
:100F10004FF0004501F14C0701F13406B4FA84F3B7
:100F200025FA03F2D24391B2A9F8101014401B3BEA
:100F3000B8F1000F5DD0042B2CD8DFE803F0504649
:100F40003B300300D8F80C30D9F82CA033B19B68A3
:100F500023B11FFA8AF108F104009847D8F8243029
:100F600033B19B6823B11FFA8AF108F11C0098473E
:100F7000D8F83C302BB19B681BB11FFA8AF1304680
:100F80009847D8F854302BB19B681BB11FFA8AF1EF
:100F900038469847002CC1D102B0BDE8F087D8F898
:100FA0000C30D9F834105B6808F104009847002C25
:100FB000B4D1F1E7D8F82430D9F838105B6808F1DB
:100FC0001C009847002CA9D1E6E7D8F83C30D9F8A6
:100FD0003C105B6830469847002C9FD1DCE7D8F87E
:100FE0005430D9F840105B6838469847002C95D1AA
:100FF000D2E7042B07D8DFE803F00319140F0A0027
:10100000D9F840300193019B002C87D1C4E7D9F86F
:101010002C300193019BF7E7D9F834300193019B01
:10102000F2E7D9F838300193019BEDE7D9F83C306D
:101030000193019BE8E700BF38B5284C94F8E42CF5
:10104000012A034603D0022A09D0002038BD2449D2
:10105000D1F8F023A2B984F8E42C002038BD002593
:1010600040F20112C0E95455C0E95655A0F8442198
:1010700000F5A2716EF08EFD84F8E45C002038BDAE
:10108000402AD4F80C0819D9403AC1F8F02340227C
:101090008118C4F80C1880B2124940F201140144BE
:1010A0000020C3E95411C3E95620A3F8444118466F
:1010B00003F5A2716EF06EFD002038BD4FF0000503
:1010C000C1F8F05302EB0001C4F80C1808BF02216C
:1010D00080B208BF84F8E41CDEE700BFE01A0020FD
:1010E000D82B0020C827002001EB810138B500EB88
:1010F000C1010E4DB1F88C1304462846FFF7D0FA13
:10110000E378C4F8A85340210022C4E9EC1201227C
:1011100093422046A4F89C2304F5677108BFC4F8E5
:10112000AC536EF037FD002038BD00BFCC2F00203F
:1011300038B52A4BD3F834240F2A04D0511CC3F8F5
:101140003414002038BD264A92F8E45C0021C3F82C
:101150003414002DF5D1D2F80C18D2F81048B1F59E
:10116000006F30D0A14235D002F6E84594BF641A32
:10117000C1F5006415FA81F5402C19D82144C2F854
:101180000C184FF00001C3F8F0130CBF0223012329
:1011900082F8E43C40F201120023C0E95455C0E952
:1011A0005643A0F8442100F5A2716EF0F3FCC8E7A5
:1011B000403CC3F8F04340310123C2F80C1882F8D8
:1011C000E43C4024E6E7C2F80C581CB1294602F67C
:1011D000E845D1E7002382F8E43CB2E7D82B0020B1
:1011E000E01A002038B5224DD5F8403495F858C49F
:1011F000044623B195F844345CEA030331D001235B
:10120000E06984F8463140F20112A4F844210268F2
:101210001849002AA8BFC2F380739B0301EA124158
:1012200043F020030B4363F31F42BCF1020F026043
:1012300000D038BDE278104BC4F8A8331F2000213D
:10124000C4E9EC01012A4FF00101A4F89C1308BF86
:10125000C4F8AC3304F567712046BDE838406EF041
:1012600099BC01216EF04CFB95F858C4C7E700BF4C
:10127000D82B0020DFBFFFFF1030002070B590F8A2
:10128000CF2590F8D13590F8CE5590F8D0C590F88C
:10129000CC1590F8CD6505EB02250CEB032C90F8EE
:1012A000D32590F8D23503EB0223012284B080F8D5
:1012B000112101F01F029BB2ADB21FFA8CFC012A72
:1012C00004468DF80810ADF80A50ADF80CC0ADF822
:1012D0000E30C0F840318DF809600AD0022A57D08C
:1012E000002A3CD001F080016EF00AFB002004B01F
:1012F00070BD90F81231032B2BD15FFA8CFCBCF13E
:10130000010F26D8D0F8E43502A99B689847BDF8AC
:101310000E30002BEAD1C4E94A33C4E94C3304212E
:101320004FF4807284F81111A4F81C2104F58E7119
:1013300020466EF0C1FB636DC44A1A61E278012A4F
:10134000D4D104F2CC545C614FF0802219681A6049
:10135000CCE720466BF01CFD002004B070BD092EC8
:10136000F7D801A252F826F013140008231500083C
:10137000531300085D150008531300088B1500086F
:101380003714000853130008A1140008D1140008F2
:1013900001F0600120295FFA8CF334D0012E00F0B7
:1013A0006181032E00F09581002E9FD190F81221CB
:1013B000022A00F01B81032ACBD11CF0800F40F0E1
:1013C000A48103EB830300EBC30393F87633002B74
:1013D00000F0A6819E4B0122C3F868249D4A022397
:1013E000C4E94E334FF48070002184F81131A4F821
:1013F0001C01C4E94C31C4E94A2204F58E7120462F
:101400006EF05AFB72E7D0F8E43502A99B68984762
:101410006CE790F81231023B012B9AD88C4BD0F834
:1014200018210021C3F8601412B10222C3F860240D
:10143000894A0223D4E72E0A022EADF8063000F0C6
:10144000CD81032E00F09181012E82D1D0F8EC35B0
:1014500080781B680DF106019847BDF80630002B17
:101460003FF444AFBDF80E20002A3FF43FAF934253
:1014700028BF13464FF480720221A4F81C210022D9
:10148000C4E94A0084F81111C4E94E33C4E94C326E
:1014900004F58E712046ADF806306EF00DFB25E7A1
:1014A000012B7FF456AF90F81221022A00F04981F7
:1014B000032A7FF44EAF4FF4807100F5887202204A
:1014C000A4F81C11C4E94E3384F81101002190E7FF
:1014D000EDB25F4E012D86F859543FF63AAF90F8C1
:1014E0001231022B00F02181032B7FF432AF002D4B
:1014F00000F07F8190F81011012910D0D0F8E43568
:101500005B68984796F85914D4F8E43584F81011BC
:101510001B6820469847D4F8E8359B689847002315
:10152000F9E690F81231023B012B3FF612AF012D84
:101530007FF4DCAED0F8E43500259B68C0F8185184
:1015400002A9984704224FF48073C4E94A55C4E9BC
:101550004C5584F81121A4F81C31E7E6012D00F068
:10156000CC80022D7FF4C2AE5FFA8CF3002B7FF4A7
:10157000BDAE02694FEA1C23023B5268032B00F206
:101580005681DFE803F05B426B5F5CEA03037FF4A4
:10159000E0AE90F81221032A3FF4DBAE016905F0BA
:1015A0007F0680F8146108681A4665F30A12024340
:1015B0000A604FF480720421C4E94A33C4E94C3311
:1015C00084F81111A4F81C2104F58E7120466EF0E8
:1015D00073FA636D1D4A1A61E278012A0DD0002E5C
:1015E00000F01281022384F812317FE65A063FF49C
:1015F0007DAE19466EF084F978E604F2CC525A6159
:101600004FF0802219681A60E9E7032363F306129A
:1016100001210F4D84F816110421002384F81111C3
:101620004FF48071A4F81C11C4E94A33C4E94C3367
:1016300004F58E712046C5F864247AE6022363F32C
:101640000612E5E7052363F30612E1E718000860D8
:10165000D82B00204030002038300020042363F3D2
:101660000612D5E790F81221022ABFD0032A7FF490
:1016700070AE002D7FF43AAE13F07F023FF44FAF0F
:101680001CF0800F40F0C48003EB830100EBC1012C
:1016900081F8742381F8765381F87553282101FB72
:1016A000030300EB820293F87713506D03688A1EE0
:1016B000012A6FF35553D4F8E4258CBFC3F30071AE
:1016C000012161F31C739268036002A920469047D0
:1016D00025E790F81221022A88D0032A7FF439AE38
:1016E00025B9590602D019466EF00AF9D4F8E43546
:1016F00002A99B682046984711E7D0F8E43502A973
:101700009B68C0F81851984709E703F07F0303EB83
:10171000830300EBC30393F81E31002B7FF45AAE12
:10172000454B0022C3F8682458E6002D3FF40AAF69
:1017300001210322D0F8E43580F8101180F812213D
:10174000E6E63E4984F811214FF480700022C4E996
:101750004A11A4F81C01C4E94E33C4E94C3204F523
:101760008E7120466EF0A8F9C0E5EDB2052D3FF66A
:10177000F0ADDFE805F02B231B130B03D0F8EC359D
:1017800080789B690DF10601984766E6D0F8EC3544
:1017900080785B690DF1060198475EE6D0F8EC357C
:1017A00080781B690DF10601984756E6D0F8EC35B4
:1017B0008078DB680DF1060198474EE6D0F8EC35ED
:1017C00080789B680DF10601984746E6D0F8EC3525
:1017D00080785B680DF1060198473EE6D0F8E43565
:1017E00080789B6A0DF1060198474670C4F8F005B1
:1017F00033E60222D0F8E43580F8122180F8105147
:101800005B68294698479DE6012384F812316DE50F
:10181000282303FB020181F81C2100EB820281F8DE
:101820001E5181F81D61906991F81F113EE7012357
:1018300063F30612ECE600BFD82B00203430002002
:1018400010B5044629B990F81121032A0DD00020C3
:1018500010BDD0F8E4359B69002BF8D090F8122128
:10186000032AF4D19847002010BDD0F890230B46EE
:10187000D0F87C138A4213D9C078521A0128C4F8D0
:10188000902336D08A4228BF0A4692B2C4E9E223A6
:1018900004F55D71A4F8743320466EF00DF9D6E7B7
:1018A000D0F8E4351B691BB190F81221032A1ED031
:1018B00000234FF480720421C4E94A33C4E94C3355
:1018C00084F81111A4F81C2104F58E7120466EF0E5
:1018D000F3F8636D104A1A61E278012AB7D104F275
:1018E000CC545C614FF0802219681A60AFE79847CA
:1018F000DEE78A42D4F88003A4F8743328BF0A468E
:10190000084492B2C4E9E22304F55D71C4F880038F
:10191000C4F88403C0E700BF1800086038B5044667
:1019200049B990F81131022B11D094F81631012BDE
:1019300040D0002038BDD0F8E4355B69002BF8D0EA
:1019400090F81221032AF4D19847002038BDD0F82E
:101950003831D0F82421934236D9C178012908BF03
:10196000D0F82811A3EB020318BFD0F82821C0F843
:10197000383108BF52189BB24FF480710025C0E97E
:101980004C35A0F81C11C0E94A2200F58E716EF0AA
:1019900093F8E378C4F88053012BC4E9E255A4F826
:1019A000745308BFC4F8845304F55D7120466EF08B
:1019B00083F8BAE72A4B2269D3F8641451600023F4
:1019C00084F81631002038BDD0F83C31B3FBF2F575
:1019D00002FB1535ADB99A4213D8D0F84021934295
:1019E0000FD24FF48073A0F81C31C0E94A55C0E90A
:1019F0004C5500F58E716EF05FF8E378C4F84051F5
:101A0000C8E7D4F8E435DB681BB194F81221032A47
:101A100023D0E2780023012A4FF0050108BFC4F863
:101A20008433C4E9E23384F81111C4F88033A4F894
:101A3000743304F55D7120466EF03EF8636D094A1B
:101A40001A61E278012A7FF470AF04F2CC525A6135
:101A50004FF0802219681A6067E720469847D8E758
:101A6000D82B002018000860F8B50B7813F060063A
:101A70000D46044620D0202E25D1CE884EB31B061D
:101A800049D5384F687832463946FEF7C5FDEB88B0
:101A90000222002684F811214FF48072C4E94E33EB
:101AA000C4E94A77C4E94C36A4F81C2104F58E71C8
:101AB00020466EF001F80AE04B780A2B17D00B2B6A
:101AC0000ED0062B03D120466BF062F90226304679
:101AD000F8BD022248781144FEF79EFD3046F8BD5D
:101AE0008B78002B3AD1204BC3F86C64EFE70222CD
:101AF00080F811214FF48072A0F81C211B4A0123A9
:101B0000C0E94E33C0E94A22C0E94C3600F58E7177
:101B10006DF0D2FFDBE7164B164A4978116003F6E9
:101B200018020321C0E9E46680F81111C0F8886347
:101B3000C0F88023C078C3F8146801284FF0000370
:101B4000C4F88C33A4F8743304F55D7108BFC4F88D
:101B5000842320466DF0B0FF0026B8E76BF018F93B
:101B6000B5E700BFF8220020D82B00204430002029
:101B7000E01A002000000020002310B5194604469A
:101B800040226DF029FF80212046002340226DF085
:101B900023FFD4F8E835A078012284F812215B688D
:101BA0009847002010BD00BF10B502230446402214
:101BB00081216DF011FF20460223402201216DF0AA
:101BC0000BFF20460323082282216DF005FF0E4BF8
:101BD0000222A3F84C20FEF70BFDE2780B4BC4F871
:101BE000A83340200021C4E9EC01012A4FF0010193
:101BF000A4F89C13204604F5677108BFC4F8AC3301
:101C00006DF0C8FF002010BD00000020CC2F002088
:101C100070B5812182B00446314E6DF0ABFE0121DA
:101C200020466DF0A7FE0025022340228121204698
:101C300086F890596DF0D0FE012102234022204603
:101C40006DF0CAFE274B86F89059D3F8702483F8BC
:101C500058541268284690470095009BE16843F06D
:101C600010030093009B0B610A691F4B009203E075
:101C70000A690092013B02D0009AD006F8D40023F2
:101C80000193019B43F020030193019A164B01201D
:101C900060F38A120192019A0A610A69019203E0D3
:101CA0000A690192013B02D0019A9206F8D4E278C7
:101CB0000E4BC4F8A83300211F20C4E9EC01012A0F
:101CC0004FF00101A4F89C1304F5677105D020467C
:101CD0006DF060FF002002B070BDC4F8AC33F6E7D1
:101CE000E01A0020D82B0020400D03001030002007
:101CF0002DE9F047294FDFF8AC90294CDFF8A8A078
:101D000082B000F10108002606E09DF80700FF28D8
:101D10002FD1013646452CD0D7F8845995F910308B
:101D2000AA6803EB830309EB83039207186E23D59C
:101D3000012300220DF107016DF0DEFFAB689B0768
:101D4000E3D4D7F8882961684FF4FA7303FB02F2F1
:101D5000AAFB0232920963685B1A9A42FBD26B6952
:101D6000002BD2D09DF807001A689B881383FF28A8
:101D7000CFD002B0BDE8F0876B6913B11A689B88B9
:101D80005383D7F888296168D200AAFB02329209EE
:101D900063685B1A9A42FBD2CAE700BFE01A0020D0
:101DA000001000E000000020D34D621070B5044622
:101DB00008200D46FFF79CFFFF2822D0FE2801D007
:101DC000022070BD254E2146D6F884092B460022FC
:101DD0006DF0E2FFD6F88449214A94F91030A168E9
:101DE00003EB830302EB83038A07186E0BD50022F3
:101DF000022311466DF080FFA3689B0716D50020D3
:101E000070BD012070BD636913B11A689B8853834C
:101E1000D6F888291349144B4D68D200A3FB02322F
:101E200092094B685B1B9A42FBD2E0E7D6F88829FF
:101E30000C490D4B4FF4FA7000FB02F2A3FB023287
:101E4000486892094B681B1A9A42FBD260690028C5
:101E5000B7D0036882881A83002070BDE01A002082
:101E600000000020001000E0D34D621070B52E4C31
:101E70002E4AD4F8845995F9103003EB830302EB12
:101E80008303AA6882B000204FF6FF519207C4F87E
:101E90005009ADF80410186E33D5022301AA0021B1
:101EA0006DF02AFFAB689B0714D50120FFF720FFD8
:101EB000FF2809D0D4F88C39C4F84439092200200D
:101EC00084F8542902B070BD0423022084F85439E8
:101ED00002B070BDD4F888391549164E48684FF4E1
:101EE000FA7203FB02F2A6FB023292094B681B1A3C
:101EF0009A42FBD26B69002BD7D01A689B88138358
:101F0000D3E76B6913B11A689B885383D4F8882987
:101F10000749084B4E68D200A3FB023292094B6876
:101F20009B1B9A42FBD2B8E7E01A00200000002079
:101F3000001000E0D34D621070B582B004460B0E65
:101F4000080C0A0A44F040058DF8013095238DF8FD
:101F500000508DF802008DF803208DF804108DF8E4
:101F600005306AF0B3FE08B9002C44D1234D244A51
:101F7000D5F8844994F91030A16803EB830302EB90
:101F800083038A07186E0CD506236A4600216DF07C
:101F9000B3FEA3689B0717D50820FFF7A9FE02B080
:101FA00070BD636913B11A689B885383D5F888297B
:101FB0001449154B4E68D200A3FB023292094B68BC
:101FC0009B1B9A42FBD2DFE7D5F888290D490E4BBF
:101FD0004FF4FA7000FB02F2A3FB02324868920948
:101FE0004B681B1A9A42FBD26369002BD4D01A6843
:101FF0009B881383D0E7FF2002B070BDE01A002059
:1020000000000020001000E0D34D62102DE9F041E7
:102010003A4C82B00546884617461E4694F8540945
:1020200004280DD0082807D1D4F84C39AB425FD032
:10203000FFF71CFF0228F1D0012002B0BDE8F081BB
:10204000D4F884391A79022A36D094F84A398BBBED
:1020500069021820FFF770FF002843D194F8543923
:10206000082B4FF0FF038DF804300CBFFC23FE2338
:10207000D4F884098DF8053001AA022300216DF0FF
:102080008BFED4F884094246802300216DF084FE43
:10209000012206230020C4F83089C4F83459C4F85A
:1020A0003C79C4F8406984F8382984F8543902B07E
:1020B000BDE8F0812946CCE79A689207C5D55B69EF
:1020C00013B11A689B885383D4F888390C49DA0015
:1020D0000C4B4868A3FB023292094B681B1A9A42C8
:1020E000FBD2B2E7FEF708FBFEF754FB0320A4E7A0
:1020F000FF238DF80430FC23BAE700BFE01A00206C
:10210000001000E0D34D621070B51F4C94F85439A4
:10211000042B06460D4609D0082B25D1D4F84C399E
:1021200083422FD0FFF7A2FE02281DD1D4F88409E4
:1021300007F010FF00213720FFF7FEFE2946172089
:10214000FFF7FAFEC0B994F84A397BB97102192039
:10215000FFF7F2FE80B9082384F85439C4F85059C7
:10216000C4F84C69022070BD012070BD31461920B1
:10217000FFF7E2FE0028EED0FEF7BEFAFEF70AFBFC
:10218000032070BD022070BDE01A00202DE9F0414F
:10219000284C94F854C9BCF1040F074688461646EB
:1021A0001D4609D0BCF1080F02D00020BDE8F08127
:1021B000FFF75CFE0228F8D1D4F884391A79022A94
:1021C00022D094F84A39B3B979021120FFF7B4FE4E
:1021D000B8B9D4F88C39C4F83089052284F8542968
:1021E000C4F83479C4F83C69C4F84059C4F8443997
:1021F0000120BDE8F08139461120FFF79DFE00283F
:10220000E7D0FEF779FAD0E79A689207D9D55B69EB
:1022100013B11A689B885383D4F888390649DA00C9
:10222000064B4868A3FB023292094B681B1A9A427C
:10223000FBD2C6E7E01A0020001000E0D34D621088
:102240002DE9F043844CD4F8840987B000283AD0B3
:1022500094F85409814E824D824F431E082B1CD89E
:10226000DFE813F09800C30042011B0009005D0085
:1022700045001B003400D4F830094FF40071FFF71B
:1022800095FD012800F09581022800F09A81002830
:1022900000F0C78194F85409431EDBB2022B0AD820
:1022A000D4F88C39D4F844299B1AC82B06D9FEF7E8
:1022B00071FA94F85409042800F09981A0F10800FB
:1022C000B0FA80F0400907B0BDE8F0836AF0FEFC88
:1022D000002840F05B82D4F84439D4F88C29FA33D2
:1022E0009342D7D2FEF756FA94F85409B5E76AF04C
:1022F000EDFC0028EFD0D4F850390022012B84F8EF
:10230000482940F24B82D4F84C290820013B013285
:10231000C4F85039C4F84C2984F85409CEE7D4F8ED
:10232000303994F83829D4F8840903EBC21200211B
:1023300080236DF031FD94F838390133DBB2042B82
:1023400084F83839A6D1D4F8840902233246002112
:102350006DF022FD0123D4F88409002202A96DF05A
:102360001BFD9DF8083003F01F03052B00F0F681DC
:10237000FEF710FAD4F83C89B8F1000F00F0348170
:102380000120D4F84039D4F834190022C04794F819
:10239000540962E7D4F8840907F0DCFD00210846FF
:1023A000FFF7CAFD8046FEF7A7F9B8F1010F4AD141
:1023B000D4F884094FF0000984F8499907F0CAFD60
:1023C00040F2AB110820FFF7B7FD052800F011819E
:1023D000012800F05881FEF78FF994F84939002B55
:1023E00000F0B981022384F85439D4F8840907F045
:1023F000B1FD94F84939022B0CBF4FF080484FF0E3
:10240000000800213720FFF797FD41462920FFF7FC
:1024100093FD8046FEF770F9B8F1000F13D194F8E0
:102420004939022B00F0128184F84A89D4F88439A2
:102430001A79022A00F0E08000210920FFF77CFDD4
:1024400090B1FEF759F9D4F88409022107F068F831
:1024500094F85409431E20E7E01A0020B48A0708C4
:10246000001000E0D34D6210D3481021FFF79EFC0E
:102470000028E6D194F87F39DB07E2D594F870198B
:10248000891100F016810129DBD194F87729DFF852
:102490002CE39200D2B216214FF0020CCCF10803CB
:1024A0008B4228BF0B46C3F1080C42FA0CF298404D
:1024B000C91A40EA02004FF0000C1EF8012FEDD1BE
:1024C000431C9B02C4F85839FEF716F9D4F8840966
:1024D00007F040FD00210A20FFF72EFD002840F004
:1024E000E180032384F85439102102A8FFF75EFC31
:1024F0000028A8D19DF8083084F85E39BDF809306D
:102500009DF816209DF810105BBAA4F85C399DF870
:102510000B3084F85F399DF80C3084F860399DF8F1
:102520000D3084F861399DF80E3084F862399DF8D9
:102530000F3084F863399DF815301B01DBB243EA94
:10254000121302F00F0203F5FA6384F86C29DDF828
:102550001120A4F86A390B0912BA84F8683901F01D
:102560000F0384F86939C4F86429FEF7C5F894F8B4
:102570004A397BB9D4F8840907F0ECFC4FF40071B8
:102580001020FFF7D9FC8046FEF7B6F8B8F1000F2F
:102590007FF4A8AED4F88409022106F0C1FF00221E
:1025A00004230120C4F8502984F8543907B0BDE849
:1025B000F083D4F84439D4F88C2964339342BFF4BF
:1025C00069AEFEF799F8FEF7E5F8D4F83C89B8F162
:1025D000000F09D000221046D4F84039D4F834193D
:1025E000C04794F8540938E694F8540935E60120B8
:1025F00069E684F84989EEE69A6892077FF51CAF90
:102600005B6913B11A689B885383D4F88839696869
:10261000DA00A7FB023292096B685B1A9A42FBD27E
:102620000AE70190FEF768F8D4F83C59019884F85D
:102630004809042384F85439002DD8D0D4F84039FF
:10264000D4F83029D4F83419A84723E6D4F88409FB
:1026500007F080FC41463A20FFF76EFC4246814677
:102660000423D4F8840902A96DF096FBFEF744F820
:10267000B9F1000F7FF436AE029B1BBAC3F380732F
:1026800084F84A39D2E60423D4F884094A4602A9D8
:102690006DF082FB9DF80B30AB2B04BF022384F856
:1026A000493998E6FEF728F8FEF774F894F85409CB
:1026B000D3E594F8753994F87909DFF8048103F0CB
:1026C0000F0380014FF0010C0CFA03FC5FFA80F954
:1026D00003234FF0060ECEF108029A4228BF1A4695
:1026E000C2F1080049FA00F091409B1A18F8019FC6
:1026F00041EA00014FF0000EEDD194F87689DFF841
:10270000C4904FEA881802315FFA88F80C2006223C
:1027100000E00022C2F10802824228BF0246C2F154
:10272000080E48FA0EFE9340801A19F8018F4EEAFF
:102730000303EED1013303FA01F14FEAEC72A1FB7E
:102740000C3C01FB02C15B0A43EAC153C4F858398F
:10275000FDF7D2FFBAE684F8543974E6D4F83C5950
:10276000D4F88C39C4F84439072084F85409002D72
:102770003FF4A4ADD4F84039D4F83029D4F8341952
:102780000120A84794F85409431E86E50190FDF7FF
:10279000B3FF0423019884F8543994E505D0042349
:1027A00084F85439FDF7A8FF74E5FFF75FFB0228B2
:1027B0007FF470ADF6E700BF5024002057240020BE
:1027C000592400205624002070B50D230022342106
:1027D000022009F0ABFF2F4DC5F88409002855D021
:1027E000002106F09DFE0EF09DF904460E460EF007
:1027F00099F9031B61EB0602B3F57A7F72F10003CE
:10280000F5D3D5F88429536913B119689B880B83D4
:1028100092F91030204E214C03EB830306EB830327
:102820000022186E11460A236DF066FAD5F8840965
:102830000379022B0CD190F9103003EB830306EBE4
:1028400083031B6E1A8992070DD51B891B060AD4B8
:10285000D5F88C19C5F844190122002385F85429AC
:1028600085F8483970BD013CE5D1022106F058FEDB
:10287000D5F8840909F000FF95F84839C5F884496E
:10288000013385F8544985F8483970BD85F85409F5
:1028900070BD00BFE01A002000000020A1860100EA
:1028A0001049114BD1F8882042F4700210B4C1F8DD
:1028B00088201A680D4C002042F001021A609860CE
:1028C0001A6822F0847222F480321A605C601A68FE
:1028D000074C22F480221A60D8608C605DF8044BAB
:1028E000704700BF00ED00E00038024010300024C7
:1028F00000000008704700BF2DE9F84346697EB923
:10290000D0F80080C8F30D0904460F46B9F1000F56
:1029100026D03F68FDF702FD092804D06FF00106BC
:102920003046BDE8F8834A4D2B6923F440732B6190
:102930002B6943F400732B612B6943F001032B6176
:10294000C8F80070FDF7EAFC2B69092823F00103A1
:102950002B61E3D12368043323603046BDE8F8835C
:102960003C4B98452AD303F58043984524D303F57F
:102970008043984554D3384B984554D903F5803358
:10298000984553D903F50033984552D903F50033E0
:10299000984551D903F5003398453ED903F50033E6
:1029A00098454CD903F5802398454BD9B8F1016F70
:1029B0004BD305200EF012F94FF00809FDF7AEFCDD
:1029C000092804D04FF0FF363046BDE8F883204D8B
:1029D0002B6923F440732B612B6943F400732B6143
:1029E0002B6923F0F8032B612B6943EA090343F0B9
:1029F00002032B612B6943F480332B61FDF78EFCBE
:102A00002B6923F002032B612B69092823F0F803BB
:102A10002B61D7D1D4F800807BE74FF03809CDE7A0
:102A20004FF01009CAE74FF01809C7E74FF0200927
:102A3000C4E74FF02809C1E74FF03009BEE74FF077
:102A40004009BBE74FF04809B8E74FF05809B5E730
:102A5000003C024000400008FFFF00080148FDF76D
:102A6000D9BB00BF280100200148FDF7D3BB00BF40
:102A7000740300200148FDF7CDBB00BFC005002056
:102A8000704700BFF0B5254B0268254983B0064664
:102A9000002401E051F834309A4209D001340E2C60
:102AA000F8D100211F4A052005F04CFB002113E05E
:102AB0001D4F07EB8407D7F8745485B1717901EB8A
:102AC000410305EBC30300221820C3E9032200FBE6
:102AD00001559E601A75291D084603B0F0BD0721F7
:102AE0006C2005F029FC0146C7F8740470B1294632
:102AF0006C2273F087FF0A4BD7F8745403EBC404BD
:102B0000C5E90045ED616D63ED64D7E70190074AC3
:102B1000052005F017FB0199DEE700BF000001402A
:102B2000B88A0708DC290808D82B0020042A0808DE
:102B3000704700BFB0B14B6810B4A3B18B6813B33A
:102B400043681A68816058799189022383400B4356
:102B50009BB2938193899BB243F0010393815DF80B
:102B6000044B7047704743681A685C7993894FF04B
:102B7000020C0CFA04FC9BB28C6823EA0C039381D0
:102B8000A4B18160E6E744682268938923F00103D9
:102B90001B041B0C93818160607991895DF8044B63
:102BA000022383400B439BB293817047938923F0A8
:102BB00001031B041B0C93818160D0E738B5D0E979
:102BC000004307EE902A1B68354A2068013993427A
:102BD00004688DB216D002F58062934212D002F5DD
:102BE000705293420ED002F5806293420AD002F5F1
:102BF0008062934206D02B4BD3F808385B0807EE6F
:102C0000103A04E0274B03F6080393ED007ADFED5A
:102C1000266AB8EE477AF8EE677A87EE270A30EE32
:102C2000260A6EF045FF1E4A23880138944280B27E
:102C30009BB212D002F5806294420ED0B4F1804F64
:102C40000BD0A2F58032944207D002F58062944204
:102C500003D002F58062944202D123F070039BB24C
:102C6000124A944212D002F5806294420ED023F4AC
:102C7000407302F56C429BB294422380E56220854A
:102C80000AD1002323860123A38238BD2380E56275
:102C900020850123A38238BD054B9C42F1D0F8E783
:102CA00000000140000000200AD7233C0010004033
:102CB0000004014070B54068837903F0020213F00C
:102CC000040300F0C9804FF0000E1346042472463E
:102CD000754690F805C0BCF1030F30D8DFE80CF062
:102CE0008E5F30020368188C20F480500004000CC2
:102CF0001884188C9C8820F4005000042A43000C8F
:102D000040EA0232988B6C4D20F4E6400004000C3F
:102D1000AB42A4B240F4C04000F0B08005F580653D
:102D2000AB4200F0AB809C80988319641A849A8B24
:102D300022F400621204120C42F400629A8370BD05
:102D40002A4305685C4E288C20F480700004000C37
:102D50002884288CB5F804C020F400700004000C0E
:102D600040EA0222A88B20F073000004000CB54258
:102D70001FFA8CFC40F0600073D006F58066B54207
:102D80006FD0A5F804C0A883E9632A84AB8B23F035
:102D900008031B041B0C43F00803AB8370BD2A43DC
:102DA0000568454E288C20F010000004000C288493
:102DB000288CB5F804C020F020000004000C40EA84
:102DC0000212288B20F4E6400004000CB5421FFAE2
:102DD0008CFC40F4C04061D006F58066B5425DD001
:102DE000A5F804C02883A9632A842B8B23F40063ED
:102DF0001B041B0C43F400632B8370BD00682E4E34
:102E00002A43058C25F001052D042D0C0584058C25
:102E1000B0F804C025F002052D042D0C2A43058BC3
:102E200025F073052D042D0CB0421FFA8CFC45F0E3
:102E3000600528D006F58066B04224D0A0F804C012
:102E4000058341630284038B23F008031B041B0CDE
:102E500043F00803038370BD4FF4807E1C460125B8
:102E600037E722F4006242EA032222F480622CF463
:102E7000405C42EA04224CEA0E1C82E724F48044BF
:102E800044EA8E144FE74FF6F37616402CF4407C5C
:102E900046EA03024EEA0C0C2243CFE722F08002FE
:102EA00042EA031222F040022CF4406C42EA04127F
:102EB0004CEA8E0C94E700BF000001404268537951
:102EC000032B0FD8DFE803F00B0805021068403031
:102ED000704710683C307047106838307047106891
:102EE0003430704700207047024B0348D3F8741405
:102EF000FEF704B8D82B00200000014010B5064CA6
:102F00000648D4F87414FDF7F9FFD4F89414044873
:102F1000BDE81040FDF7F2BFD82B002000000140B3
:102F20000040014010B5064C0648D4F87414FDF773
:102F3000E5FFD4F898140448BDE81040FDF7DEBF63
:102F4000D82B0020000001400044014010B5064C81
:102F50000648D4F87414FDF7D1FFD4F89C14044843
:102F6000BDE81040FDF7CABFD82B0020000001408B
:102F700000480140034B4FF08040D3F87814FDF730
:102F8000BDBF00BFD82B0020024B0348D3F87C14F0
:102F9000FDF7B4BFD82B002000040040024B0348CB
:102FA000D3F88014FDF7AABFD82B002000080040FA
:102FB000024B0348D3F88414FDF7A0BFD82B0020A0
:102FC000000C0040024B0348D3F89014FDF796BF65
:102FD000D82B00200004014010B5064C0648D4F858
:102FE0009014FDF78BFFD4F8A0140448BDE81040FE
:102FF000FDF784BFD82B00200004014000180040DA
:1030000010B5064C0648D4F89014FDF777FFD4F8B5
:10301000A4140448BDE81040FDF770BFD82B002071
:1030200000040140001C004010B5064C0648D4F8CE
:103030009014FDF763FFD4F8A8140448BDE81040CD
:10304000FDF75CBFD82B00200004014000200040A9
:103050000348D0F8183813B100F60C001847704731
:10306000000000200348D0F8383813B100F62C00D7
:1030700018477047000000200348D0F8583813B1B3
:1030800000F64C0018477047000000200348D0F8B5
:10309000783813B100F66C00184770470000002024
:1030A0000348D0F8983813B100F68C0018477047E1
:1030B000000000200348D0F8B83813B100F6AC0087
:1030C00018477047000000200348D0F8D83813B1E3
:1030D00000F6CC0018477047000000200348D0F8E5
:1030E000F83813B100F6EC001847704700000020D4
:1030F0000348D0F8183913B100F60C101847704780
:10310000000000200348D0F8383913B100F62C1025
:1031100018477047000000200348D0F8583913B111
:1031200000F64C1018477047000000200348D0F804
:10313000783913B100F66C10184770470000002072
:103140000348D0F8983913B100F68C10184770472F
:10315000000000200348D0F8B83913B100F6AC10D5
:1031600018477047000000200348D0F8D83913B141
:1031700000F6CC1018477047000000200348D0F834
:10318000F83913B100F6EC10184770470000002022
:1031900002683649002310B422F00102212488423B
:1031A0000260036043608360C3600361446138D0A0
:1031B0002F4B98422ED02F4B98423CD02E4B98420A
:1031C00040D02E4B984232D02D4B984241D02D4BBF
:1031D000984246D02C4B984217D02C4B98423CD06A
:1031E0002B4B984216D02B4B984224D02A4B984216
:1031F00028D02A4B98421AD0294B984229D0294BE3
:1032000098422ED0284B984208D14FF03D5243F8B7
:10321000AC2C03E04FF4746243F8202C5DF8044BAF
:103220007047224B5DF8044B3D229A607047204A5C
:1032300043F8642CF2E74FF474125DF8044B43F842
:10324000382C70474FF074625DF8044B43F8502CF3
:103250007047184A43F87C2CE0E73D2243F8082CDD
:10326000DCE7154A43F8942CD8E700BF1060024011
:103270002860024040600240586002407060024096
:1032800088600240A0600240B860024010640240C2
:103290002864024040640240586402407064024066
:1032A00088640240A0640240B864024000600240AA
:1032B0003D000020400F002000003D2000222DE9AD
:1032C000F04713460D684FF0010E032604E001336A
:1032D000102B02F1020239D00EFA03FC3CEA05047D
:1032E000F5D1076806FA02F427EA040707600F79A8
:1032F000D0F800A007FA02F9013F49EA0A09012FB4
:10330000A046C0F800906FEA040411D887683C40DA
:1033100084604C79876894403C438460446824EA24
:103320000C0444608C7947689C40A4B23C434460E0
:10333000C46824EA0804C460CC79C76894400133A7
:103340003C43102BC46002F10202C5D1BDE8F087F6
:103350002DE9F0412348244F244E254C82B03822D9
:10336000002173F04FFB002557F82510324600234B
:1033700001E054F8332091422ED001330E2BF8D1C6
:103380000020053569F05CFF3C2DEDD1DFF8588059
:10339000184F08F1F0054FF0007698F8040008F097
:1033A00081FF08F11408044688B1036803F13F4324
:1033B00003F57E0307EB932393F8CC0069F040FFFD
:1033C000A3880196206800936946FFF777FFA84518
:1033D000E3D102B0BDE8F081064A02EBC30393F8E3
:1033E0006000CEE74C3000200C0A002000000140B5
:1033F000B88A07085C8A0708224A936803F00C031E
:10340000042B10B421D0082B22D01F4B03601D4C7D
:103410001E4AA168C1F30311114491F8FC1ACB4074
:103420004360A168C1F38221114491F8FC1A23FA88
:1034300001F18160A1685DF8044BC1F342310A4497
:1034400092F8FC2AD340C3607047114B0360DEE75B
:103450005368516813F4800F01F03F01536814BFA3
:103460000B4A094AB2FBF1F1064A5268C2F3014223
:10347000C3F38813013201FB03F35200B3FBF2F3F1
:103480000360C4E7003802400024F400000000207C
:1034900000127A0070B5446B8668A38923F4005348
:1034A0001B041B0CA38182790546407912F0040F9E
:1034B00014BF4FF4805C4FF0000C110310F0010FAB
:1034C0004FEA02220CBF0023042302F4806280072B
:1034D00048BF43F0080342EA0C021343228A92B227
:1034E00001F4005122F440520A432282A28922F4BC
:1034F000B05222F00C021204120C1A43A281A38AC9
:1035000023F440731B041B0C84B0A3826846FFF7AE
:1035100073FF244B9C4205D003F580639C4201D08D
:10352000029A00E0039AA3891F491B0402EB82025E
:103530004CBF7300B30002EB8202B2FBF3F3A1FBBA
:103540000302A08952096426000406FB12334FEAE5
:1035500002121FD41B013233A1FB0313C3F3431325
:1035600013439BB22381AB796A6B13F0080F938AE4
:103570000AD09BB243F00803938293899BB243F431
:103580000053938104B070BD23F008031B041B0C8F
:103590009382F2E7DB003233A1FB0313C3F3421340
:1035A0001343DEE7001001401F85EB512DE9F8437E
:1035B0001D462A4B9DF820809DF8249098420F4686
:1035C00016463BD0264B984240D0264B984224D1F9
:1035D0004B46424629460320FDF7CAFB044600231A
:1035E000C4E90B76C4E90733C4E9093384F80580DC
:1035F000A56084F806902046FFF74CFF18F0010FF5
:10360000626B13D118F0020F0BD193899BB243F474
:10361000005393812046BDE8F88300242046BDE88E
:10362000F883D36843F08003D360EEE74FF6DF738F
:103630001380D36843F02003D360E3E74B46424650
:1036400029460020FDF794FB0446C8E74B46424656
:1036500029460120FDF78CFB0446C0E7001001401D
:1036600000440040004C0040816013E7417111E7C5
:103670002DE9F043DFF8148208EBC00985B0054658
:10368000C70099F8100B08F00DFE044699F8110BCD
:1036900008F008FE064699F8120B69F0D1FD6B1C84
:1036A000DBB2002C00F0AD8040F60C122372E280F9
:1036B000002E00F0C380337240F60C232046F380C6
:1036C00004223A2108F0F4FF042230463A2108F09F
:1036D000EFFF08EB0703624AD3F80C4B944200F06B
:1036E0009880604B9C4200F09E805F4B9C4200F0B3
:1036F000AB80474497F8132B022A5CD0032A7ED074
:103700005A4B5B4E012A18BF1E46A7886846FFF732
:1037100073FE27F03F07029B564AB3FBF6F63F04C1
:10372000A2FB03233F0C47EA9347A780228822F09D
:1037300001021204120C2280B2B2C6F30B069B0CDB
:10374000002E59D04FF4967101FB03F34A49A1FBB7
:1037500003139B0901339BB242F400422384A283EA
:103760002388464A9BB243F001032380238823F435
:10377000816323F002031B041B0C4FF4804143F4CC
:10378000806323802181238823F080031B041B0C8A
:10379000238023889BB202EB451243F00103238070
:1037A0000121002382F8B05482F8B11482F8B234B7
:1037B00005B0BDE8F083A6886846FFF71DFE26F039
:1037C0003F06029A2B4B3604A3FB0213360C46EA43
:1037D0009346A680218821F001010904090C21806B
:1037E0009B0C2749013392092384A1FB02329209E1
:1037F000042A38BF0422B2E742F00102A2E7214EB8
:1038000083E7002E3FF465AF337240F60C23F3805C
:103810005AE71D4B1A6A42F400121A621A6A22F41D
:1038200000121A6265E703F5F0331A6A42F4800267
:103830001A621A6A22F480021A625AE704222046A7
:103840003A2108F035FF44E703F5EE331A6A42F4F3
:1038500000021A621A6A22F400021A6249E700BFE3
:103860000054004000580040005C0040804F1200AF
:10387000009F240083DE1B43D34D6210D82B002011
:10388000632D3E05C02709000038024000000020DB
:103890002DE9F047954D90F900108046807805EBB2
:1038A000C1060138CC0090B0D6F80C1B14282ED8D5
:1038B000DFE810F053012601150057006100A20057
:1038C000AA00CB01BD017D00870045020D02E00189
:1038D000C500D50030003800AA019C015B01888A30
:1038E0000C8B81B2824841EA044130EA010100F0C8
:1038F0002681D8E90210521A42F2107163EB0003DC
:103900008A4273F1000302D3152388F8023010B005
:10391000BDE8F08798F813000882C8E90223122056
:1039200088F80200888A0C8B80B240EA0440714C0F
:1039300034EA000000F0B68000200E900F900120C5
:103940000F910E900E99002900F01E820F991431EC
:103950000F910F9909684905CBD5142388F80230D7
:10396000D5E798F8110000F0FE000882C8E90223AC
:10397000052088F80200888A0C8B80B240EA044057
:103980005D4C34EA000000F0A4800020009001901B
:103990000120019100900099002900F00182019915
:1039A00014310191019909684F05D6D4A1E798F81F
:1039B000110040F001000882C8E902230B2088F8BA
:1039C0000200888A0C8B80B240EA04404B4C34EAF7
:1039D00000006FD000200490059001200591049014
:1039E0000499002900F0D6810599143105910599B3
:1039F00009684D05B1D47CE798F813000882C8E93E
:103A00000223072088F80200888A0C8B80B240EAE3
:103A10000440384C34EA00005FD00020029003904C
:103A20000120039102900299002900F0C5810399B9
:103A300014310391039909684E058ED459E708881B
:103A400020F480600004000C088098F8110000F059
:103A5000FE000882C8E90223102088F80200888A44
:103A60000C8B80B240EA0440234C34EA000012D0B0
:103A700000200C900D9001200D910C900C990029C4
:103A800000F094810D9914310D910D990968480544
:103A90003FF563AF2DE798F81330FF2B06D198F868
:103AA00010301BB1132388F8023030E7112388F857
:103AB00002302CE7D8F81400012800F09381022886
:103AC00000F049820E20098B88F80200C8E9022321
:103AD0001DE7062388F8023019E7D8F814000028FB
:103AE00000F07081082388F8023010E70000002001
:103AF00001000300840007008200070002000300A9
:103B0000088820F400600004000C0880088880B257
:103B100040F480600880088880B240F4807008809B
:103B2000032088F80200888A0C8B81B2AB4841EAF6
:103B30000441C8E9022330EA01037FF4E8AE98F8B3
:103B40001230002B40F0D38198F81330FF2B00F097
:103B50004682042388F80230D9E6098889053FF5B2
:103B6000C8AE002388F80230D1E62C4494F8100B3C
:103B700008F098FB064694F8110B08F093FB984A5E
:103B8000B2F8103501339BB28246A2F8103516B157
:103B90003368B2881A83BAF1000F04D0DAF8003023
:103BA000BAF804201A831121304605F067FC112170
:103BB000504605F063FC4FF0090965272EB13368C4
:103BC000B28819690A4240F02881013F00F0228141
:103BD0000CF0A8FF04460D460CF0A4FF001B61EB9F
:103BE0000501052871F10003F6D3E7E7088880B2E4
:103BF00040F4007008804FF6FF3088820121C8E948
:103C0000022388F8021082E6D8F81400002800F099
:103C10007281D8F8184014F8016B0E820138122511
:103C2000C8E90504C8E9022388F802506FE6888ACB
:103C30000C8B81B2694841EA044130EA01017FF40A
:103C400058AE0A2388F8023061E6088880B240F452
:103C500080700880092088F80200888A0C8B81B265
:103C60005E4841EA0441C8E9022330EA01037FF4D7
:103C70004EAEE6E7002401250A940B940B910A95B9
:103C80000A98002800F04A810B9814300B900B988A
:103C9000006846077FF52DAED8F81400032800F021
:103CA0007281022800F24681088820F480600004B6
:103CB000000C0880088880B240F400700880098AEF
:103CC00088F81C40C8E9022388F802501FE600204B
:103CD000012408900990099108940898002800F0A0
:103CE00017810998143009900998006847077FF5F3
:103CF00000AEEFF31185102080F31288088880B29F
:103D000040F400700880D8F818000E8A471CC8F8E4
:103D10001870EDB2067085F311880D8AD8F8181066
:103D20006FF001004E1CC8F818600D70C8E902233E
:103D3000C8F8140088F81C4088F80240E7E5002025
:103D400006900790012007910690069C002C00F039
:103D5000EB80079C14340794079C246864067FF565
:103D6000C8AD0C8AD8F818104D1CC8F818500C7043
:103D7000D8F8141088F81C000139C8E90223C8F8E3
:103D8000141088F80200C2E50F9918310F910F99AD
:103D90000968AEE505991831059105990968A8E506
:103DA00001991831019101990968A2E50D9918311D
:103DB0000D910D9909689CE50399183103910399B8
:103DC000096896E5088880B240F4007008800121F7
:103DD000C8E9022388F8021099E500BF010003003A
:103DE000D82B0020088820F480600004000C088094
:103DF000EFF31184102080F31288088B088880B2BA
:103E000040F40070E4B2088084F311880C2188F833
:103E100002105BE616B13368B2885A830CF082FE5A
:103E200004460D460CF07EFE031B61EB0501052BDD
:103E300071F10003F6D316B13368B2881A830CF01F
:103E400071FE04460D460CF06DFE031B61EB05018F
:103E5000052B71F10003F6D3B9F101097FF4ADAE82
:103E600016B13368B2885A830CF05CFE04460D46E6
:103E70000CF058FE031B61EB0501052B71F10003EB
:103E8000F6D3BAF1000F04D0DAF80030BAF8042003
:103E90005A830CF047FE04460D460CF043FE031B0C
:103EA00061EB0501052B71F10003F6D316B1336800
:103EB000B2881A830CF036FE04460D460CF032FE32
:103EC000031B61EB0502052B72F10003F6D3BAF177
:103ED000000F04D0DAF80030BAF804201A8398F9F9
:103EE0000000441C3FF43DAEFFF7C2FB39E60F2350
:103EF00088F802300BE5088880B240F40070088032
:103F00000121C8E9022388F81C1088F80210FEE499
:103F100009991831099109990968EAE40B9918314E
:103F20000B910B990968E4E40799183107910799F7
:103F30000968DEE4D8F81800098A441CC8F818405B
:103F40000170D8F81410C8F808200139C8F8141006
:103F5000C8F80C30DBE4088880B240F400600880C8
:103F6000EFF31184102080F31288088B088820F466
:103F700080600004000CE4B2088084F311880D21F5
:103F800088F80210A2E5088820F480600004000C84
:103F90000880EFF31184102080F31288D8F81800FD
:103FA0000D8A461CC8F818600570088880B240F475
:103FB0000070E4B2088084F31188D8F81800098AE8
:103FC000441CC8F818400170D8F814100C200239AD
:103FD000C8E90223C8F8141088F8020097E498F89A
:103FE0001030002B3FF4B5AD2BE600BF38B5184DAF
:103FF0009DF814E005EB40144FEA401C94F8B1041E
:1040000000B938BD84F8C324C4F8C43401220023A5
:10401000490005F5966584F8C22484F8CC34049AE6
:1040200084F8C0E4022384F8C114C4F8C82484F8D6
:10403000B23465440CF076FD02460B462846FFF785
:1040400027FC94F8B234002BF4D194F8CC0438BD9A
:10405000D82B002038B5184D9DF814E005EB40141E
:104060004FEA401C94F8B10400B938BD490084F807
:10407000C324C4F8C43484F8C1140023049984F818
:10408000C0E4022205F5966584F8C234C4F8C81469
:1040900084F8CC3484F8B22465440CF043FD024625
:1040A0000B462846FFF7F4FB94F8B234002BF4D10A
:1040B00094F8CC0438BD00BFD82B0020F0B587B0F1
:1040C0000023824A00930193136843F48033136002
:1040D00003E0009BB3F5A04F09D0136803F400334D
:1040E0000193009B01330093019B002BF1D0774B90
:1040F0001B6813F4003318BF01230193019B012BAC
:1041000001D000BFFDE7714B71491A6C714842F054
:1041100080521A640A6842F440420A609A689A60BF
:104120009A6842F400429A609A6842F4A0529A60F7
:1041300058601A6842F080721A601A689201FCD5C1
:10414000654A40F205711160996821F00301996098
:10415000996841F00201A2F580629960936803F0CA
:104160000C03082BFAD1936803F00C03042B00F026
:104170008C80082B00F08E80584D594BC5F80838BC
:10418000524BD5F808189A68564C5748C2F3031298
:104190002A44002692F8242BD140544AC5F8081826
:1041A000E260534A596FA260596B524A21F0800174
:1041B0005963596F41F080715967196B0A431A634B
:1041C0005A6B5A639A6B9A631A6C4B490A431A6486
:1041D000596C4A4A0A435A6402A948F2FF7302938F
:1041E0004FF6FF770396FFF769F800F580600297B6
:1041F000FFF764F800F580600297FFF75FF800F5BD
:104200008060FFF75BF800F58060FFF757F800F576
:104210008060FFF753F800F58060FFF74FF800F576
:104220008060FFF74BF800F58060FFF747F808461D
:10423000FFF7E2F8D4F8FC30029A3149314843F0F4
:104240008073C4F8FC30304BC3F8B01F5E6019684F
:1042500041F001011960D5F808384FF47A71B3FBC9
:10426000F1F3013BB3F1807F2849B2FBF1F2C0F8D2
:10427000882908D24FF0E022F0215361072384F807
:1042800023109661136107B0F0BD144D204BC5F8A3
:10429000083875E753685168104D13F4800F01F02A
:1042A0003F01536814BF1A4A0D4AB2FBF1F1074AA5
:1042B0005268C2F30142C3F38813013201FB03F3D6
:1042C0005200B3FBF2F3C5F8083859E70038024052
:1042D0000070004008544007003C024000000020ED
:1042E0000024F40000ED00E0000002400003FA05A5
:1042F00000000008FF916700FFC9FE103357070058
:1043000055CEACC5E01A0020001000E040420F007E
:1043100000127A0082B0064B002201920193019BA9
:1043200003EB80000190019B196002B0704700BF51
:104330005028004010B51C2007F0B4FF112104469E
:1043400005F09CF84CB12368A2885A83C8200CF071
:1043500017FC2368A2881A8310BDBDE81040C8204E
:104360000CF00EBC704700BF704700BF704700BF25
:1043700010B5124C94F81E3523B9114B4FF480221E
:104380005A6110BD4FF0E022D2F8103D23F0060331
:10439000C2F8103DFEF784FA94F81E35002BECD0DD
:1043A000D4F824359B68DB07E7D5D4F820261368BA
:1043B00023F0030161F307031360DEE7D82B00202D
:1043C000003C01402DE9F04FB34CD4F820355A6938
:1043D000D2078BB002D50BB0BDE8F08F5A699B694C
:1043E00012EA0309F7D0C9F3074319F4002F009329
:1043F00040F0E180009B590743D419F0020F5FFAA7
:1044000089F603D0D4F8203502225A61B9F1000FA1
:10441000C0F2EE8119F4006FC9F3072540F04A811C
:10442000330708D59D4B9E48D3F8403B9847D4F8B6
:10443000203508225A61F70600F1C481EE0600F12A
:104440006F81A90600F1E880009BDA0609D5934B3D
:104450009348D3F8503B9847D4F820354FF4801256
:104460005A61009B9B06B6D58C4B8D48D3F8543BC4
:104470009847D4F820354FF400125A610BB0BDE8CC
:10448000F08FD4F824259369D26913401FFA83FA78
:10449000BAF1000FB1D0DFF81882CDF80C90A8F176
:1044A000180500271AF0010F78D0FEB2D4F82425A1
:1044B00004EB86031069D3F82C15536B8968F3401D
:1044C000DB01DBB203430B4013F00109D9B240F02A
:1044D000AB810A0740F1C881D8F800200823936017
:1044E000994619F0800F59D0D5E94CC0D5F8243140
:1044F000D8F800E0ACEB00018B42DEF8182028BFB2
:104500000B4692B20333B2EB930F47D9D4F824256C
:1045100094F81795323604EB8603CDE901786746A7
:1045200098469446874237D9D5F82431391A9942AA
:1045300028BF194601F1030BD5F828314FEA9B0B30
:10454000B9F1000F10D18AB203329210D8F81C656D
:104550000AD04846013053F8047B37608242F9D1D3
:10456000D5E94C70D5F8283108440B44B842C5F859
:104570002831C5F83401DEF818300AD195F81C113D
:10458000012202FA01F1DCF8342022EA0102CCF81F
:1045900034209BB29B45C5D3DDE901785FEA5A0A16
:1045A00007F1010708F1040805F128057FF47AAF47
:1045B000DDF80C9021E7D4F824359D69DB691D40B6
:1045C0002D0C3FF417AF04F21458DFF8D0B004F507
:1045D000AD660027C24608E06D0807F1010706F145
:1045E000040608F128083FF405AFEB07F4D5F9B24B
:1045F00004EB8103D4F82425D3F868359B6852690D
:104600001340D807DAB200F13F81930740F1678188
:10461000336802229A60DFE7D4F82435D4F82C15E9
:104620009A680868C2F34102022A06BF032262F3B5
:104630000A006FF30A0008605A6842F480725A60F8
:1046400006A8FEF7D9FED4F82025D4F82415D3689F
:10465000079D6FF38D23D36088681249C0F3410032
:10466000014491F8D410032900F05F810E490F48EE
:104670000126294484F8166581424FF04006A4F8CB
:10468000186500F2AC810E2161F38D234FF40051C7
:10469000D3605161D8E600BFD82B00200000002075
:1046A000EC3000205C8A0708401E1BFF3F420F00D1
:1046B0000431002000238DF8133094F826368DF84D
:1046C0001330B64BB648D3F8483B9847D4F8243556
:1046D000D4F82025986894F81E354FF40061516194
:1046E000002B3FF49DAEC2077FF59AAE94F82936B1
:1046F000012B7FF495AE9DF81330032B7FF490AE21
:10470000D4F82036A7491A6842F001021A601A68E4
:1047100042F003021A600B6943F006030B617FE667
:10472000D4F82465D4F820157368002723F001031A
:1047300073600597059B43F020030593059B67F382
:104740008A130593059B0B610B690593BC46964B39
:1047500003E00A690592013B02D0059A9006F8D45D
:1047600094F8152552B1914B03EB820EFF2253F8BA
:10477000040F8260D86B73458260F8D10B2363F31A
:10478000070763F3070C4FF0FF33B3614FF00113DA
:10479000F3617761C6F810C0336885486FF30A1378
:1047A000336094F81725D4F86835012A186100F0B1
:1047B000B5804FF480534B61784B7948D3F8443B34
:1047C00098473EE6D4F820359A6922F010029A61A3
:1047D0001A6AC2F34340022802F00F0100F0B080D1
:1047E000062800F087809A6942F010029A6125E657
:1047F00094F81E353BB1D4F82026136823F003014A
:1048000061F307031360D4F82425644B6448D3F89C
:104810004C1B536823F0010353608847D4F82035BC
:104820004FF000425A61F5E5516BD8F800005B4B40
:104830004FF0010C0CFA07FC21EA0C015163012234
:10484000D3F8383B826031465548984794F817357D
:10485000012B00F0B18019F0020F3FF442AED8F8FE
:10486000003002229A6099E6CB0604D5D8F80030D1
:1048700010229A6092E6480658BF8946EBD5D8F8D0
:10488000003040229A6089E694F8172533680120A9
:104890008242986007D11A69D8F87C33C2F31202B9
:1048A0009B1AC8F88C33DBF8343B5046984794F891
:1048B0001735012B7FF490AE002F7FF48DAE94F866
:1048C0002536052B7FF488AED4F86835384A1A614E
:1048D000384A5A611A684FF080221A607CE6100745
:1048E0007FF57AAEDBF83C3B5046984733680822A8
:1048F0009A6071E601EB810104EBC101D4F8E46533
:10490000D1F8A008C2F30A1202443068C4F8E00AE1
:104910003068C4F8E40AC1F8A02864E7254A5A615F
:104920001A684FF080221A6043E7002184F81615B8
:104930004FF40071A4F81815092161F38D23A5E641
:1049400047F6F07010423FF44EAFC2F30A1201EB8B
:10495000810004EBC00002F1030C5FEAAC0CD0F85C
:104960009468D4F8E4E54FEA810818BF002006D027
:104970000130DEF8007046F8047B8445F8D14144EC
:1049800004EBC101D1F894081044C1F89408D1F89F
:10499000A0080244C1F8A02825E700BF00000020BD
:1049A000EC30002000ED00E0400D0300003100205D
:1049B00018000860B8360020002F7FF44CAF94F840
:1049C0002536042B7FF447AFD4F868352B4A1A619B
:1049D0002B4A5A611A684FF080221A603BE7294837
:1049E000A5F57401A1F51051814203D80D2161F3A1
:1049F0008D234BE6244925482944814203D20C21CA
:104A000061F38D2342E62248A5F18C71A1F5434163
:104A1000814203D80B2161F38D2337E61D491E48DF
:104A20002944814203D20A2161F38D232EE61B49DA
:104A30001B482944814203D2092161F38D2325E6D5
:104A40001848A5F1B771A1F55851814203D2082148
:104A500061F38D231AE6144914482944814203D294
:104A6000072161F38D2311E611491248294481423F
:104A700034BF0621052161F38D2307E61800086085
:104A8000B8360020DFC810002013FBFE20D613002C
:104A9000FF69180000D3CEFE40771B00C05BB3FE59
:104AA000C091210040AC2700C01D6AFE40E13300E8
:104AB000803C36FEE09C41000378022B12D00E4968
:104AC00043680269D1F8180210B41840D1F81042B6
:104AD000D1F80C12931E400A04FB030008445DF851
:104AE000044B7047044B4268D3E9800100EB41005E
:104AF00000EB5220704700BF185700202DE9F84FF7
:104B000012F0020E01D000283CD08A4DD5F8087270
:104B1000002F43D14FF0FF3C874CE146E046E24690
:104B200000262768B84200F0D98094F80EB0BBF197
:104B3000000F4ED0BBF1010F16D1804F06F5817BDF
:104B400007EB0B1B9BF807B01BF0010F0CD11BF000
:104B50007E0F09D15FEADB1740F0B480D4F808B0CB
:104B6000D34501D2DA46B1460136082E04F11004CD
:104B7000D7D1BCF1FF3F38D1B8F1FF3F30D06F4CF7
:104B8000C44633E06B4D95F8B431A5F58054E3B1DC
:104B90000123637002263046BDE8F88FD5E98346CD
:104BA00006FB0744A042B5D395F8B43113B90123ED
:104BB00085F8B431614B012200265A703046BDE8B9
:104BC000F88F95F8B431002BE2D1012385F8B43188
:104BD000DEE7B4460136082E04F11004A1D1C8E77F
:104BE000B9F1FF3F18BFCC4674D0544CD5F898604B
:104BF00004EB0C1841F21809013648F8090041F29B
:104C00001C090CF5817748F809604FEA0718C5F8C8
:104C1000986044F8086004EB07164FF00008C6F8E7
:104C2000048004EB0716B679042ECAD8DFE806F034
:104C3000031952192F0012F0010868D104EB071074
:104C4000D61090F80790032B66F3C71980F80790E9
:104C50005BD94FF6FF70834228BF034604EB071071
:104C60008380BEF1000F12D0D5F89830D5F89C00A3
:104C700001330130C5F89830C5F89C0004EB0C10E6
:104C800041F21C05435104EB0713042098715007AF
:104C900005D504EB0710C37943F00103C371D306B4
:104CA00008D504EB0714E379C3F34502013262F33C
:104CB0004603E371224B012603EB4C230B60304685
:104CC000BDE8F88FB0460136082E04F110047FF4D9
:104CD00028AF4EE700263046BDE8F88F174C06F5A2
:104CE000817704EB071C4FEA07189CF806C0BCF15B
:104CF000000F01D1B44679E7B446D5F89860013683
:104D000044F80860C5F898608BE74346A6E70D4B6A
:104D1000D3F8E03C002BDDD009495D680A4A01EB7D
:104D20004C210023A8470028D4D004EB0714022309
:104D3000A37130E718570020305700201847002093
:104D400030470020E01A0020F107000870B5104E2F
:104D50003378022B0F4B0BBF020AC0F3D412C4B23C
:104D600000F07F04D3F8000282B010440D46002307
:104D7000032201A9FFF7C2FE012807D13378022BD5
:104D8000019B0CBF23F8145043F8245002B070BDAF
:104D900018470020185700202DE9F04FDFF82C812C
:104DA00098F80060032E85B00C46154643D00128C4
:104DB0008CBF00220122022E0B68019269D14FEABA
:104DC0001329DFB24FF4807A0138012820D84FF040
:104DD000010B9D4217D93C4ED6F878211AB1D6F86E
:104DE0009411994258D0D6F8000200234844092271
:104DF00003A9FFF783FE01282CD0022817D020B189
:104E000023689D42E8D82560032005B0BDE8F08FF7
:104E1000F7B12D4B93F8B42112B9012283F8B421D4
:104E20000123022088F8013005B0BDE8F08F022090
:104E300005B0BDE8F08F01288CBF0023012301934A
:104E40000B684FF0800AC3F3D41903F07F07BBE768
:104E5000D346BEE798F800200399DDF804C0022A83
:104E600014D0032AE3D151F8273023F07043B3FA6A
:104E700083F35B0963455F44236821D05B44574556
:104E80002360ECD309F101090027BAE731F81730A4
:104E9000EDE74FF4807AD6E7D6F81012013A02EB2C
:104EA00041224902B2FBF1F21344B3FBFBF20BFBCC
:104EB00012320AB15B449B1A9D4223608CD8A2E750
:104EC000AB42A2D39FE700BF18570020184700202D
:104ED0002DE9F04FDFF86CB19BF800C0BCF1020F78
:104EE000894683B009688246174640F08C800BF5EE
:104EF0008053CEB2D3F80052A6EB010805EB112582
:104F000090444FF480739844B94208F1FF38B8FBDD
:104F1000F3F84CD2A844BCF1030F07EB06040CBF16
:104F200080224FF48072641A9442A8EB050328BFD4
:104F3000144666B994422CBF0A220B2201A92846C6
:104F4000FFF7DCFD012809D003B0BDE8F08F0B228C
:104F500001A92846FFF7D2FD0128F5D19BF800C032
:104F6000D9F80010BCF1020F01F1010323D0B442C3
:104F700010D9019906F18042013A01EB820204390D
:104F800001EB840142F8043F914203F10103F9D19E
:104F9000D9F80010A61B3144BAF1010FC9F800106E
:104FA00021D08F4205F101054FF00006B3D8012052
:104FB00003B0BDE8F08FB442ECD9019806F100428D
:104FC000013A00EB4202023800EB440022F8023FB3
:104FD000904203F10103F9D1A61B3144BAF1010F4C
:104FE000C9F80010DDD1B942DBD1BCF1020F1DD0F0
:104FF00004F18044019B013C4FF0FF3243F8242030
:10500000D9F80010CDE70BF5805301F07F06D3F8F7
:105010000032BCF1030FC1F3D415A6EB01081D4407
:10502000904414BF4FF4807380236CE704F1004474
:10503000019B013C4FF6FF72504623F8142003B049
:10504000BDE8F08F1847002030B50446C06983B032
:1050500010B9012003B030BD0D460023032201A981
:10506000FFF74CFD0128F5D1B4F92030002B0ADA06
:10507000144B93F8B4210AB983F8B401124B0122FE
:105080005A700220E6E7019A012D4FEA431102EB24
:10509000431303D0022D11D1E5255554A268DA61DE
:1050A0002278032A04D100221A775A779A77DA777E
:1050B000626A5A83120C9A8203B030BDE268DA61E8
:1050C000EEE700BF18570020184700202DE9F041F7
:1050D00090F83C30002982B0044614BF0221002120
:1050E000042B7BD8DFE803F0030C3D486900FFF791
:1050F000ABFF012870D1626B002A75D184F83C00A7
:10510000404EDFF808814FF6F77706F5805516E038
:10511000BA424FD867F0B0FD01284FF000011DD111
:10512000206BFFF713FE012818D1019AD5F814124D
:105130002263531E8B4228BF0B46C5F814323278C7
:10514000236B032A01A918469AB2E1D1434531D80D
:1051500067F092FD01284FF00001E1D002B0BDE8F8
:10516000F081426B04F130010020FFF7B1FE01280D
:1051700032D1032384F83C302348E16AD0F89431DB
:10518000D0F81022C0F894115B1A02FB03F3D0F898
:10519000782102EB4322C0F87821D0F87C2102EB81
:1051A0004323C0F87C31002100F5B870FFF74CFFB5
:1051B000012811D1042384F83C3094F82830042BC2
:1051C00004BF002384F82830A36B8BB12046984796
:1051D000012002B0BDE8F0810228BFD194F8283048
:1051E000042B09D00220B9E7022384F83C30B9E748
:1051F000012002B0BDE8F081002384F828300220AD
:10520000ACE700BF1847002018570020F7FFFF0F3A
:1052100038B590F834300446052B43D8DFE803F066
:105220001E033C0F185E006B4FF0FF31FFF78EFD41
:10523000012837D1E06AB8BB032384F83430002159
:105240002046FFF701FF01282CD1042384F83430D5
:1052500094F82830082B2BD0012038BD204DD5F8EC
:10526000082200F1300102320120FFF795FD0128EC
:1052700023D00238C0B2012814D8052384F8343072
:1052800094F82830082B04BF002384F82830012329
:1052900085F8B531022038BDC06A216BFFF756FD95
:1052A0000128C9D0002038BD022384F83430F4E747
:1052B000002384F82830012038BDE368D5F81012A7
:1052C000D4E90B2003EB4123C5F81402C4E90330F1
:1052D00002B96062012384F83430A5E7004DCFE7BE
:1052E0001857002010B590F838300446032B4DD8DD
:1052F000DFE803F0022F38432B4AC068117802F52B
:1053000080530329D3F81012D3F894210CBF4FF027
:10531000800C4FF4807C01FB0CF100EB4120C4E9D0
:105320000302D3F87801A0EB4120C3F87801D3F849
:105330007C01A0EB4121E06AC3F87C1102EB0C0177
:10534000C3F89411C4E90C2148BB6262012384F8BC
:10535000383016480021FFF777FE012811D10223CB
:1053600084F83830626B04F130010120FFF7B0FDA2
:10537000012806D1032384F8383000212046FFF7A6
:1053800063FE431EDBB2012B01D910BD022094F84D
:105390002830062B04BF002384F8283010BDA2EB70
:1053A0000C022263D2E700BF184700208858002073
:1053B0002DE9F0434368C3F308020A44B2F5007FC5
:1053C00083B004460D4605D22B446360012003B030
:1053D000BDE8F08390F91A20501C0AD0444902F528
:1053E000817201EB0212D1796FF30001D171FF22BA
:1053F000A27694F91B20511C16D03D4802F581710C
:1054000000EB011200EB0111D279C879C2F3450219
:10541000012A86BF02F1FF3202F03F020022FF267E
:1054200062F34600C871E67694F800C0BCF1020F42
:10543000CAD0DFF8C480D8F81022B5EB422F4FEA6B
:10544000422915DCD8F818721F407A42AA420FDCB4
:10545000EA194A4510D220690028B7D0244A1278A8
:10546000032A40D080B24FF6F7729042ACD9ADE734
:10547000002003B0BDE8F083227E206912F0080608
:1054800026D0D8F89421411C8A4213D300D10021A0
:105490004B44A5EB0905DB1BBCF1020F60613D44E9
:1054A000216163600846D7D1D8F82022B3EB422FA0
:1054B0008AD38BE798F8B42122B9012388F8B43154
:1054C000636820690A4A0126567094F800C0DFE735
:1054D00001A967F0D1FB0128CAD10199636894F84A
:1054E00000C02069D4E7034A90427FF66DAF6DE7B4
:1054F00018470020F7FFFF0F185700202DE9F0474D
:1055000090F8384082B00546032C00F2AD80DFE809
:1055100004F00219730BFFF77BFE012810D002285C
:105520000AD1032385F838302B6C002085F8280039
:10553000002B71D098470224204602B0BDE8F087C6
:1055400085F838002B78022B62D0484A6B68D2F875
:10555000182203EA0208C8F34F282846FFF7ACFADE
:10556000424F0646A8EB0008A7F5805901A9022280
:1055700000233046FFF7C2FA08EB060401281FFAA1
:1055800084FA4FF400724FF000010446D4D1019820
:1055900071F038FAEB694FF40071284613B16B686B
:1055A000002B3DD0D7F810325A1E924506F1010665
:1055B0000DD2FFF7FDFE0028D8D197F8B43113B90A
:1055C000012387F8B431012389F80130CEE7C3EB1A
:1055D000C353590201F500712846FFF7E9FE40B9AF
:1055E00097F8B43113B9012387F8B431204B012265
:1055F0005A70022385F838302B6C002285F8282059
:1056000063B1284698470124204602B0BDE8F087E0
:105610006B68C3F34F28A0E702248DE701248BE7D2
:10562000019B4FF020324FF02E0E4FF0100C1A60FD
:105630005A6083F800E0C3F807206C6A1A625A6265
:1056400083F80BC0C3F8272083F820E083F821E01B
:10565000EA6B5C835A8724FA0CF422FA0CF29C82DF
:1056600083F82BC09A869DE7002465E71857002031
:10567000184700202DE9F041B1F904300F2B82B01A
:105680000E460446174635D02046FFF715FA94F922
:105690001B80B8F1FF3F3ED0554B41F2180203EB9F
:1056A00008118A58904211D1183303EB4825B3886A
:1056B00001331BB205EB4315B38020463D60FFF775
:1056C000FBF93060012002B0BDE8F08103F58052A3
:1056D00092F8B41100296AD001225A702278022A65
:1056E00069D02369002B50D1002301203B6002B018
:1056F000BDE8F0814FF40071FFF75AFE002852D048
:105700004FF6FF73B3802046FFF7D6F994F91B805C
:10571000B8F1FF3FC0D12278022A54D02369002B70
:10572000DDD03349097803290EBF32499BB24FF6C9
:10573000F7718B4294BF00230123002BCFD138B9DE
:105740002D4A92F8B431002B4ED0294B01225A70C9
:105750000023112201A9FFF7D1F9012842D1019DAF
:10576000264BEB1A48BF03F2FF13B3F5805F4FEAF5
:10577000632230D3204A92F8B43113B9012382F85E
:10578000B4311B4B01225A7027E0194A1278032AC0
:105790000EBF184A9BB24FF6F772934294BF002394
:1057A0000123002BA0D1002002B0BDE8F08101212F
:1057B00082F8B41190E7104A6368D2F82022B3EB64
:1057C000422F91D2EFE70C4A6368D2F82012B3EB74
:1057D000412FB4D3F1E74FFA82F884F81B80002DF3
:1057E0007FF465AF22787AE7012382F8B431ACE721
:1057F00018470020F7FFFF0F185700203047002000
:105800002DE9F04790F8303086B00446042B54D888
:10581000DFE813F005000E005600F8004F00C44802
:1058200068F02AF84FF6FF720123228484F83030A2
:10583000DFF8FC8204F11C0501AE04F131093246A7
:1058400029464046FFF716FF012800F00281022892
:1058500033D1B84901F5805595F9D221531C0AD0AE
:1058600002F5817201EB0212D3796FF30003D37159
:10587000FF2385F8D23195F9D3315F1C16D003F59B
:10588000817301EB031201EB0313D279D979C2F3CF
:105890004502012A86BF02F1FF3202F03F020022D8
:1058A00062F34601FF22D97185F8D321042384F8DD
:1058B00030300020E36A2070984706B0BDE8F087DA
:1058C0009D4D95F8E031002BF7D1994F04F11C095B
:1058D00001AE4FF00908324649463846FFF7CAFE86
:1058E000012840F021810198002800F0FD80037814
:1058F000E52B01D0002BEED1904A821A48BF02F26C
:10590000FF12B2F5805F4FEA622380F05C81894923
:105910001B018B4A13449A7B042A0CD0D5F898209B
:105920000132C5F898205A6004229A73D5F89C3049
:105930000133C5F89C3095F9D2315E1C0AD003F5CD
:10594000817301EB0313FF2285F8D221DA796FF31B
:105950000002DA7195F9D3315A1C18D003F581731E
:1059600001EB031201EB0313D279C2F34502012AC2
:105970004FF0FF0188BF02F1FF3285F8D311D979CA
:105980008CBF02F03F02002262F34601D97120224F
:10599000002171F037F8019BD4F83120D4F835108C
:1059A00059601A60B4F8392094F83B1099721A8142
:1059B000019B627EDA7203A802F094FF002800F0D7
:1059C000E5809DF80E509DF80F10BDF80C00019B6E
:1059D0009DF8102041EA4511A0F2BC7041EA402137
:1059E0008DB219829DF81110D20242EA41129DF83F
:1059F000121042EA510290B2DA8103221D83D8824A
:105A000084F83020237E980608D5E069002311220F
:105A100002A9FFF773F801287FF44FAF204667F023
:105A20002BFF2369002B00F08D80237E03F0F7020B
:105A300013F00403227640F09380122A00F0B18024
:105A40000022E36A84F828202046984706B0BDE883
:105A5000F087019F002F00F0C2803B78002B00F000
:105A6000BE8097F80BA01AF0080F7FF4E8AE0B2267
:105A70004946384670F060FF00287FF4E0AE637E50
:105A80008AEA0303D90640F1EB802A4901F58055E3
:105A900095F9D2315A1C0AD003F5817301EB031337
:105AA000FF2285F8D221DA7960F30002DA7195F9E4
:105AB000D321571C3FF4FAAE02F5817201EB0213B9
:105AC00001EB0211DB79CA79C3F34503012B86BFD1
:105AD00003F1FF3303F03F03002363F34602FF2388
:105AE000CA7185F8D331E1E695F8B831022B3FF45D
:105AF000DDAE95F8E031002B7FF4D8AEC5E97D33FB
:105B000085F8F03185F8EC31D5F8CC31C5F8E431C1
:105B1000D5F8143285F8E081C5F8E8313846FFF74A
:105B2000EDFC01283FF4D7AE02283FF4BFAEC4E637
:105B3000D058002018470020185700203047002078
:105B400030570020237E19077FF57AAF664B93F814
:105B50009821002A7FF4B1AE072283F898216FE7DD
:105B6000A568E66A002384F8283029462046FFF716
:105B70001FFC00286ED194F82830002B7FF49DAED6
:105B80000223C4E90B6584F8283096E6019B6FF088
:105B90007E01472219745A749873D87344F2817540
:105BA0002BE7626AE16AA163042084F82800C4E953
:105BB0000B22C4E9023384F83C30636363622046FD
:105BC00067F05AFE79E695F8B43113B9012385F8E8
:105BD000B431464901234B706FF00F0399E64349F6
:105BE00001F5805595F9D2315F1C0AD003F5817318
:105BF00001EB0313DA796FF30002DA71FF2385F802
:105C0000D23195F9D3315E1C16D003F5817301EBC7
:105C1000031201EB0313D279D979C2F34502012AA9
:105C200086BF02F1FF3202F03F02002262F346011A
:105C3000FF22D97185F8D321237ED8067FF536AEB1
:105C40002B4867F019FE4FF6FF720223228484F876
:105C5000303036E6002E3FF430AE2046B0472CE61A
:105C6000BA8A7B8B204D43EA02436362D5F8102247
:105C7000FB69A3605202B3FBF2F102FB113109B1DF
:105C800013445B1AE36084F819A095F9D2311749DF
:105C90005E1C0AD003F5817301EB0313DA796FF30D
:105CA0000002DA71FF2385F8D23195F9D321501C17
:105CB00016D002F5817201EB021301EB0211DB79C0
:105CC000CA79C3F34503012B86BF03F1FF3303F009
:105CD0003F03002363F34602FF23CA7185F8D331E3
:105CE000032384F830308DE6185700201847002031
:105CF000D058002010B5037890F818C0023B012B53
:105D0000044602D91CF0060F6AD11CF0200F44D1C2
:105D100094F91A30591C0AD0384A03F5817302EB02
:105D20000313FF21DA796FF30002DA71A17694F997
:105D30001B305A1C16D0314903F5817301EB031255
:105D400001EB0313D279D979C2F34502012A86BF48
:105D500002F1FF3202F03F02002262F34601FF220D
:105D6000D971E2761CF0080F0ED0254B93F89821DC
:105D7000072A06D093F8B421002A3BD01F4A0121FC
:105D80005170002283F89821E26A0023237084F87E
:105D9000283022B3BDE81040104700231949E069BC
:105DA0001A018A58904206D00133082BB0D01A014C
:105DB0008A589042F8D1114903F5817301EB03121F
:105DC000D279C2F34502012A12D9013A02F03F0208
:105DD00001EB0313D97962F34601D97198E710BD3D
:105DE0000121FFF731F90128F9D194F818C08CE7A7
:105DF0000022EDE7012283F8B421BFE71847002015
:105E000018570020305700204FF0FF302DE9F041A7
:105E1000344A354D0446002304E00133082B02F1D7
:105E2000100216D011780429F7D103F5817105EB22
:105E30000111C979CF07F0D4661C52F80A1C01D0B1
:105E40008142EAD21C460133082B084602F11002B7
:105E5000E8D1631C02D10120BDE8F081224DDFF8BA
:105E6000988004F5817705EB07139988F9B91F4EDF
:105E7000D8F8E03C06EB442123B3D3F80C801C4A4D
:105E800041F2180305EB0414E0580023C047C8B1E1
:105E9000022824D106F6E87605EB0715D6F89C30E3
:105EA0000122013BC6F89C30AA710020D4E7D8F843
:105EB000E03C3BB19A6841F2180005EB0413185816
:105EC0009047D4E70B4BD3F89C2005EB0715032034
:105ED000013A0121C3F89C20A87183F8A01000208A
:105EE000BDE8F0813E5700201847002030470020D1
:105EF0006908000818570020E01A00202DE9F04F2B
:105F000090F82830013B83B00446082B0BD8DFE81B
:105F100003F0383C1E2305290A2E33000121FFF728
:105F2000D5F8012802D003B0BDE8F08F2378002215
:105F300084F82820002BF6D0D4E901138B4238BF17
:105F40000B46226CA360032184F82810E2622046ED
:105F500003B0BDE8F04FCDE6002103B0BDE8F04F3F
:105F6000FFF7B4B803B0BDE8F04FFFF7BBB903B01B
:105F7000BDE8F04FFFF74CB903B0BDE8F04FFFF7B5
:105F8000BDBA03B0BDE8F04F3AE4534F4368D7F8C9
:105F90001852016BD7F810221D406818B0EB422F41
:105FA0004FEA42269C46C0F0938094F800E0DFF868
:105FB0002C91A7F5805A4FF6F778BEF1020F14D056
:105FC0002069002857D1D4F804C0A368E26A634569
:105FD00038BF63460021A36084F82810002AA2D0AD
:105FE000204603B0BDE8F04F1047D4F804C0D7F8FE
:105FF0002022BCEB422FE8D22069227E12072CD54A
:10600000D7F8942100F1010C624522D297F8B4210F
:1060100022B9012387F8B4316368216B01228AF821
:10602000012094F800E0891B294433445B1B8E4215
:10603000C4E904C0636021639C464FF00005BCD9ED
:10604000BEF1020F3ED020690028BED0DFF890B02C
:106050001FE0E8D14FF0000CE5E701A966F00CFE67
:1060600001287FF460AF2069DDF804C094F800E0F7
:106070006368216BD7E79AF80020032AD3461AD029
:1060800082B2424594BF00220122002AB5D0D4F842
:1060900004C09BF80030032B0EBF104B80B24FF6AC
:1060A000F773984294BF0020012000288DD18C44C2
:1060B000C4F804C089E7484594BF00220122002AA1
:1060C0009BD0E4E7D7F82022B3EB422FEFD37CE755
:1060D00094F800E0B4E700BF18570020F7FFFF0F67
:1060E0001847002010B5184C18484422002170F0C1
:1060F00089FC237804F580544FF6FF70D4F81C22F5
:10610000A4F8D201022B4FF0030118BF03234FF074
:10611000100C84F8D01104F5DC700021C4F8C821FB
:1061200084F8B831C4F8DC2184F8D1C1FFF740F914
:1061300038B994F8E03123B9C4E97933022284F8FC
:10614000E021012010BD00BF18470020D0580020DA
:1061500070B51A4D1A4BC5F8083B1A4B85F8141B3D
:10616000002683F8906905F60833C0E954330D23FF
:106170000446C0F8583140F20113C0F85C6100F5E4
:10618000A271A0F8443169F005FDE378C4F8B46366
:106190001F22C4F8B023012205F587659342C4F895
:1061A000A853A4F89C2308BFC4F8AC5304F5677146
:1061B0002046BDE8704069F0EDBC00BFD82B002040
:1061C00055534253E01A0020F0B50B7813F06006E7
:1061D00083B00C46054633D0202E2DD14A78FE2AB6
:1061E0006BD0FF2A63D14A88002A40F08B80CA888E
:1061F000002A40F08780190600F184806148624BD4
:1062000080F89029C5F8B423EA78012183F858145E
:10621000A5F89C1303F587631F21012AC5F8B01365
:10622000C5F8A83305F5677108BFC5F8AC33284633
:1062300069F0B0FC002600E00026304603B0F0BD57
:106240004B780A2B6AD00B2B63D0012BF5D18B88AE
:10625000D9B21B0676D40196019BC06843F01003A7
:106260000193019B036103690193484B03E00269B9
:106270000192013B02D0019AD206F8D42846424F3F
:1062800069F078FB022321794022284669F0A4FBBB
:1062900097F85834022B6DD094F90420002ACCDAF8
:1062A000012BCAD001212846FFF752FFC5E766F04F
:1062B0006FFD0226304603B0F0BD4E8816BBCC8879
:1062C000012C1FD118061DD52F4FD7F870349B69AC
:1062D0009847C0B287F8180BA0B1022307F6183709
:1062E00085F811314FF48073C5E94E44C5E94A770A
:1062F000C5E94C46A5F81C3105F58E71284669F0B4
:10630000DBFB9AE7284666F043FD0226304603B0E1
:10631000F0BD1D4B4A8883F8192B8EE7022280F8C6
:1063200011214FF48072A0F81C21194A0123C0E901
:106330004E33C0E94A22C0E94C3600F58E7169F04F
:10634000BBFB7AE70096009BC06843F020030093F4
:10635000009B61F38A130093009B03610369009320
:106360000A4B03E002690092013B87D0009A97062E
:10637000F8D483E78121284669F0C2FA002387F820
:1063800058345AE7E01A0020D82B0020400D0300B3
:10639000F136002010B50D4B93F89039022B07D041
:1063A000033B012B02D80021FFF7D2FE002010BDD5
:1063B000074B93F84514044666F094F80028F5DA84
:1063C00001212046FFF7C4FEF0E700BFE01A0020DD
:1063D000D82B0020F8B5404E96F89059074655B195
:1063E000012D06D13D4B93F8451466F07BF800284B
:1063F00032DB0020F8BD394CB0F8B433D4F83C247B
:10640000C4F80C2B1F2BD4F84024C4F8102B08D14F
:10641000334BD4F838249A4203D194F84514012917
:106420001FD994F81A3B04EBC3020133DBB2042BEF
:106430004FF0050108BF002382F81C1B4FF40051E8
:1064400084F81A3B38460223C2F8201B84F85834DB
:10645000FAF7C8FE0020F8BD29463846FFF778FE57
:10646000C7E794F84634013B0F2BDAD866F03AF8C8
:10647000002827DB96F89039013B022BB9D9B4F8F4
:106480003C3B1BB3042286F89029164AC7F85C519E
:10649000C7E95422D4F8402484F8145B934228BFFF
:1064A0001346D4F8102BC7F8583140F20111A7F861
:1064B0004411D31A07F5A2713846C4F8103B69F0AD
:1064C00069FB96E73846FAF78DFE92E7194638469B
:1064D000FFF73EFE8DE700BFE01A0020D82B00201A
:1064E0005553424318370020704700BF704700BF24
:1064F000D0ED007AD0ED036A30EE677AE6EE877A67
:10650000B0EE670AC0ED007A704700BFD0ED017AA7
:10651000F5EE407AF1EE10FA09D1DFED0E7A60EE79
:10652000A70AB7EE007AC7EE207AC0ED017A31EE05
:10653000277AD0ED007A80ED021AC1EE076A30EEBC
:10654000677AC0ED036AE6EE877AB0EE670AC0EDBF
:10655000007A7047DB0FC94090ED017AD0ED036AF5
:10656000D0ED027A30EE470AA6EE807A90ED000A6E
:1065700080ED017A37EE676AE6EE867A37EEC07A0A
:10658000C0ED027AA6EE870A80ED000A704700BFD0
:10659000D0ED056AD0ED017A90ED007A90ED066AB3
:1065A000D0ED025A90ED035A80ED050A66EEA77A07
:1065B000C0ED066AE7EE007A90ED077AE5EE867A9E
:1065C00090ED086AD0ED045A80ED087AE5EE477A3E
:1065D000E5EEC67AB0EE670AC0ED077A704700BFF5
:1065E000D0ED057A90ED006A90ED037AD0ED025A75
:1065F000E6EE007AF0EE406AB0EE670A90ED016ACE
:10660000D0ED047A27EE407A67EEC07AA6EE267ABD
:10661000E5EEA67A90ED066AC0ED067A36EE077AC8
:1066200080ED057A704700BF03685A1C026019703C
:10663000704700BF03685A1C02601970704700BFA2
:10664000024B186803681B68184700BF40590020B8
:10665000007970470079C0F3401070470079400915
:10666000704700BF90F83C20034602F0FF0012B1D3
:10667000002283F83C2070474FF480538381704799
:106680004FF40063838170474FF400638381704748
:106690004FF40063838170474FF400638381704738
:1066A0004FF40063838170474FF400638381704728
:1066B000074B10B403F11001002453F8042B82425D
:1066C00008BF43F8044C8B42F7D15DF8044B704788
:1066D0004459002070B5374C638CA08AB4F92C5013
:1066E000B4F92660B4F91AC0C01A238C00FB03F376
:1066F000B4F92A0005EBE335C00290FBF5F000EB9E
:10670000E330A0F57A6EB4F9243020630EFB0EF569
:106710002D1305FB06F605FB03F3B4F91C500EFB25
:106720000CFC4FEAEC2C0EFB05FE1B14B4F91850C0
:106730000CEBE62C03EB6E330CEB850C0233B4F957
:106740003450A66BE48B9B1003F500430CFA05FC58
:1067500004FB03F30CF1020C4CF25034A6EBAC0C2E
:106760002C4104FB0CF4002C4FEAD333ABBF640084
:10677000B4FBF3F3B4FBF3F35B0089B11C120E4DD1
:1067800004FB04F440F6DE3606FB04F403FB05F5D7
:10679000241404EB254404F6CF6403EB24130B60AC
:1067A0002AB100EB80004000083000111060012089
:1067B00070BD00BF4059002043E3FFFF0120704738
:1067C000012070472DE9F84F6E4DD5F83CC0B5F863
:1067D0004000B5F94A90B5F846E0C0EB2C1303FB36
:1067E00003F4B5F94430241303FB04F44000B5F975
:1067F0004230C0EBEC0003FB00F0A41304EBE024F8
:10680000B5F94830AC650F46A4F5FA31164683FB5E
:10681000013281FB018C12034FEAE97B42EA1352F9
:106820004FEA033A09FB0CF308FB0B3BA9FB0839C1
:10683000D9441B0A43EA096313EB0A0342EB2922FA
:1068400002F50042A3FB0E390EFB029E4FEAEE73E7
:106850004FEA6E0253EA6E0E4FF0000000F08580A2
:10686000B5F9509009FB0CFEB5F94EC08CFB011C2C
:106870004FEAE97A4FEA4C4C08FB0AEE4CEAD13C6D
:10688000A9FB0898490411EB0901F04448EB0C0CF2
:106890004018E96DC1F58019B5F94C1009F0004EAA
:1068A0004FEAC978B8EB00080CEBC1014EEA590E6B
:1068B0006EEB010E18EB080C4EEB0E011CEB080CF6
:1068C0004EEB01014FEA81194FEA8C1049EA9C69AD
:1068D0001CEB000C41EB0901890041EA9C714FEA75
:1068E0008C0C1CEB080C4EEB01014FEA8C0089006C
:1068F00010EB080041EA9C714EEB01016AF05AFA74
:10690000B5F95620B5F954E0B5F952504FEA61385F
:10691000430B43EAC14302FB08FC4FEAE27903FB65
:1069200009C9A2FB032CCC4402FB08F803FB0C882A
:10693000A2FB032CC444520E42EACC12121841EBC3
:106940006C6C4FEAEE730EFB01F103FB0011AEFB22
:1069500000300144DB0C43EA4133D0184CEBE141F9
:10696000000A40EA016000EB05100FB1000A386030
:1069700026B104EB84048034241234600120BDE885
:10698000F88F00BF4059002031B10A4BD3ED1E7A79
:10699000FDEEE77AC1ED007A52B1064B9FED067A23
:1069A000D3ED1F7A67EE877AFDEEE77AC2ED007AC3
:1069B00001207047405900200000C8422DE9F04FE7
:1069C000634D85B0B5F88E30D5F88000B5F88C8071
:1069D00001911B02B5F88810B5F88A60B5F89040AF
:1069E000C01A67EB07074FEA014EA8FB001CB5F879
:1069F000863008FB07CCC90941EA4C6111EB0E0156
:106A000093464FEAC332A6FB003E06FB07EE4FEA71
:106A1000132343EA0E634FEAEC1C4CF1000C9B1865
:106A2000A4FB002604FB07644FEAD25242EA442248
:106A30004FEA2E2E4FEAE4544EF1000E12F5FA6999
:106A400044F10006B9F5FA6F029476F1000403965A
:106A500031DA029CA2FB02A602FB04F806EB480412
:106A60004FEA84084FEA8A0616EB0A0648EA9A7843
:106A700044EB08084FEA560A4AEAC87AB608354C89
:106A8000B1EB0A0146EA88766CEB680C9B1B039E0F
:106A90006EEBA80EA1454FF0FF3476EB040427DB24
:106AA00000FB07F7A0FB000202EB4707C00F40EA1C
:106AB0004700B9EB0009019C8CB1D5F89400A0FB0C
:106AC000033200FB0E2E5B0D43EACE235B1A4FEA26
:106AD0006E5E6EEB0C0CDB0B43EA4C432360BBF1A8
:106AE000000F01D0CBF80090012005B0BDE8F08F79
:106AF00040F6AC56029C921944F1000402FB04F4E7
:106B0000A2FB028202EB4404E6004FEAC802B8EBA3
:106B1000020246EA587664EB060651184CEB060C66
:106B200018EB080644EB040A16EB080644EB0A0AC5
:106B30004FEA8A0A4AEA967AB600B6EB08026AEB8E
:106B40000404520842EAC4729B1A6EEB640EA7E773
:106B50004059002024FAFFFF0120704710B4114B68
:106B6000114C1B68D4F898001B1AFA2B0FD811B1DE
:106B7000D4F8A0300B6032B1D4F8A43013600120F7
:106B80005DF8044B704701205DF8044B7047074ADD
:106B90001368002023F0040384F89C0013605DF860
:106BA000044B70476C240020405900200000001066
:106BB000064B00220021C3F8A820C3F8AC20C3F87C
:106BC000B020C3F8B4100120704700BF4059002026
:106BD000104B114A1B68D2F8B4105B1AFA2B16D866
:106BE000D2ED2A6A92ED2B7AD2ED2C7AFDEEE66A8E
:106BF000BDEEC77A16EE903AFDEEE77AC38617EE41
:106C0000103A038717EE903A43870120704700201F
:106C1000704700BF6C2400204059002038B514464E
:106C2000002944D0344B9FED356AD3ED2E7AB3F969
:106C3000D02093ED300AB8EEE77AD3ED357AC7EE7F
:106C4000066A0D4604EE902AB3F9CC20F8EEE77AF6
:106C500005EE902AB3F9CE2087EE864AF8EEE44A94
:106C600005EE102AF8EEE55AB3F9CA20D3ED317AD1
:106C7000B3F9C830E6EEA45A06EE102AB8EEE77A69
:106C8000B8EEC55AB8EEC66AA6EEA57AA6EE856A33
:106C900007EE903AB8EEC00AF8EEE77AA6EE870A59
:106CA000E6EE867AA4EE270A6AF002FF28600CB3AB
:106CB000114BDFED125A93ED357AB3F9BE20B3F9DB
:106CC000BC309FED0F0AB8EEC76A07EE902A86EE39
:106CD000257A06EE903AF8EEE77AF8EEE66A67EE85
:106CE000277AB6EE006AE6EE867A27EE800A6AF028
:106CF000DFFE2060012038BD405900200000F04A2E
:106D00000000C8422DE9F0410446D0E900301344A8
:106D100083421DD88E188E4217D00D4604F10C0800
:106D2000002701E0AE4210D023695A1C226123449F
:106D300015F8010B1873042AF4D141462046FBF7DD
:106D4000DBFDAE42C4E90470EED16069BDE8F081BC
:106D50004FF0FF30FAE700BF70B50446234894F9BE
:106D6000103003EB8303154650F82300A3689A07FD
:106D700082B00CD5019069F057F80198294669F066
:106D800053F8A3689B0717D5012002B070BD636953
:106D900013B11A689B885383154B164A1B685668B3
:106DA0004FEAC30C144BA3FB0C3C4FEA9C1C5368EA
:106DB0009B1B9C45FBD2DDE70D4B0E491A680E4B21
:106DC0004FF4FA7000FB02F2A3FB0232486892090A
:106DD0004B681B1A9A42FBD26369002BD4D01A6805
:106DE0009B881383012002B070BD00BF60000020AB
:106DF00068240020001000E0D34D621010B5046834
:106E00002379012B84B010D0022B0BD1A368DB07B0
:106E10004FF0F0024CBFFF217F21204604B0BDE8B7
:106E2000104099E7002004B010BDA268617C94F97D
:106E3000100002F0010201920DF10F020092F02405
:106E4000FF228DF80F40FDF7D1F804B010BD00BF50
:106E500010B504682379CA4341EA0211012B84B0BA
:106E6000CAB20ED0022B09D1A368DB074CBFD221D6
:106E70005221204604B0BDE810406DE7002004B068
:106E800010BD8DF80F20A268617C94F9100002F00B
:106E900001020DF10F04CDE90042D222FDF7A6F860
:106EA00004B010BD10B504682379012B84B010D054
:106EB000022B0BD1A368DB074FF0B4024CBFFF21BC
:106EC0007F21204604B0BDE8104045E7002004B013
:106ED00010BDA268617C94F9100002F001020192D9
:106EE0000DF10F020092B424FF228DF80F40FDF740
:106EF0007DF804B010BD00BF10B504682379012BE4
:106F000084B00FD0022B0AD1A368DB070A462046C3
:106F10004CBFA521252104B0BDE810401CE700208E
:106F200004B010BDA26894F910008DF80F1002F0A3
:106F30000102617C0DF10F04CDE90042A522FDF7AD
:106F400055F804B010BD00BF10B504682379012BBB
:106F500084B010D0022B0BD1A368DB074FF0960250
:106F60004CBFFF217F21204604B0BDE81040F3E66E
:106F7000002004B010BDA268617C94F9100002F0FA
:106F8000010201920DF10F0200929624FF228DF86A
:106F90000F40FDF72BF804B010BD00BF10B504681A
:106FA0002379012B84B00FD0022B0AD1A368DB0711
:106FB0000A4620464CBF8721072104B0BDE8104097
:106FC000CAE6002004B010BDA26894F910008DF844
:106FD0000F1002F00102617C0DF10F04CDE90042B7
:106FE0008722FDF703F804B010BD00BF10B5046898
:106FF0002379C901012B84B0CAB20AD0022B05D172
:107000007821204604B0BDE81040A5E6002004B079
:1070100010BD8DF80F20A268617C94F9100002F079
:1070200001020DF10F04CDE900427822FCF7DEFFEA
:1070300004B010BD10B504682379012B84B010D0C2
:10704000022B0BD1A368DB074FF055024CBFA521E3
:107050002521204604B0BDE810407DE6002004B0A4
:1070600010BDA268617C94F9100002F00102019247
:107070000DF10F0200925524A5228DF80F40FCF768
:10708000B5FF04B010BD00BF10B504682379012B13
:1070900084B010D0022B0BD1A368DB074FF02E0277
:1070A0004CBFF4217421204604B0BDE8104053E6E3
:1070B000002004B010BDA268617C94F9100002F0B9
:1070C000010201920DF10F0200922E24F4228DF89C
:1070D0000F40FCF78BFF04B010BD00BF10B5154B7F
:1070E00004689A8E237992013432012B84B0D2B293
:1070F0000ED0022B09D1A368DB074CBFF421742109
:10710000204604B0BDE8104026E6002004B010BDC3
:107110008DF80F20A268617C94F9100002F0010242
:107120000DF10F04CDE90042F422FCF75FFF04B03B
:1071300010BD00BF4059002010B504682379012B11
:1071400084B00ED0022B09D1A368DB074FF03102C7
:107150004CBFF42174212046FFF7FEFD012004B04E
:1071600010BDA268617C94F9100002F00102019246
:107170000DF10F0200923124F4228DF80F40FCF73C
:1071800035FF012004B010BD10B504682379012B30
:1071900084B00BD0022B06D101225821204604B026
:1071A000BDE81040D8E5002004B010BDA26894F9F5
:1071B0001000617C8DF80F3002F0010201920DF198
:1071C0000F0200925822FCF711FF04B010BD00BF5F
:1071D00010B504682379012B84B00BD0022B06D1A3
:1071E00001224821204604B0BDE81040B4E500204B
:1071F00004B010BDA26894F91000617C8DF80F30C6
:1072000002F0010201920DF10F0200924822FCF7F8
:10721000EDFE04B010BD00BF10B504682379012B4A
:1072200084B00BD0022B06D11A460821204604B0A8
:10723000BDE8104090E5002004B010BDA268617C5C
:1072400094F9100002F0010201920DF10F02009278
:10725000022408228DF80F40FCF7C8FE04B010BDD0
:1072600010B504682379012B84B00BD0022B06D112
:1072700001220821204604B0BDE810406CE5002042
:1072800004B010BDA26894F91000617C8DF80F3035
:1072900002F0010201920DF10F0200920822FCF7A8
:1072A000A5FE04B010BD00BF2DE9F0410C4E3568BD
:1072B00073691D4011D0DFF82C800127B5FA85F4E1
:1072C000C4F11F0408EB840307FA04F4D3F8D800D0
:1072D00003689847A5437461F0D1BDE8F08100BF11
:1072E000003C0140405900202DE9F041634CD4F8A6
:1072F000180190B028B1624A0321FBF75FFCD4F873
:107300001801604E0021FBF7D5FCD4F818516F68C6
:107310003B6900224FEA133E4FEA132C4FEA421812
:1073200006EB421056F808308EEA13318CEA13232C
:1073300001F0030103F00F0351EA030402F101021B
:1073400006D0102AEAD10020E86010B0BDE8F08134
:10735000027F3B68E8601AB1204610B0BDE8F081BA
:10736000B3F844206FEA42426FEA524292B2A3F865
:1073700044201A8892B242F080021A80BA79198C9D
:1073800012F0040F7A79404F17F802C014BF04229C
:10739000012202FA0CF292B289B221EA02011984A6
:1073A000198C89B20A431A841A8892B242F00102F7
:1073B0001A804268354B9A42354A136B0CBF43F42E
:1073C000001343F48003136306EB080307229A8338
:1073D000294665F003FFEB689868FBF7D9FEEB6878
:1073E0009868036823F001030360FBF7D1FE0023D4
:1073F0006A680693CDE90C33CDE90E330A935379CD
:10740000032B06D8DFE803F035312D02136803F1B2
:107410004004137CE96807EB83071E4B88687A6891
:107420000192CDE902434FF400330B9340F22B312C
:1074300040224FF480430591049209934FF48062F7
:107440004FF4805301A90792089365F0EDFFEB68B4
:107450009A681368012043F01003136010B0BDE870
:10746000F081136803F13C04D3E7136803F1380497
:10747000CFE7136803F13404CBE700BF4059002085
:10748000009F24000C0800205C8B0708006002406D
:10749000003802405C5A002010B5114CD4F8180195
:1074A00028B1104A6421FBF789FBD4F818010021A8
:1074B000FBF700FCD4F818315B681A68B2F8443066
:1074C0006FEA43436FEA53439BB2A2F844301388F8
:1074D00001219BB20B43138084F8C81D10BD00BF6F
:1074E00040590020009F240010B54FEA511E02446D
:1074F00000EB8E0C624529D901F01F014FF0FF34DB
:1075000004FA01F350F82E100B4093FAA3F3B3FAE8
:1075100083F3DBB2202B16D10CF104018A4202D88E
:1075200017E08A4212D98C460431DCF8003093FA15
:10753000A3F3B3FA83F3DBB2202BF2D0ACEB000061
:1075400003EBC00010BD03EB4E1010BD4FF0FF3039
:1075500010BD204610BD00BF30B503694268474DDD
:1075600083B00BB9002A63D0D0ED067AC46A013328
:1075700077EE807A0361631C012BC0ED067AC3624B
:1075800046D0D0ED075A90ED097A296807EE903A77
:1075900030EE656AF8EEE76A8A1AC6EE267A8168E6
:1075A0008A4277EEA57A30EE670AC0ED087AA6EE39
:1075B000007AC0ED077A80ED0A7A80ED097A01D869
:1075C00003B030BD012B4BDD07EE904AF8EEE77AB1
:1075D00087EE270AB5EEC00AF1EE10FA43DBB5EEEE
:1075E000400AF1EE10FA41D4F1EEC07AF4EE677A77
:1075F000F1EE10FA37D690ED057AB4EEE77AF1EEB7
:1076000010FA18D5037B23B30323037003B030BDF6
:107610002B688168DFED1A7A80ED080A9A1A8A428F
:1076200080ED070AC0ED097ACAD9B0EE670ADBE738
:107630002A68426098E7D0ED047AD0ED066AF8EE49
:10764000677A022386EEA77A037080ED067A03B08C
:1076500030BD29684160002203618261C362AFE7E7
:107660009FED070AC0E7DFED067AC4E701906AF0F4
:107670002DFB0198F0EE407AB8E700BF6C240020A3
:107680000000000070B52DED028B044682B000F1C1
:10769000480503460026B1EC017AD3ED067ADA6A92
:1076A00077EE877A0132012AC3ED067ADA626DD06D
:1076B00093ED075A93ED096A07EE902A77EE455A43
:1076C000F8EEE77AC5EEA76A76EE857AF0EE466ABE
:1076D00037EE677AC3ED087AE5EE876AC3ED077A7D
:1076E000C3ED0A6AC3ED096A1833AB42D3D103690B
:1076F000394E42680133036133689B1A82689342B2
:1077000040D99FED368AE36A012B4DDD013B07EE40
:10771000903A94ED0A7AF8EEE77A87EE270AB5EE0A
:10772000C00AF1EE10FA4DDBB5EE400AF1EE10FAA8
:107730004BD4F1EEC07AF4EE677AF1EE10FA41D64E
:1077400090ED057AB4EEE77AF1EE10FA24D418340D
:10775000AC42D8D1D0ED047AD0ED066A90ED0C7A27
:10776000D0ED125AF8EE677A022386EEA76A03700C
:10777000C7EE276A85EEA77A80ED066AC0ED0C6A2F
:1077800080ED127A02B0BDEC028B70BD83ED087AF9
:1077900083ED077A5E62A7E7037B43B1032303709F
:1077A00002B0BDEC028B70BDB0EE480AC1E700220A
:1077B0003168416003618261C36202634364826431
:1077C000C365DFE7F0EE487ABAE701906AF07EFA27
:1077D0000198F0EE407AAEE76C2400200000000033
:1077E000F0EEC07AB0EEE07AB4EEE77AF1EE10FA9D
:1077F000D4BFB0EE676AB0EE476AB5EE406AF1EE0C
:1078000010FA48D0B4EEE77AF1EE10FA54BFF0EE79
:10781000675AF0EE475AC5EE866ADFED202ADFEDA3
:10782000203ADFED204A9FED205A9FED203A9FED50
:10783000204A9FED206AE6EEA23AA6EE834AE6EEE3
:10784000A34AF7EE005AA6EEA45AE6EE845AA6EE34
:10785000856AB1EE466AC6EE256AB4EEE77AF1EEC5
:1078600010FA48BFDFED147AF5EEC00A48BF77EE94
:10787000E66AF1EE10FA48BFDFED107AB5EEC00A05
:1078800048BF77EEE66AF1EE10FA48BFF1EE666A9D
:10789000B0EE660A7047DFED0A6ADEE739094E3D51
:1078A000E3B59EBE88FA16BE45FE7FBF99FB243F16
:1078B00069A2163EA7DFA8B4DB0FC93FDB0F494022
:1078C000A7DFA83491ED007AD0ED047AD0ED055A07
:1078D00090ED064AD0ED074A90ED085A90ED096AFE
:1078E000D0ED0A6AE7EE077AF7EE003AC0ED047AC7
:1078F00091ED007AD1ED017AE7EE275A90ED0B7AFF
:10790000C0ED055AD1ED025A91ED003AD0ED0C7A56
:10791000A3EE254A80ED064AD1ED005A74EEA54A41
:10792000C0ED074AD1ED014AD1ED005AA4EEA55AA7
:1079300080ED085A91ED015AA5EE056A80ED096ABD
:10794000D1ED015A91ED026AE5EE866AC0ED0A6A50
:10795000D1ED016A37EE267A80ED0B7AD1ED026A1D
:1079600091ED007AE6EE877AC0ED0C7A91ED026A2D
:10797000D1ED016AD0ED0D7A90ED0E7A90ED0F4ABF
:10798000D0ED104A90ED115AD0ED135AE6EE267A5A
:1079900075EEA35AC0ED0D7AD1ED026AD0ED127AE0
:1079A00090ED006AA6EEA67AD0ED016A80ED0E7A1F
:1079B00091ED027A34EE074A90ED027A80ED0F4A9B
:1079C00091ED004A74EE844AC0ED104AD1ED014AAF
:1079D00035EE245A80ED115A91ED025AC0ED135A3A
:1079E00077EE857AC0ED127AD1ED017AD1ED005AA9
:1079F00091ED025A67EEA77AE5EEA57AE5EE057AF3
:107A0000A5EEA76A80ED006A91ED016AE6EE276AAD
:107A1000C0ED016AD1ED026AA6EEA77A80ED027A86
:107A200090ED037A77EE277AC0ED037A704700BFB6
:107A30002DE9F04F89B0CDE9011200F1100983461C
:107A400000F13008CE4607464E46054684460024DF
:107A5000CDF80C906246284684B1D2ED007A0146FA
:107A60003B468946F3EC016A99ED007AE6EEC77A67
:107A7000634501F11001C2ED007AF2D10432724582
:107A800000F10400E8D1032C04F1010A30D0624671
:107A90003046ABEB05099CB1D2ED047A009409EBBA
:107AA000000329460C46F3EC016A94ED007AE6EEF9
:107AB000C77A834201F11001C2ED047AF2D1009C31
:107AC000D2ED046A16ED047AC6EE877A103242458A
:107AD00000F11000C2ED007ADDD10CF1140C08F1B8
:107AE0000408043514360EF1100E10375446B1E771
:107AF000DDE902290025002301350593069307934C
:107B0000042D52F8043B049305A80BF1140418D07B
:107B1000F2EC017A04A9C0ED007A4B46B1EC017A8F
:107B2000F3EC016AE6EEC77AA342C0ED007AF5D124
:107B30000135042D09F1100900F1040004F11404C9
:107B4000E6D1019A08AE76ED017A022510320BF1EA
:107B50004004022D2046A2F1040142ED017A20D01A
:107B60002346F3EC016AB2EC017AE6EEC77A98425A
:107B7000C1ED007AF5D154ED016A87EEA67A6B1C4F
:107B800081ED007A14D076ED017A013D0A46022D8E
:107B9000A4F11404A0F11000A2F1040142ED017A55
:107BA000DED154ED016A87EEA67A02ED017AEAE7AA
:107BB00009B0BDE8F08F00BF10B584B00C46024696
:107BC00069461030FFF734FFDDED007A9DED017A54
:107BD000DDED026AB6EE006A67EE867A27EE067A77
:107BE00066EE866AF4EE677AF1EE10FAC4ED007A7A
:107BF00084ED017AC4ED026A0DD6B4EE477AF1EE57
:107C000010FA13D6F4EE666AF1EE10FA78BF01208E
:107C100016D604B010BD9FED106AF0EEE77AF4EED0
:107C2000467AF1EE10FAE8DD0020F2E7DFED0A7A9D
:107C3000B0EEC77AB4EE677AF1EE10FAE2DDF3E760
:107C4000DFED057AF0EEE66AF4EE676AF1EE10FA1F
:107C5000D4BF01200020DCE7FFFF7F7FDFED257A26
:107C6000B4EEE70AF1EE10FA08DD9FED237A30EE6C
:107C7000470AB4EEE70AF1EE10FAF8DCDFED1F7AFE
:107C8000B4EEE70AF1EE10FA08D59FED1B7A30EE5C
:107C9000070AB4EEE70AF1EE10FAF8D4DFED187A2D
:107CA000B4EEE70AF1EE10FA18DD30EE670A37EEAF
:107CB000C00A60EE007A9FED137A9FED136ADFED44
:107CC000136AA7EE876A9FED127AE7EE866A60EE86
:107CD000275AA7EEA67AA5EE870A70479FED0D7A80
:107CE000B4EEC70AF1EE10FA44BF30EE270A37EEC1
:107CF000400ADEE7DB0F4940DB0FC940DB0F49C01C
:107D0000DB0FC93F9A7C2E36FAAF4FB93587083C56
:107D1000A4AA2ABEDB0FC9BF10B53E4CB4FBF2F4D7
:107D2000A1420DD300234FF07E5202604360836076
:107D3000C36003610023836143610362C36110BDBB
:107D400007EE902AB8EE677ADFED337A27EE277ACE
:107D5000B7EE006AC6EE076A07EE901A9FED2F7A1B
:107D6000F8EE677AB0EE405A67EE877AC7EEA64A19
:107D7000FDEEE47A17EE902A2032402A47D8B0EE82
:107D8000640AFFF76BFFB0EE404A9FED250A34EE20
:107D9000800AFDEEC07A17EE902A2032402A31D8B0
:107DA000FFF75CFFF8EE006A60EE266A012B24D034
:107DB000F7EE007A37EEC00AF6EE005A60EE255A6A
:107DC00035EE055AB7EE007A84EE056A76EE077A4C
:107DD00037EE467A80EE275A85EEA76AC6EEA75A96
:107DE000C7EE276A80ED006A80ED015A80ED026AD5
:107DF000C0ED035AC0ED046A9CE7B0EE660AF7EEE8
:107E0000005ADDE7DFED076A9FED070ACEE79FED39
:107E1000064ABAE720A10700BD378635DB0FC94007
:107E2000DB0FC93F0000008000000000DFED077A93
:107E300030EE270AFDEEC07A17EE903A2033402B41
:107E400000D80BE79FED020A704700BFDB0FC93F68
:107E50000000000091ED005A9FED520A35EE000A35
:107E600008B5FDEEC07A17EE903A2033402B7DD84E
:107E7000FFF7F4FEFDEEC57AB0EE403A17EE903A09
:107E80002033402B7BD8B0EE450AFFF7E7FEB0EE7B
:107E9000405AF1EE402A91ED014A9FED420A34EE3C
:107EA000000AFDEEC07A17EE903A2033402B74D8CA
:107EB000FFF7D4FEF0EE404AB1EE402AFDEEC47A60
:107EC00017EE903A2033402B64D8B0EE440AFFF707
:107ED000C5FEB0EE404AD1ED021A9FED320A31EEF6
:107EE000800AFDEEC07A17EE903A2033402B4ED830
:107EF000FFF7B4FEF0EE403AFDEEE17A17EE903A6D
:107F00002033402B40D8B0EE610AFFF7A7FE63EEA6
:107F1000836A20EE037A63EE857A20EE055AF0EE4E
:107F2000475AB0EE666AE7EE845AA5EE446AE7EE79
:107F3000047AA6EEC45A63EEA43A62EEA42A22EEB4
:107F4000000A64EE834AC0ED003A80ED010A80ED3C
:107F5000024AC0ED035A80ED046AC0ED052A80EDA7
:107F6000065AC0ED077AC0ED084A08BDFDEEC57A95
:107F70009FED0D3A17EE903A2033402B83D9DFED79
:107F80000B2A9FED095A86E79FED070ABFE7DFED51
:107F9000063AB1E79FED044A9DE79FED042ADFED25
:107FA000024A8BE7DB0FC93F0000000000000080A1
:107FB0002DE9F04F83B005469DF830400D9E0192AB
:107FC000002C14BF4FF030094FF020091C1E8846CA
:107FD0004ADB16F8010B014600286CD0002C65D056
:107FE0004FF0000A324601E0002C34D012F8013B79
:107FF0002746013C002BF7D1BAF1000F3CD1023FDC
:10800000002C65D0BA4645450AF1FF3A4946284654
:1080100001D2019B9847BAF1FF3FF4D10D9A107835
:1080200023463C1B01469B4688B14FF0000A0133B2
:108030009F1B454506EB070B284601D2019B98473D
:1080400016F8011B0029F4D1BAF1000F18D15846D7
:1080500003B0BDE8F08FBAF1000F31D0014683467E
:108060000028F4D02346E2E716F8010B634258B328
:108070001C464FF0010AB5E7014683460028D6D1D9
:10808000002C04F1FF36E2DD3446454506F1FF36AB
:108090004946284601D2019B9847731CF5D10BF144
:1080A000010BA344584603B0BDE8F08F2346A24617
:1080B0004FF0FF34BBE7671EA346002CA2D1C6E7F2
:1080C00023464FF0FF34ADE7E64383463446DCE712
:1080D00023463C46A6E700BF0FB430B583B006ABDD
:1080E0000B4C53F8042BD4F8E81FD4F8E40F019399
:1080F00065F040FA0546206803685B6998470028E8
:10810000F9D0284603B0BDE8304004B0704700BF46
:10811000405900200EB410B583B005AB044653F8A7
:10812000042B0749009301A8019465F023FA019BF1
:1081300000221A7003B0BDE8104003B0704700BFC2
:10814000356600080CB4F0B53C4CD4F8EC3FADF506
:10815000277D002B4CD094F8F43F994240D8384BFF
:10816000384A1B68A2FB031292094FF47A7101FB93
:10817000123306A83449FFF7CDFF06AB0344334959
:10818000AC9A01930646ADAB01A8009365F0F2F9F5
:10819000019BD4F8EC5F0A210246581C019019702B
:1081A000019B591C01910021197035B32B681B6A82
:1081B0001BB128469847D4F8EC5F9DF8181049B1D8
:1081C0000DF119042B6828461B68984714F8011B09
:1081D0000029F7D10DF5277DBDE8F04002B07047CA
:1081E000D4F8F82F012303FA00F01042B7D1F1E7D9
:1081F000D4F8F03F002BAED1ECE7D4F8F07F002F9D
:10820000E8D0901926AB841CFD20CDE9045506A9C1
:108210002246ADF8100018466CF056FA02220346CA
:10822000044402A93846CDE9023435F0A1FF0DF52A
:10823000277DBDE8F04002B0704700BF40590020E4
:108240006C240020D34D62102C2A080829660008EF
:1082500010B54FF4004086B034F0B0F958B14FF487
:108260000041044634F0D4F9022806D1226848F2CD
:1082700001039A4224D006B010BD00234FF46121BF
:10828000022294F904008DE80E001A464FF40041D2
:1082900034F0C8F91D4BC3F8EC0F0028EBD01C4A92
:1082A0001C4B1D4C1D481E490091CDE90332CDE900
:1082B00001041C4B1C4A02210020FFF743FFDAE7B0
:1082C0001A4B00244FF4004083F8984163F016F9EC
:1082D0000028D0D00D4BD3F8FC2F82420CD003F5F0
:1082E0008052D2F8D81081420BD0D2F8B4219042FB
:1082F00009D0C3F8F04FBEE703F6FC72C3F8F02FC5
:10830000CDE70B4AFAE70B4AF8E700BF40590020D7
:10831000502A08085C2A0808682A0808742A0808ED
:10832000382908084C290808382A0808386A002023
:10833000186A0020F46A002038B5184CD4F89C5113
:10834000033005EB9003B3F5007F18D804EB8101EF
:1083500020F00302D1F8A009C4F89C311044C3F501
:10836000007304F5D074C1F8A0090D4A04EB85042C
:108370009B0004210020FFF7E5FE204638BD0021C8
:108380000846084AFFF7DEFE074AD2F89C30002470
:1083900043F00073C2F89C30204638BD386A002094
:1083A0007C2A0808A02A08080000001038B50568D3
:1083B000EB690446F3B1987800B938BDB3F90A20E7
:1083C00007EE902AF8EEE77A0120C4ED057AB3F9BA
:1083D0000C2007EE902AF8EEE77AF1EE677AC4ED0A
:1083E000047AB3F90E3007EE903AF8EEE77AC4ED6E
:1083F000067A38BD09211420FFF79EFF0346E86185
:10840000D9E700BF38B50568EB690446E3B1987851
:1084100000B938BDB3F9042007EE902AF8EEE77AE8
:108420000120C4ED047AB3F9062007EE902AF8EE95
:10843000E77AC4ED057AB3F9083007EE903AF8EE22
:10844000E77AC4ED067A38BD09211420FFF774FFDE
:108450000346E861DBE700BF38B50568EB69044611
:10846000E3B1987800B938BD9A88D2BA07EE902A5D
:10847000F8EEE77A0120C4ED047ADA88D2BA07EE82
:10848000902AF8EEE77AC4ED057A1B89DBBA07EE8D
:10849000903AF8EEE77AC4ED067A38BD0921142047
:1084A000FFF74AFF0346E861DBE700BF38B5046821
:1084B000E3690D467BB1987800B938BD5B89094AFC
:1084C000DBBA82FB0312DB17C3EB221303F26D133B
:1084D0002B80012038BD09211420FFF72DFF034612
:1084E000E061E8E7797878782DE9F041944603EB8C
:1084F00043031CF8068B86B0144602EB4303154673
:108500004FFA88F69CF80070A0EB070E821BBEF1B4
:10851000000FB8BFCEF1000E002AB8BF52429645F8
:10852000B8BF65460CF1060CB8BF7EB26345E9D111
:10853000B0456F88A3F1060206D0BE46A24216D00F
:1085400014F8068FB045F8D1B4F80280CB1BA1EB2C
:10855000080C002BB8BF5B42BCF1000FB8BFCCF1D8
:10856000000C6345BE46E9DD47462546E5E76B79E5
:1085700004932B7903932B78064A0091CDE9013EB1
:10858000032103460120FFF7DDFD284606B0BDE8C4
:10859000F08100BFB02A080803681A46591C016020
:1085A00012F8021B0260587841EA0020704700BFB1
:1085B00002681146531C036011F802CB0160D31C02
:1085C0005178036093781B0443EA0123111D016075
:1085D000D07843EA0C0343EA0060704712B370B5E9
:1085E0000446864604E0981B17D114EB0C0C15D0FA
:1085F0001EF8013BA3F14100192811F8010BA0F16D
:10860000410598BF2033192DA2EB0E0C00F1200676
:10861000E9D91B1A04D10028E7D170BD604670BDAE
:10862000184670BD1046704710B40288C378174CC6
:10863000A2F5FA6202F0030140F2B55C9208013B38
:108640000CFB0233827801EB4101013A02EB81021B
:1086500004EB420102798C8E4179234403EB4303FE
:1086600002EBC30384790A4A0089C3EB031301EBCD
:108670008303C3EB0313224402EB830200214FF474
:108680007A73C2FB03015DF8044B70475C8B0708EB
:1086900080436D382DE9F04117461E4605464FF4DC
:1086A0007A7200233846314668F084FB4349444AD5
:1086B000014482FB0143C8170B44C0EB631382FBE8
:1086C00003021A44D8173F4CC0EB621284FB020429
:1086D0004FEAE27C3C48CCEBA40C80FB0C404FEA18
:1086E000EC74C4EBE010C3EB0314A1EB8401A9719B
:1086F000C2EB0211A3EB81036B710CEB4C03A2EBF9
:10870000C30240F2B55303FB10CCBCF5896F2A714C
:108710004FEA800044DA40F2DA239C4547DCBCF59E
:10872000B77FB4BF00220122284B02EB420103EBCA
:10873000C1034FEA4208B3F84A3091B2244C08EB27
:10874000020E04EBCE0416344FF00B0E01E034F8A9
:10875000023D63451FDDBEF1010EF8D11B4B4244C3
:1087600003EBC2024FF0010E938E85F802E000F594
:10877000FA600CF1010C0844ACEB030C288085F87E
:1087800003C04FF47A7200233846314668F012FB7A
:108790002A81BDE8F0810EF1010E5FFA8EFEE4E75A
:1087A000032140F296530A464FF00608C6E702211D
:1087B00040F229430A464FF00408BFE780BC92C745
:1087C00089888888ABAAAA2A73B06D165C8B0708C3
:1087D000908B070830B52E4D84468E460FCD8DB058
:1087E0006C460FC40FCD0FC495E80F001CF0030FAB
:1087F00084E80F000DD1274B274A03FB0CF3B2EBA3
:10880000B30F43D3254AB2EB331F2CBF1D241C24C6
:1088100000E01C240CF1FF33002B40F26D121946CE
:1088200002FB0CF2B8BF0CF1020102EBA1021C49E1
:108830001C4D019481FB0301DB17A3EB6110024483
:10884000C3EBE1131A44253285FB02301044D317E1
:10885000C3EBA000C0EBC000ADF10403101A0DF192
:10886000040C03EB8E0E01E05CF8044F031985FB4A
:108870000320C218D817C0EBA200C0EBC000E64529
:10888000A3EB0000F0D1201A0DB030BD1D24C1E7CC
:10889000F08B0708295C8FC2285C8F020AD7A300DF
:1088A0001F85EB519324499208B50C4B53E90223E1
:1088B00052EA030C09D1002340F201124280838066
:1088C000837103800381184608BD054909688A1829
:1088D00043F10003FFF7DEFE012008BD68740020AD
:1088E0006C24002030B5144DD5F8282AD5F82C3A40
:1088F00052EA030183B0044609D1002040F201137B
:1089000020806380A080A071208103B030BD0B491E
:1089100009688A1843F10003FFF7BCFEB5F8303A46
:10892000ADF8063020460DF10602214664F0EEF85F
:10893000012003B030BD00BF386A00206C24002045
:1089400088422DE9F0414FF001043DD301FB04F4CE
:10895000B0FBF4FC8C45F9D23CB3002616E0BCF128
:10896000090F274698462C4623DD002A14BF4FF0F6
:10897000370E4FF0570EF444B94288F800C003F1A7
:10898000010306F1010610D8B0FBF5FCB4FBF1F5CC
:1089900004FB1C00002EE2D1BCF1000FDFDCA14281
:1089A0000AD90CF1300C03F801CB00221A70BDE893
:1089B000F0814FF0300EDEE7B0FBF5FC2C4605FBF6
:1089C0001C00B5FBF1F5E7E78446C6E790422DE9C8
:1089D000F0410B46044615460AD2B0FBF5F6134AA1
:1089E00005FB16441846135D00F8013BBDE8F08115
:1089F000B0FBF2F69642B6FBF2F706D20B4A05FB45
:108A00001767D15D03F8011BEAE7BA42B7FBF2F83A
:108A100007D9064A05FB187812F8081003F8011B5D
:108A2000EDE74046FFF7D2FF0346F2E7EC2A0808DD
:108A3000B5EEC00ADFED347AF1EE10FACCBF30EEBD
:108A4000270A30EE670ADFED317A20EE270A70B58B
:108A5000FDEEC07A86B017EE904A054684EAE470CF
:108A6000002303A9A0EBE470CDE90033029364F086
:108A700007FD002CACBF20232D2303A88DF8003068
:108A800067F0D0FA01286E4628D0022832D0032899
:108A90001CD003A930466EF005FF304667F0C2FADD
:108AA0000338C4B22246314628466BF00DFE00233F
:108AB0002B55284667F0B6FA2E232B540130311976
:108AC00028446EF00BFF284606B070BD302303A982
:108AD00030468DF801306EF0E5FEDEE7302303A965
:108AE00030468DF801308DF802308DF803306EF08D
:108AF000D9FED2E7302303A930468DF801308DF836
:108B000002306EF0CFFEC8E76F12033A00007A44DD
:108B10000278202A034600F10100F9D0092AF7D093
:108B20002D2A29D02B2A03BF5A78B7EE000A034614
:108B3000B7EE000AA2F13001C8B20928DFED4C7A85
:108B400010D8F2EE046A07EE101AB8EEC77A13F8DE
:108B5000012FA7EEA67AA2F13001C8B20928F0EEE3
:108B6000477AF0D92E2A49D0197801F0DF0145293A
:108B700007D020EE270A70475A78BFEE000A034656
:108B8000D8E710B459782D2962D02B2954D0A1F1FF
:108B90003002092A03F1010355D80024002202EB18
:108BA000820201EB420213F8011FA1F130000928F3
:108BB000A2F13002F3D9B2F59A7F134628BF4FF4E1
:108BC0009A73072A50D9DFED2B6A1A46B7EE007A5E
:108BD000083A072A27EE267AFAD803F007032BB1C2
:108BE000F2EE046A013B27EE267AFBD16CB3C7EEA6
:108BF000877A5DF8044B20EE270A70475978A1F177
:108C00003002D0B2092803F10103AED8F2EE046AB3
:108C1000F0EE665A07EE102AB8EEC77A13F8011F75
:108C200087EE266AA1F13002D0B2092866EEA56A65
:108C300077EE867AEED998E79978A1F13002092A81
:108C400003F10203A9D9B7EE007A67EE877AD0E77D
:108C50009978A1F13002092A03F1020388BFB7EE27
:108C6000007AC4D8012499E7B7EE007AB7E700BFCD
:108C70000000000020BCBE4C00B50378202B01464C
:108C800000F10100F9D0092BF7D02D2B03BF4B7851
:108C90004FF0FF3E01464FF0010E0022A3F1300CD1
:108CA0005FFA8CF3092B03D90EFB02F05DF804FB8D
:108CB00002EB820211F8013F0CEB4202EEE700BF2B
:108CC000F0B5384D2B78082141F221008B4002E0AD
:108CD000013993B209D013F4004F4FEA4302F7D0A1
:108CE00080EA430301399BB2F5D1B5F80120002A8F
:108CF00055D0DFF8C0C02C4EB4452DD2ACF1060CD7
:108D00000CEB0204B44227D2052A41F2210022D9F9
:108D1000A44514D00CF1FF3C04F1FF3E1CF8011FE8
:108D2000082283EA012313F4004F80EA43010ABFBB
:108D30005B008BB29BB2013AF5D1E645EED12288B9
:108D400062B1A11DB14206D2A118B142A44602D21D
:108D5000052A0C46DCD800210846F0BDA71C264693
:108D600041F2210016F8011B082283EA012313F4C3
:108D7000004F80EA43010ABF5B008BB29BB2013A0D
:108D8000F5D1B742EED16188084AC91AB1FA81F12A
:108D9000231D49095B1BA2F8343A0846F0BD044F75
:108DA000BC1EDCE700000E0800001008386A002036
:108DB00003000E0807000E082DE9F04F9B4B9C4A5C
:108DC0008FB09A1ACDE9013203230393984B07938E
:108DD000029B0993019B08930023CDE90A33CDE957
:108DE0000C33944A1369002BC0F2A181914B924934
:108DF000F322DA6000220C92019A01238A428DF854
:108E00003430C0F08C810B937E238DF828300822FB
:108E10004FF4FC4341F2210103E05B00013A9BB2B5
:108E200006D01804F9D581EA4303013A9BB2F8D180
:108E3000824AADF81230824B934280F08E8103F16A
:108E4000140801997A4B41F2210538F8120C38F8D0
:108E5000142CC0F30B06B41DADF81440C2F30B0480
:108E6000120B8DF8182000270204ADF816408DF87B
:108E700019705DD406338B4200F251810DF1140953
:108E80000DF11A0A4C4601E0A24513D00B9B14F8D1
:108E9000011B03F138026A440133042B02F8101C51
:108EA0000B93F1D10AA907A8F9F726FDA245CDE950
:108EB0000B70EBD10C9B002BC0F23181BDF812403E
:108EC00019F8013B84EA0324082327044CBF85EAF0
:108ED00044046400013BA4B2F7D1CA45F0D158F86C
:108EE000101C324607A8FDF70DFF0028C0F21781BD
:108EF00058F8102C91198A4210D0013A013912F811
:108F0000013F84EA0324082320044CBF85EA44047B
:108F10006400013BA4B2F7D19142F0D1474BADF8C8
:108F20001240984574D2DDE9073108F114088CE746
:108F3000B946CDF8008009F1010906335FFA89F9D5
:108F40008B428DF8199000F2EA800DF1140A0DF1B0
:108F50001A0BD046002401E0C34513D00B9B18F830
:108F6000011B03F138026A440133042B02F8101C80
:108F70000B93F1D10AA907A8F9F7BEFCC345CDE9C7
:108F80000B40EBD10C9B002BC0F2C980BDF8124006
:108F90001AF8013B84EA0324082322044CBF85EA23
:108FA00044046400013BA4B2F7D1D345F0D1009B47
:108FB00053F8102C02EB070A5146324607A8FDF77A
:108FC000A1FE0028C0F2AB800AEB06018A4511D051
:108FD0000AF1FF32013912F8013F84EA0324082321
:108FE00020044CBF85EA44046400013BA4B2F7D1DD
:108FF0008A42F0D1B9F1030FADF81240374402D0E4
:10900000DDE9073197E7DDF800800C4B98458AD3FE
:10901000DDE90731023300229942ADF814207ED3F6
:109020000DF115040DF1160516460FE000001008AD
:1090300000000E08003C024001000E0870A608085F
:1090400070A10808A54213D014F8012B0B9B03F163
:10905000380169440133042B01F8102C0B93F1D132
:109060000AA907A8F9F748FCA542CDE90B60EBD1A6
:109070000C9B002B53DBBDF81230082241F221017A
:109080001C0454BF5B0081EA4303013A9BB2F7D151
:10909000082241F2210118044CBF81EA43035B001E
:1090A000013A9BB2F7D1ADF81230079B0899023311
:1090B0008B4234D814460DF1120505AE01E0B542DD
:1090C00013D00B9B15F8011B03F138026A440133DE
:1090D000042B02F8101C0B93F1D10AA907A8F9F789
:1090E0000BFCB542CDE90B40EBD10C98002816DB08
:1090F0000B9B13B3079A08991A448A420FD80AA9FE
:10910000C818C3F1040200216DF07CFC0AA907A86D
:10911000F9F7F2FB002398420C900B930DDA039BB6
:10912000013B03937FF452AE052007F057FD0F4B30
:10913000536003F18833536058E69DF834307BB9AF
:109140000028ECD10A4B1B787E2BEDD1FFF7B8FD40
:109150000028E9D00FB0BDE8F08F0199044B59E722
:10916000044A136943F000431361E9E723016745AB
:1091700000000E08003C024070B545880B460446CE
:10918000C5F30B052A46002118466DF03BFC21690A
:10919000084A9142034602D3074A914205D319B1C6
:1091A000BDE870401846084770BD2A46BDE87040CB
:1091B0006BF08ABA70A6080817AB080810B50379D7
:1091C000012B84B08E460ED0022B09D18368DB07B9
:1091D00058BF01F07F0104B0BDE81040FDF7BCBDF1
:1091E000002004B010BD144682688DF80F4002F0D4
:1091F000010201920DF10F020092417C90F91000E2
:109200007246FAF7F3FE04B010BD00BFF8B578223D
:10921000044600210068FFF7D1FF052707F082FC14
:1092200005460E4607F07EFC431B61EB0602B3F5D4
:109230007A7F72F10003F5D3013FEFD1206820223D
:109240000121FFF7BBFF052707F06CFC05460E4622
:1092500007F068FC431B61EB0602B3F57A7F72F1FD
:109260000003F5D3013FEFD120683A460221FFF712
:10927000A5FF642607F056FC04460D4607F052FC95
:10928000031B61EB0502B3F57A7F72F10003F5D39E
:10929000013EEFD10120F8BDF8B5072204460A21AE
:1092A0000068FFF78BFF052707F03CFC05460E46DC
:1092B00007F038FC431B61EB0602B3F57A7F72F1CD
:1092C0000003F5D3013FEFD1206824224121FFF7AD
:1092D00075FF052707F026FC05460E4607F022FC21
:1092E000431B61EB0602B3F57A7F72F10003F5D3FD
:1092F000013FEFD12068C0224221FFF75FFF052622
:1093000007F010FC04460D4607F00CFC031B61EB54
:109310000502B3F57A7F72F10003F5D3013EEFD178
:109320000120F8BD10B50446002221210068FFF796
:1093300045FF2068FC222021FFF740FF20684022E3
:109340002421FFF73BFF20680C222321FFF736FF83
:10935000206800222221FFF731FF012010BD00BF4D
:10936000F8B50122074610210068FFF727FF00B972
:10937000F8BD142607F0D6FB04460D4607F0D2FBD5
:10938000031B61EB0502B3F57A7F72F10003F5D39D
:10939000013EEFD13868A022BDE8F84011210DE769
:1093A00030B505682B79012B85B0044611D0022B0E
:1093B0000CD101220B212846FDF7CEFC30B12068EC
:1093C0001D22092105B0BDE83040F7E6002005B0B8
:1093D00030BDAA6895F91000697C8DF80F3002F055
:1093E000010201920DF10F0200920B22FAF7FEFD2D
:1093F000E4E700BF10B50446C06900B110BD092103
:109400001420FEF799FFE06110BD00BF184B03EB7D
:109410008000406848B310B5164C00EB400004EBE8
:10942000800393F939CABCF1FF3F1FD093F8410A7A
:10943000D0B104EB0C0293F8400A92F88CEA8C232A
:10944000142103FB0CFC00220CEB000304EB430390
:109450000139B3F8903A704412FA83F2F4D1064815
:10946000A0FB0230C0F30F1010BD7047002010BDEC
:1094700040590020386A0020CDCCCCCC28B30368FA
:10948000124A30B503F13F4303F57E039B0A0546BC
:1094900083B00C46D05C63F0D3FEA988009104F041
:1094A0000303C4F381028DF8043028688DF8052089
:1094B000C4F300136946C4F341148DF806308DF8E7
:1094C0000740F9F7FBFE03B030BD7047288B070853
:1094D00070B5114B114CA34203D319E00C33A342D6
:1094E00016D293F805C08C45F8D193F804C0844592
:1094F00001D00028F2D193F807E09645EED11D681F
:1095000095F804E0E645E9D12E689E42E6D100E0F8
:109510000025284670BD00BF18AB0808D4AC080869
:109520000379022B00D0704710B590F91020204825
:1095300082B00831694403244FF0000C02EB820230
:109540004FF0010E8DF800C08DF801E08DF802306B
:109550008DF8034050F8222011F8084C15498A4232
:1095600022D0A1F578418A4220D001F580618A425B
:1095700018D1118821F04001090403EB8303090C81
:10958000118000EB83001388C16823F0380331F8A1
:1095900024101B041B0C0B43138013889BB243F055
:1095A0004003138002B010BD6346E2E77346E0E774
:1095B0006000002000300140F8B507460021006837
:1095C000FFF7AEFF3868B6221421FFF7F7FD6426D7
:1095D00007F0A8FA04460D4607F0A4FA031B61EB56
:1095E0000502B3F57A7F72F10003F5D3013EEFD1A6
:1095F000812210213868FFF7E1FD07F093FA044655
:109600000D4607F08FFA031B61EB0502B3F57A7F75
:1096100072F10003F5D3802215213868FFF7CEFDE3
:1096200007F080FA04460D4607F07CFA031B61EB55
:109630000502B3F57A7F72F10003F5D33868032190
:10964000BDE8F8406CE700BFF8B5044600210068AB
:10965000FFF766FF2068B6227E21FFF7AFFD642783
:1096600007F060FA05460E4607F05CFA431B61EB13
:109670000602B3F57A7F72F10003F5D3013FEFD113
:109680003A4620687C21FFF799FD642707F04AFAE3
:1096900005460E4607F046FA431B61EB0602B3F59A
:1096A0007A7F72F10003F5D3013FEFD120680422E5
:1096B0007D21FFF783FD642707F034FA05460E4647
:1096C00007F030FA431B61EB0602B3F57A7F72F1C3
:1096D0000003F5D3013FEFD18C2240212068FFF732
:1096E0006DFD07F01FFA05460E4607F01BFA431BF7
:1096F00061EB0602B3F57A7F72F10003F5D3022223
:1097000041212068FFF75AFD07F00CFA05460E4686
:1097100007F008FA431B61EB0602B3F57A7F72F19A
:109720000003F5D320680221FFF7FAFE4FF400632F
:10973000A381F8BD2DE9F041046884B00546B62246
:109740007E212046FFF73AFD4FF0640807F0EAF962
:1097500006460F4607F0E6F9831B61EB0701B3F5F8
:109760007A7F71F10003F5D3B8F10108EED102213F
:109770002046FFF7D5FE636913B11A689B885383AF
:1097800007F0D0F906460F4607F0CCF9831B61EBD2
:109790000702B3F57A7F72F10003F5D3636913B161
:1097A0001A689B8813834FF00A0807F0BBF9064636
:1097B0000F4607F0B7F9831B61EB0701B3F57A7F1A
:1097C00071F10003F5D3B8F10108EED142467C21D6
:1097D0002046FFF7F3FC07F0A5F906460F4607F011
:1097E000A1F9831B61EB0702B3F57A7F72F10003E5
:1097F000F5D3002259212046FFF7E0FC07F092F94B
:1098000006460F4607F08EF9831B61EB0702B3F59E
:109810007A7F72F10003F5D394F91030A2688D4974
:1098200003EB83035E2092078DF80F0051F82300AD
:1098300040F1E48001230DF10F020021019066F058
:109840005BFA4FF4A473844A0198002166F054FA3D
:10985000A3689B0740F1E5804FF00A0807F062F922
:1098600006460F4607F05EF9831B61EB0701B3F56F
:109870007A7F71F10003F5D3B8F10108EED101222E
:1098800059212046FFF79AFC07F04CF906460F468F
:1098900007F048F9831B61EB0702B3F57A7F72F199
:1098A0000003F5D38C2240212046FFF787FC07F008
:1098B00039F906460F4607F035F9831B61EB0702BD
:1098C000B3F57A7F72F10003F5D3032241212046DC
:1098D000FFF774FC07F026F906460F4607F022F959
:1098E000831B61EB0702B3F57A7F72F10003F5D3B6
:1098F000AA6B5A4E95F83500B6FBF2F2092391B2E5
:10990000574AFEF7F1FD4388B6FBF3F62E64027961
:10991000422142F0C0022046FFF750FC07F002F956
:1099200005460E4607F0FEF8431B61EB0602B3F551
:109930007A7F72F10003F5D3082243212046FFF716
:109940003DFC07F0EFF805460E4607F0EBF8431B29
:1099500061EB0602B3F57A7F72F10003F5D30422BE
:1099600058212046FFF72AFC07F0DCF805460E4692
:1099700007F0D8F8431B61EB0602B3F57A7F72F16A
:109980000003F5D30A2253212046FFF717FC07F006
:10999000C9F805460E4607F0C5F8431B61EB060201
:1099A000B3F57A7F72F10003F5D300227C212046C3
:1099B000FFF704FC07F0B6F805460E4607F0B2F8CC
:1099C000431B61EB0602B3F57A7F72F10003F5D316
:1099D00006227D212046FFF7F1FB07F0A3F804469D
:1099E0000D4607F09FF8031B61EB0502B3F57A7F84
:1099F00072F10003F5D304B0BDE8F081636913B1DF
:109A00001A689B885383174B17491A68174B4E687F
:109A1000D200A3FB023292094B689B1B9A42FBD2F5
:109A200008E7104B10491A68104B48684FF4FA7653
:109A300006FB02F2A3FB023292094B681B1A9A4200
:109A4000FBD26369002B3FF407AF1A689B8813832E
:109A500002E700BF60000020208C070840420F0092
:109A6000688D070868240020001000E0D34D6210C4
:109A70002DE9F041604A0468816B604FB7FBF1F15A
:109A80000646102389B290F83500FEF72DFD00211F
:109A90004388B7FBF3F7054637642046FFF740FDE0
:109AA00080226B212046FFF789FB4FF0640807F006
:109AB00039F806460F4607F035F8831B61EB0701BE
:109AC000B3F57A7F71F10003F5D3B8F10108EED157
:109AD000032268212046FFF771FB4FF0640807F06E
:109AE00021F806460F4607F01DF8831B61EB0701BE
:109AF000B3F57A7F71F10003F5D3B8F10108EED127
:109B000001226B212046FFF759FB4FF00F0807F0A9
:109B100009F806460F4607F005F8831B61EB0701BD
:109B2000B3F57A7F71F10003F5D3B8F10108EED1F6
:109B300018221B212046FFF741FB4FF00F0806F0CB
:109B4000F1FF06460F4606F0EDFF831B61EB0701B0
:109B5000B3F57A7F71F10003F5D3B8F10108EED1C6
:109B600018221C212046FFF729FB4FF00F0806F0B2
:109B7000D9FF06460F4606F0D5FF831B61EB0701B0
:109B8000B3F57A7F71F10003F5D3B8F10108EED196
:109B90002A791A212046FFF711FB4FF00F0806F033
:109BA000C1FF06460F4606F0BDFF831B61EB0701B0
:109BB000B3F57A7F71F10003F5D3B8F10108EED166
:109BC0006A7919212046FFF7F9FA642706F0AAFFFF
:109BD00005460E4606F0A6FF431B61EB0602B3F5F1
:109BE0007A7F72F10003F5D3013FEFD120460321C4
:109BF000BDE8F04194E400BFA08D070840420F008B
:109C00002DE9F0416C4A0468816B6C4FB7FBF1F1B0
:109C10000646102389B290F83500FEF765FC002156
:109C20004388B7FBF3F7054637642046FFF778FC17
:109C300080226B212046FFF7C1FA4FF0640806F03E
:109C400071FF06460F4606F06DFF831B61EB0701AF
:109C5000B3F57A7F71F10003F5D3B8F10108EED1C5
:109C6000072268212046FFF7A9FA4FF0640806F0A2
:109C700059FF06460F4606F055FF831B61EB0701AF
:109C8000B3F57A7F71F10003F5D3B8F10108EED195
:109C900042466B212046FFF791FA4FF0640806F028
:109CA00041FF06460F4606F03DFF831B61EB0701AF
:109CB000B3F57A7F71F10003F5D3B8F10108EED165
:109CC00001226B212046FFF779FA4FF00F0806F0CA
:109CD00029FF06460F4606F025FF831B61EB0701AF
:109CE000B3F57A7F71F10003F5D3B8F10108EED135
:109CF00018221B212046FFF761FA4FF00F0806F0EB
:109D000011FF06460F4606F00DFF831B61EB0701AE
:109D1000B3F57A7F71F10003F5D3B8F10108EED104
:109D200018221C212046FFF749FA4FF00F0806F0D1
:109D3000F9FE06460F4606F0F5FE831B61EB0701B0
:109D4000B3F57A7F71F10003F5D3B8F10108EED1D4
:109D50002A791A212046FFF731FA4FF00F0806F052
:109D6000E1FE06460F4606F0DDFE831B61EB0701B0
:109D7000B3F57A7F71F10003F5D3B8F10108EED1A4
:109D80006A7919212046FFF719FA642706F0CAFEFE
:109D900005460E4606F0C6FE431B61EB0602B3F510
:109DA0007A7F72F10003F5D3013FEFD12046032102
:109DB000BDE8F041FFF7B4BBA08D070840420F009B
:109DC0001EE700BFF0B5044683B000680021FFF72E
:109DD000A7FB0C2225212068FFF7F0F90A22262193
:109DE0002068FFF7EBF9002263212068FFF7E6F90E
:109DF000206881222721FFF7E1F9142706F092FE5F
:109E000005460E4606F08EFE431B61EB0602B3F5D7
:109E10007A7F72F10003F5D3013FEFD10C222521A7
:109E20002068FFF7CBF90A2226212068FFF7C6F940
:109E30000F2263212068FFF7C1F9206881222721C2
:109E4000FFF7BCF90A2706F06DFE05460E4606F040
:109E500069FE431B61EB0602B3F57A7F72F10003E2
:109E6000F5D3013FEFD1032301AA1021204661F071
:109E700083FE0A2706F056FE05460E4606F052FE01
:109E8000431B61EB0602B3F57A7F72F10003F5D351
:109E9000013FEFD19DF804009DF805109DF80620C4
:109EA0002B4B803080318032A3F8D80DA3F8DA1D17
:109EB000A3F8DC2D25210C222068FFF77FF926214D
:109EC0000A222068FFF77AF93A4663212068FFF7F3
:109ED00075F9206881222721FFF770F90A2706F01B
:109EE00021FE05460E4606F01DFE431B61EB0602F1
:109EF000B3F57A7F72F10003F5D3013FEFD10DF195
:109F0000030201230221204661F036FE01230DF1F8
:109F100003020921204661F02FFE20680C22252132
:109F2000FFF74CF920680A222621FFF747F920683D
:109F300012226321FFF742F9812220682721FFF7CF
:109F40003DF920680321FFF7EBFA012003B0F0BDD3
:109F5000386A00200379022B00D0704783689B0782
:109F6000FBD5436913B11A689B885383064B074995
:109F70001A68074B4868D200A3FB023292094B686B
:109F80001B1A9A42FBD2704768240020001000E0A0
:109F9000D34D6210F0B5054690F91000244C00EB4B
:109FA000800085B054F82000AC68A40710D5CDE936
:109FB0000223019065F038FFDDE9022301980021BA
:109FC00065F09AFEAB689B0718D5012005B0F0BD7F
:109FD0006C6914B12668A4887483164C164E2468E4
:109FE00077684FEAC40E154CA4FB0E4E4FEA9E1E36
:109FF0007468A4EB070CE645FAD2D8E70D4B0E497E
:10A000001A680E4B4FF4FA7000FB02F2A3FB023207
:10A01000486892094B681B1A9A42FBD26B69002B65
:10A02000D3D01A689B881383012005B0F0BD00BF10
:10A030006000002068240020001000E0D34D621072
:10A0400030B50579012D83B08E460DD0022D08D193
:10A050008468E40758BF41F0800103B0BDE8304098
:10A0600098E7002003B030BD14468268009402F0E7
:10A070000102417C90F9100001927246F9F7B6FF97
:10A0800003B030BDF0B50546164695F910202448BA
:10A0900002EB820283B050F82200AA6892070FD523
:10A0A000CDE9000365F0C0FE019B00980022314617
:10A0B00065F022FEAB689B0718D5012003B0F0BD08
:10A0C0006A6912B1146892886283164A1468164A43
:10A0D0004FEAC40E154C5768A4FB0E4E4FEA9E1E65
:10A0E0005468A4EB070CE645FAD2D9E70D4B0E49AC
:10A0F0001A680E4B4FF4FA7000FB02F2A3FB023217
:10A10000486892094B681B1A9A42FBD26B69002B74
:10A11000D3D01A689B881383012003B0F0BD00BF21
:10A120006000002068240020001000E0D34D621081
:10A1300030B50579012D83B08E460DD0022D08D1A2
:10A140008468E40758BF41F0800103B0BDE83040A7
:10A1500098E7002003B030BD14468268009402F0F6
:10A160000102417C90F9100001927246F9F772FFEA
:10A1700003B030BD2DE9F043814A0568816B814C05
:10A18000B4FBF1F185B00646102389B290F8350092
:10A19000FEF7AAF900214388B4FBF3F407463464C0
:10A1A0002846FFF7BDF980226B212846FFF706F805
:10A1B0004FF0960906F0B6FC0446884606F0B2FC5D
:10A1C000031B61EB0801B3F57A7F71F10003F5D34E
:10A1D000B9F10109EED1032268212846FEF7EEFF0E
:10A1E0004FF0960906F09EFC0446884606F09AFC5D
:10A1F000031B61EB0801B3F57A7F71F10003F5D31E
:10A20000B9F10109EED103226B212846FEF7D6FFF2
:10A2100006F088FC0446884606F084FC031B61EBCC
:10A2200008010F2B71F10003F6D310226A21284692
:10A23000FEF7C4FF06F076FC0446884606F072FC82
:10A24000031B61EB08010F2B71F10003F6D3002211
:10A250006C212846FEF7B2FF06F064FC04468846EF
:10A2600006F060FC031B61EB08010F2B71F100038A
:10A27000F6D37A7919212846FEF7A0FF06F052FCA2
:10A280000446884606F04EFC031B61EB08010F2BC9
:10A2900071F10003F6D318221B212846FEF78EFF2A
:10A2A00006F040FC0446884606F03CFC031B61EBCC
:10A2B00008010F2B71F10003F6D318221C21284648
:10A2C000FEF77CFF06F02EFC0446884606F02AFCCA
:10A2D000031B61EB08010F2B71F10003F6D33A79F0
:10A2E0001A212846FEF76AFF06F01CFC07460C46BA
:10A2F00006F018FC8C4208BF8742F9D0032128469B
:10A30000FFF70EF93068062302AA4321FFF710FF7A
:10A3100028B3BDF80810BDF80A30BDF80C20C9BA42
:10A3200007EE901ADBBAD2BAF8EEE76A07EE102A07
:10A3300007EE903AB8EEC77AF8EEE77AC6ED076A0C
:10A34000C6ED087A86ED097AFDEEE77ACDED017A61
:10A350009DF90430013305D005B0BDE8F083D6ED9A
:10A36000087AF1E7D6ED077AFDEEE77ACDED017ACE
:10A370009DF904300133EFD1062006F02FFC00BF19
:10A38000A08D070840420F0010B50446006803790D
:10A3900082B0022B0CBF4321032106236A46FFF73C
:10A3A000C7FE68B1BDF80010BDF80220BDF804304A
:10A3B00049BA52BA5BBAE1866287238702B010BD00
:10A3C000E086A06302B010BD2DE9F047154D95F869
:10A3D000E13D07468A4663B90021386895F8E23DB9
:10A3E00085F8E11D52464921FFF7A2FE0120BDE894
:10A3F000F08706F097FBD5F8E84D001BC0F5FA543E
:10A40000002CE9DD06F08EFB4FEAE479064688462B
:10A4100006F088FB831B61EB0801A34271EB090383
:10A42000F6D3D9E7386A0020F0B5614C0546D4F878
:10A43000F00DC5F8360094F8E03DB4F8F42D6A87C5
:10A44000012B83B00AD0022B2ED003B3002384F853
:10A45000E03D84F8F63D184603B0F0BD94F8E13DC8
:10A46000002B41D169462846FFF7AEFF002851D0A6
:10A470009DF8003099074DD007220321284663F04C
:10A480003BFB022294F8F63D84F8E02DE3E72846F2
:10A490000122022163F030FB94F8F63D01221846B8
:10A4A00084F8E02D03B0F0BD94F8E13D05F13607E6
:10A4B00004F55F6623BB69462846FFF785FF9DF8D4
:10A4C000062003460028C1D01207BFD4B4F8D81D17
:10A4D000BDF8002012FB01F236498A4222DBB2F5B8
:10A4E000000F5EDB344A1EE006F01CFBD4F8E83DAA
:10A4F000C01AC0F5FA500028B4DD94F8F63DAAE77A
:10A5000006F010FBD4F8E83DC01AC0F5FA50002858
:10A51000D1DDF2E794F8F63D0022184684F8E02DEC
:10A5200003B0F0BD254AB4F8DA1DEA86BDF8022072
:10A5300012FB01F21F498A4205DBB2F5000F2ADB4C
:10A5400047F6FF7200E01D4AB4F8DC1D2A87BDF80B
:10A55000042012FB01F217498A4204DBB2F5000F16
:10A5600012DB154A00E0154AD5F83600C4F8F00DA4
:10A570006A87BA88B28000210122184684F8E01D5B
:10A5800084F8F62D03B0F0BD002AB8BFFF321212D6
:10A59000524212B2E8E7002AB8BFFF3242F30F225C
:10A5A000D2E7002AB8BFFF321212524212B2BAE703
:10A5B000386A002001FF7FFF0180FFFF0080FFFF5E
:10A5C00010B5044600680179012984B028D0022919
:10A5D00023D1836813F0010F08BF8221062302AA4A
:10A5E000FFF750FDB8B1BDF9083006EE903ABDF95D
:10A5F0000A3007EE103ABDF90C3007EE903AF8EE4B
:10A60000E66AB8EEC77AF8EEE77AC4ED076A84ED39
:10A61000087AC4ED097A04B010BD002004B010BD62
:10A620008368417C90F9100003F00103019302ABB1
:10A63000009302220623F9F70DFD0028D3D1EAE7A3
:10A6400030B5044600680379012B85B014D0022B85
:10A650000FD1826802AD12F0010F18BF03212A4604
:10A6600008BF8321FFF70EFD18B19DF90930002BBB
:10A6700010DB002005B030BD8368417C90F91000EC
:10A6800003F0010302AD0193009502230322F9F7C1
:10A69000E1FCE9E7206807232A461221FFF748FD7D
:10A6A0000028E6D09DF90A209DF809309DF90C108C
:10A6B00043EA022313EB430248BF03329DF80B30F9
:10A6C000921043EA012307EE902A13EB4302F8EEBF
:10A6D000E77A48BF03329DF90E109DF80D30C4EDA6
:10A6E000047A921007EE902A43EA012313EB430306
:10A6F000F8EEE77A48BF03339B10C4ED057A07EE06
:10A70000903AF8EEE77AC4ED067AB3E770B50668DA
:10A71000F46982B00546002C3FD03379012B04F157
:10A72000040205D0022B2CD00020A07002B070BD16
:10A73000B368717C96F91000009203F00103019355
:10A740000C231A46F9F786FCA0700028EED0B4F965
:10A75000043007EE903AF8EEE77AC5ED077AB4F9DF
:10A76000063007EE903AF8EEE77AC5ED087AB4F9CC
:10A77000083007EE903AF8EEE77AC5ED097A02B0B4
:10A7800070BDB36813F0010F4FF00C03304614BFD7
:10A7900019468C21FFF776FCD6E709211420FDF736
:10A7A000CBFDF06104462E68B7E700BF70B50668C0
:10A7B000F46982B00546002C3FD03379012B04F1B7
:10A7C000030205D0022B2CD00020A07002B070BD77
:10A7D000B368717C96F91000009203F001030193B5
:10A7E0000C220D23F9F736FCA0700028EED0B4F946
:10A7F0000A3007EE903AF8EEE77AC5ED077AB4F939
:10A800000C3007EE903AF8EEE77AC5ED087AB4F925
:10A810000E3007EE903AF8EEE77AC5ED097A02B00D
:10A8200070BDB36813F0010F30464FF00D0314BF35
:10A830000C218C21FFF726FCD6E709211420FDF717
:10A840007BFDF06104462E68B7E700BF10B50068D5
:10A850000379012B84B00C4618D0022B13D18368E6
:10A8600013F0010F14BF2221A221032303AAFFF733
:10A8700009FC30B1BDF90D3003EB83031B12E63345
:10A88000238004B010BD002004B010BD8368417C5B
:10A8900090F9100003F00103019303AB009322220F
:10A8A0000323F9F7D7FB0028E4D1EAE710B5044603
:10A8B00000680379012B84B02DD0022B28D1836846
:10A8C00013F0010F02AA4FF0060314BF1F219F21AE
:10A8D000FFF7D8FBD0B1BDF80810BDF80A20BDF8CD
:10A8E0000C30C9BA07EE901AD2BAF8EEE76A07EE52
:10A8F000902ADBBAB8EEE77A07EE903AF8EEE77AFC
:10A90000C4ED046A84ED057AC4ED067A04B010BD86
:10A91000002004B010BD8368417C90F9100003F062
:10A920000103019302AB00931F220623F9F792FB68
:10A93000D0E700BF10B5044600680379012B84B04E
:10A940002DD0022B28D1836813F0010F02AA4FF0FB
:10A95000060314BF2521A521FFF794FBD0B1BDF854
:10A960000810BDF80A20BDF80C30C9BA07EE901ADD
:10A97000D2BAF8EEE76A07EE902ADBBAB8EEE77AC9
:10A9800007EE903AF8EEE77AC4ED076A84ED087AAC
:10A99000C4ED097A04B010BD002004B010BD836876
:10A9A000417C90F9100003F00103019302AB009386
:10A9B00025220623F9F74EFBD0E700BF70B50668E5
:10A9C000F46982B00546002C3FD03379012B04F1A5
:10A9D000040205D0022B2CD00020A07002B070BD64
:10A9E000B368717C96F91000009203F001030193A3
:10A9F0003B220E23F9F72EFBA0700028EED0A3898E
:10AA0000DBBA07EE903AF8EEE77AC5ED077AE3890C
:10AA1000DBBA07EE903AF8EEE77AC5ED087A238ABA
:10AA2000DBBA07EE903AF8EEE77AC5ED097A02B0A4
:10AA300070BDB36813F0010F30464FF00E0314BF22
:10AA40003B21BB21FFF71EFBD6E709211420FDF7B0
:10AA500073FC0446F061B8E700B500680379012B88
:10AA600085B012D0022B0CD103AAF621FFF70AFB06
:10AA700020B1BDF80C300C4A5BBA938205B05DF88A
:10AA800004FB002005B05DF804FB8368417C90F96D
:10AA9000100003AA03F00103CDE900230223F622EC
:10AAA000F9F7D8FAE4E700BF4059002000B5006884
:10AAB0000379012B85B01FD0022B19D1032303AAE0
:10AAC000F621FFF7DFFA80B19DF80D309DF80CC03C
:10AAD00010499DF80E201B0243EA0C431343B1F9C1
:10AAE0003420C2F10802D3408B6305B05DF804FB4B
:10AAF000002005B05DF804FB8368417C90F91000EC
:10AB000003AA03F00103CDE900230323F622F9F79A
:10AB1000A1FAD8E74059002010B500680379012B4D
:10AB200084B032D0022B25D1062302AAF721FFF7E9
:10AB3000A9FAF8B19DF809209DF808409DF80A107F
:10AB40009DF80C309DF80BC0120142EA043242EA33
:10AB500011121B019DF80D10134C43EA0C3343EA0C
:10AB600011131249E265E363C1F8F82DC1F8FC3D09
:10AB700004B010BD0D4A0C4BD2F8F81DD2F8FC2DD4
:10AB8000D9650020DA6304B010BD8368417C90F978
:10AB9000100002AA03F00103CDE900230623F722E7
:10ABA000F9F758FAC5E700BF40590020386A00207D
:10ABB00000B500680379012B85B01DD0022B0AD1A6
:10ABC000836813F0010F03AA4FF0030314BF0021A1
:10ABD0008021FFF757FA9DF80D309DF80C009DF885
:10ABE0000E100C4A1B0243EA00430B430120C2F83B
:10ABF000803005B05DF804FB8368417C90F910005B
:10AC000003AA03F00103CDE9002303230022F9F78F
:10AC100021FAE0E74059002000B500680379012BD4
:10AC200085B01DD0022B0AD1836813F0010F03AA4F
:10AC30004FF0030314BF00218021FFF723FA9DF892
:10AC40000D309DF80C009DF80E100C4A1B0243EAD3
:10AC500000430B430120C2F8943005B05DF804FBBB
:10AC60008368417C90F9100003AA03F00103CDE949
:10AC7000002303230022F9F7EDF9E0E74059002013
:10AC800010B500680379012B84B029D0022B24D1A0
:10AC9000836813F0010F4FF0030303AA14BF194692
:10ACA0008321FFF7EFF9B0B19DF80C309DF90C103E
:10ACB0009DF80D209DF80EC01B04002943EA0223D5
:10ACC000B8BF4FF07F410D4AA8BF002143EA0C03F3
:10ACD0000B43C2F8D43004B010BD002004B010BD46
:10ACE0008268417C90F9100002F00102032303AC5A
:10ACF000CDE900421A46F9F7ADF9D4E740590020F2
:10AD000000B500680379012B85B02BD0022B25D12B
:10AD1000836813F0010F03AA4FF0030314BF00214F
:10AD20008021FFF7AFF9B0B19DF80C309DF90C1000
:10AD30009DF80D209DF80EC01B04002943EA022354
:10AD4000B8BF4FF07F410E4AA8BF002143EA0C0371
:10AD50000B43C2F8B83005B05DF804FB002005B025
:10AD60005DF804FB8368417C90F9100003AA03F0AE
:10AD70000103CDE9002303230022F9F76BF9D2E7A1
:10AD80004059002010B5044600230068E386A36301
:10AD90000279012A84B022D0022A1DD1836813F0DF
:10ADA000010F02AA4FF0060314BF03218321FFF70E
:10ADB00069F978B1BDF90A30BDF80810BDF80C206A
:10ADC0005B4201EB410103EB430302EB4202E186EC
:10ADD0002387628704B010BD184604B010BD836895
:10ADE000417C90F9100003F00103019302AB009342
:10ADF00003220623F9F72EF9DBE700BF70B50446FE
:10AE0000244894F9103003EB8303154650F82300CF
:10AE1000A3689A0782B00ED5019065F005F801236A
:10AE200001980022294664F067FFA3689B0717D5A5
:10AE3000012002B070BD636913B11A689B88538307
:10AE4000154B164A1B6856684FEAC30C144BA3FBFC
:10AE50000C3C4FEA9C1C53689B1B9C45FBD2DBE7D8
:10AE60000D4B0E491A680E4B4FF4FA7000FB02F2BC
:10AE7000A3FB0232486892094B681B1A9A42FBD224
:10AE80006369002BD4D01A689B881383012002B019
:10AE900070BD00BF6000002068240020001000E0AA
:10AEA000D34D621010B50379012B82B08E460DD0C0
:10AEB000022B08D18368DB0758BF41F0800102B044
:10AEC000BDE810409AE7002002B010BD1446826829
:10AED000009402F00102417C90F910000192724648
:10AEE000F9F7B8F802B010BD70B505682B79012BE1
:10AEF00084B004460E4615D0022B10D1AB68E12277
:10AF0000DB074CBF114661212846FBF725FF30B116
:10AF100020683246FF2104B0BDE87040C2E700203F
:10AF200004B070BDAA68697C95F9100002F00102B6
:10AF30000DF10F0501920095E1228DF80F20F9F730
:10AF400055F8E4E770B505682B79012B84B0044609
:10AF50000E4616D0022B11D1AB68DB074FF0C302AF
:10AF60004CBFE12161212846FBF7F6FE30B1206895
:10AF70003246FF2104B0BDE8704093E7002004B0E2
:10AF800070BDAA6895F91000697C02F00102019277
:10AF90000DF10F020092C3228DF80F20E122F9F784
:10AFA00025F8E3E770B505682B79012B84B00446DA
:10AFB0000E461AD0022B15D1AB68DB074FF0F0021A
:10AFC0004CBFE12161212846FBF7C6FE50B1224665
:10AFD000FF2152F8040BFFF765FF18B12379337096
:10AFE00004B070BD002004B070BDAA6895F91000CF
:10AFF000697C02F0010201920DF10F020092F02231
:10B000008DF80F20E122F8F7F1FFDFE7F0B50446F5
:10B0100083B000680021FEF783FA206815227E21A4
:10B02000FEF7CCF8642705F07DFD05460E4605F0D9
:10B0300079FD431B61EB0602B3F57A7F72F10003E1
:10B04000F5D3013FEFD1206811227E21FEF7B6F83B
:10B05000052705F067FD05460E4605F063FD431B19
:10B0600061EB0602B3F57A7F72F10003F5D3013F7D
:10B07000EFD120680DF107020321FFF713FF9DF8C0
:10B08000073003F03C03142B40F09A800C2240213F
:10B090002068FEF793F805F045FD05460E4605F0DD
:10B0A00041FD431B61EB0602B3F57A7F72F10003A9
:10B0B000F5D3454DA16B454AB5FBF1F1092389B2A2
:10B0C00094F83500FDF710FA4388B5FBF3F52564D5
:10B0D000027920684221FEF771F805F023FD05464C
:10B0E0000E4605F01FFD431B61EB0602B3F57A7FA8
:10B0F00072F10003F5D3082241212068FEF75EF8C3
:10B1000005F010FD05460E4605F00CFD431B61EBF6
:10B110000602B3F57A7F72F10003F5D300224321D2
:10B120002068FEF74BF805F0FDFC05460E4605F0DD
:10B13000F9FC431B61EB0602B3F57A7F72F1000361
:10B14000F5D3102251212068FEF738F805F0EAFC0B
:10B1500005460E4605F0E6FC431B61EB0602B3F51F
:10B160007A7F72F10003F5D30A2253212068FEF79B
:10B1700025F805F0D7FC05460E4605F0D3FC431B29
:10B1800061EB0602B3F57A7F72F10003F5D38022FA
:10B1900056212068FEF712F805F0C4FC05460E465D
:10B1A00005F0C0FC431B61EB0602B3F57A7F72F138
:10B1B0000003F5D320680321FEF7B2F903B0F0BD18
:10B1C000062005F00BFD00BF40420F00008E07086F
:10B1D0002DE9F0417C4A0468816B7C4FB7FBF1F1AB
:10B1E00082B006460F2389B290F83500FDF77CF94E
:10B1F00000214388B7FBF3F7054637642046FEF786
:10B200008FF90F224E212046FDF7D8FF4FF00F088F
:10B2100005F088FC06460F4605F084FC831B61EBB5
:10B220000701B3F57A7F71F10003F5D3B8F1010896
:10B23000EED16A794F2102F00F022046FDF7BEFFE2
:10B240004FF00F0805F06EFC06460F4605F06AFC4D
:10B25000831B61EB0701B3F57A7F71F10003F5D32E
:10B26000B8F10108EED16A79502102F00F022046B0
:10B27000FDF7A4FF4FF00F0805F054FC06460F46FB
:10B2800005F050FC831B61EB0701B3F57A7F71F188
:10B290000003F5D3B8F10108EED16A7942EA02124F
:10B2A0005221D2B22046FDF789FF0F2705F03AFC64
:10B2B00005460E4605F036FC431B61EB0602B3F56E
:10B2C0007A7F72F10003F5D3013FEFD103221421FD
:10B2D0002046FDF773FF0F2705F024FC05460E46B8
:10B2E00005F020FC431B61EB0602B3F57A7F72F197
:10B2F0000003F5D3013FEFD13A4663212046FDF725
:10B300005DFF642705F00EFC05460E4605F00AFCBD
:10B31000431B61EB0602B3F57A7F72F10003F5D3AC
:10B32000013FEFD1082265212046FDF747FF0DF1CF
:10B33000070264212046FFF7B5FD9DF8072022F0A3
:10B34000100242F06002642120468DF80720FDF7CC
:10B3500035FF0F2705F0E6FB05460E4605F0E2FB3C
:10B36000431B61EB0602B3F57A7F72F10003F5D35C
:10B37000013FEFD10DF106024D212046FFF792FD6E
:10B380009DF8062002F03F0242F040024D21204687
:10B390008DF80620FDF712FF0F2705F0C3FB0546C9
:10B3A0000E4605F0BFFB431B61EB0602B3F57A7F47
:10B3B00072F10003F5D3013FEFD103212046FEF7E0
:10B3C000AFF802B0BDE8F081388E070840420F00A8
:10B3D000F0B583B015460DF107021C4606460F4630
:10B3E000FFF760FD9DF8072005EA0203A34201D1A3
:10B3F00003B0F0BD22EA050222433946304603B0CD
:10B40000BDE8F040FDF7DABEF0B5044683B00D4666
:10B410001746061D20680379012B18D0022B13D183
:10B420008368DB0732464FF0FF015CBF3246FF21E5
:10B43000FFF7E4FC30B115B12379DB07EAD40FB193
:10B4400023793B7003B0F0BD002003B0F0BD8268EB
:10B45000417C90F9100002F00102CDE90062FF2268
:10B46000F8F7F8FDE6E700BF30B5044683B0051DE8
:10B4700020680379012B14D0022B0FD18368DB07DE
:10B480002A464FF0FF015CBF2A46FF21FFF7B6FCBA
:10B4900010B12379DB07EBD403B030BD002003B03B
:10B4A00030BD8268417C90F9100002F00102CDE9C4
:10B4B0000052FF22F8F7CEFDEAE700BF30B50246A2
:10B4C000044652F8040B0379012B83B00ED0022BF3
:10B4D00009D1FF21FFF792FC18B12079C04300F099
:10B4E000010003B030BD002003B030BD8568417C51
:10B4F00090F91000009205F001050195FF22F8F780
:10B50000A9FDE9E730B5B42283B00446FF21006805
:10B51000FDF754FE10B9002003B030BD2068037958
:10B52000012B04F1040514D0022BF4D18368DB074E
:10B530002A464FF0FF015CBF2A46FF21FFF75EFC61
:10B540000028E8D02379DB07E6D520680379012BB2
:10B55000EAD18268417C90F9100002F00102CDE945
:10B560000052FF22F8F776FDEAE700BF30B50A4641
:10B5700083B00446A5210068FDF720FE10B9002025
:10B5800003B030BD20680379012B04F1040514D009
:10B59000022BF4D18368DB072A464FF0FF015CBF22
:10B5A0002A46FF21FFF72AFC0028E8D02379DB0791
:10B5B000E6D520680379012BEAD18268417C90F9B5
:10B5C000100002F00102CDE90052FF22F8F742FD1F
:10B5D000EAE700BF70B582B0CDE900230446FFF76B
:10B5E00091FF10B9002002B070BD20685522A5213E
:10B5F000FDF7E4FD0028F5D0251D20682A46FF212F
:10B60000FFF750FC0028EDD02379DB07F5D40DF1CE
:10B61000FF350DF1070615F8011F2046FFF7A6FFBD
:10B620000028DFD0B542F6D1DDE700BF002A37D0D1
:10B63000F0B5013A83B004464E1E51FA82F7051D5B
:10B6400016F8012F2068A521FDF7B8FD90B900205C
:10B6500003B0F0BD8268417C90F9100002F0010255
:10B66000CDE90052FF22F8F7F5FC0028EFD023794E
:10B67000DB0710D520680379012BEBD0022BE6D134
:10B680008368DB072A464FF0FF015CBF2A46FF2193
:10B69000FFF7B4FBE9E7B742D2D1012003B0F0BD18
:10B6A0000120704770B5962282B004460E460068AD
:10B6B000FF21FDF783FD10B9002002B070BD251DEC
:10B6C00020680379012B1FD0022BF5D18368DB079B
:10B6D0002A464FF0FF015CBF2A46FF21FFF78EFB91
:10B6E0000028E9D02379DB07EAD4E122206811465B
:10B6F000FDF764FD0028DFD020683246FF2102B04C
:10B70000BDE87040FFF7CEBB8268417C90F9100025
:10B7100002F00102CDE90052FF22F8F79BFCDFE7BF
:10B72000002A46D0F0B5013A4F1C83B004460E46BD
:10B7300057FA82F7051D20689622FF21FDF73EFD8E
:10B7400090B9002003B0F0BD8268417C90F91000F0
:10B7500002F00102CDE90052FF22F8F77BFC00283D
:10B76000EFD02379DB0710D520680379012BEBD0CC
:10B77000022BE6D18368DB072A464FF0FF015CBF4E
:10B780002A46FF21FFF73AFBE9E7E122206811464C
:10B79000FDF714FD0028D4D020683246FF21FFF7C2
:10B7A00081FB0028CDD00136BE42C4D1012003B0B8
:10B7B000F0BD0120704700BF70B505460B4604463A
:10B7C000164655F8040B82B087211A46FDF7F6FCA1
:10B7D00020680379012B18D0022B13D18368DB0773
:10B7E0002A464FF0FF015CBF2A46FF21FFF706FB08
:10B7F00030B12379DA07EBD416B1C3F340133370B9
:10B8000002B070BD002002B070BD8268417C90F92A
:10B81000100002F00102CDE90052FF22F8F71AFCF5
:10B82000E6E700BF70B5782182B00446164600688E
:10B830000022FDF7C3FC10B9002002B070BD251D29
:10B8400020680379012B14D0022BF5D18368DB0724
:10B850002A464FF0FF015CBF2A46FF21FFF7CEFAD0
:10B860000028E9D02379DA07EAD45B09337002B003
:10B8700070BD8268417C90F9100002F00102CDE9B0
:10B880000052FF22F8F7E6FBEAE700BF30B5CC2212
:10B8900083B00446A5210068FDF790FC10B9002094
:10B8A00003B030BD20680379012B04F1040514D0E6
:10B8B000022BF4D18368DB072A464FF0FF015CBFFF
:10B8C0002A46FF21FFF79AFA0028E8D02379DB0700
:10B8D000E6D520680379012BEAD18268417C90F992
:10B8E000100002F00102CDE90052FF22F8F7B2FB8E
:10B8F000EAE700BF30B5B42283B00446FF210068F8
:10B90000FDF75CFC10B9002003B030BD251D206898
:10B910000379012B22D0022BF5D18368DB072A465D
:10B920004FF0FF015CBF2A46FF21FFF767FA0028AE
:10B93000E9D02379DA07EAD4CC212046FFF716FEB6
:10B940000028E0D002E02379DB07DDD520682A4615
:10B95000FF21FFF7A7FA0028F5D1D4E78268417CE0
:10B9600090F9100002F00102CDE90052FF22F8F731
:10B9700071FBDCE72DE9F04F89B00446CDE90623E1
:10B98000002004F1040B0490029103905D462046D0
:10B99000049FFFF7B7FD069BFE0003EBC70B20B922
:10B9A0000AE0237913F0010A0CD020682A46FF210F
:10B9B000FFF778FA0028F4D1079B049A1A7009B0AF
:10B9C000BDE8F08F9B07F7D5F0212046FFF7CEFDAD
:10B9D0000028F1D0069B083E334401270593D0464A
:10B9E0003E46029B002B4AD0082E48D806F1FF396C
:10B9F00043FA09F909F0010920684FEAC9127821D0
:10BA0000FDF7DCFB0028D7D020680379012B47D055
:10BA1000022B43D18368DB072A464FF0FF015CBF4E
:10BA20002A46FF21FFF7EAF90028C5D0237913F051
:10BA30000102E9D103F0600160294FEAD31C51D023
:10BA4000029919B1082E01D8E145B5D1BCF1000F1A
:10BA50003AD01BF808303B430BF808307F00013622
:10BA600017F0FF07F6B2BCD108F101085FFA88F8B9
:10BA7000B8F1080F36D0029B0127002BB4D1049BEC
:10BA8000D3B1039BB34217D9059B13F808301F426B
:10BA900014BF4FF001094FF00009ADE700208BE71C
:10BAA0008268417C90F9100002F00102CDE9005259
:10BAB000FF22F8F7CFFAB7E7039BA3EB0609B9FA21
:10BAC00089F94FEA591997E71BF8081021EA07018D
:10BAD0000BF80810990941EA531313F0010F08BF3E
:10BAE000B246BBE7402E06D8079B049A1B789342C8
:10BAF0003FF64DAF60E79BF807C00BF1FF370BF146
:10BB0000060B17F8011F082382EA010616F0010F41
:10BB10004FEA520218BF82F08C0203F1FF3318BFC4
:10BB2000D2B213F0FF034FEA5101EDD1BB45E8D18A
:10BB30009445D9D1049B0133DBB20493BAF1000FD1
:10BB40003FF43AAFCDF80CA0CEE700BF30B50568A2
:10BB50002B79012B85B0044600F09280022B08D18E
:10BB6000AB68DB0702AA4CBF082188212846FFF7F3
:10BB700045F99DF8083013F0100302D1184605B0BE
:10BB800030BD2068062302AA0021FEF7D1FA002862
:10BB9000F5D09DF809209DF808109DF80A309FED1A
:10BBA0003F6A120202EB01421344140248BF03F140
:10BBB0007F4307EE903AF8EEE77A9DF80C109DF877
:10BBC0000B409DF80D20364BC7EE866A090201EB4B
:10BBD00004410A44090248BF02F17F4207EE902A5D
:10BBE000B3F9742007EE102AB3F97020F8EEE77A63
:10BBF00005EE102A87EE864AB3F96C20B8EEC77AB4
:10BC0000B8EEC55AD3ED1A7AA6EE875AF8EEE75A7F
:10BC100004EE902AE6EE855AB3F97220D3ED197A34
:10BC200003EE902AF8EEE77AB3F96E20E6EEA57AF5
:10BC300006EE102AB3F96220F8EEE44AF8EEE33A91
:10BC400007EE102AB8EEC66AB3F96020A6EEA36A22
:10BC5000E4EE247A05EE902AB8EEC77A66EE846A9E
:10BC6000F8EEE55A27EE047AB6EE005AA5EE857A8C
:10BC7000E6EE867A83ED1F7AC3ED1E7A05B030BDFD
:10BC8000AA68697C95F9100002F00102019202AAEB
:10BC900000920822F8F7DEF96BE700BF0000784851
:10BCA0004059002030B505682B7987B00022012B60
:10BCB00004468DF80F2035D0022B12D1AB68DB077C
:10BCC0000DF10F024CBF2721A7212846FFF796F858
:10BCD00028B19DF80F3013F0080305D1184607B0BE
:10BCE00030BD104607B030BD2068062304AA2821C5
:10BCF000FEF71EFA20B3BDF91030BDF91220002B5B
:10BD0000B8BF03339B10E386BDF91430002AB8BFD7
:10BD10000332002BB8BF033392109B102287638736
:10BD200007B030BDAA68697C95F9100002F00102E5
:10BD300001920DF10F0200922722F8F78BF9C7E765
:10BD4000E086A06307B030BD30B50546002400682A
:10BD5000EC86AC630379012B87B02AD0022B0ED17D
:10BD60008368DB070DF10F024CBF21468021FFF7EE
:10BD700045F828B19DF80F4014F0080402D1204680
:10BD800007B030BD2868062304AA0121FEF7D0F9C8
:10BD90000028F5D0BDF81430BDF81010BDF8122001
:10BDA0005BBA49BA52BA5B42E9862A876B8707B009
:10BDB00030BD22468468417C90F9100004F00104F3
:10BDC00001940DF10F040094F8F744F9D1E700BF96
:10BDD00030B5044600202568E086A0632B79012B4E
:10BDE00087B027D0022B10D1AB68DB070DF10F0213
:10BDF0004CBF062186212846FFF700F828B19DF8A0
:10BE00000F3013F0040302D1184607B030BD20688C
:10BE1000062304AA0021FEF78BF90028F5D0BDF80F
:10BE20001010BDF81220BDF81430E1862287638718
:10BE300007B030BDAA68697C95F9100002F00102D4
:10BE400001920DF10F0200920622F8F703F9D5E7EF
:10BE500010B50368DA6B82B0044612B1904740B166
:10BE600023685B6B1BB1214601A8984718B9FF23D3
:10BE7000E38202B010BDBDF80630013B9BB2F7E78C
:10BE8000F0B585B0044618460D461646039364F097
:10BE9000C9F828442768A073E6732046002400945C
:10BEA000039B7C6932462946A04705B0F0BD00BF20
:10BEB00038B504468B6801600D46984700230B4A4D
:10BEC000226123752B6B13B1204698472075084BD0
:10BED00093F8003E1BB1237D23F00103237500235B
:10BEE000E3822046BDE83840B2E700BF0001FF0012
:10BEF000386A002010B5154BD3F8044E84B024B135
:10BF00002379012B10D0022B02D0002004B010BDE9
:10BF1000A16811F00101024618BF8021204604B03B
:10BF2000BDE81040FAF718BFA268617C8DF80F00D9
:10BF300002F0010294F910000DF10F04CDE9004266
:10BF40008022F8F753F804B010BD00BF386A002013
:10BF50002DE9F041264ED6F8045E84B09DB1B022A2
:10BF600080212846FDF72AF9402280212846FDF746
:10BF700025F9002280212846FDF720F91022802192
:10BF80002846FDF71BF94FF480644FF000080DF1CF
:10BF90000F0795B12B79012B15D0022B0DD1AB6872
:10BFA00013F001034FF000024FF04001284602BF9A
:10BFB0001A4640212846FAF7CFFE013CA4B29CB1B4
:10BFC000D6F8045EE5E7AA6895F91000697C8DF85B
:10BFD0000F8002F00102013CCDE90072A4B24022C0
:10BFE000F8F704F8002CEBD104B0BDE8F08100BFF5
:10BFF000386A00200B4B10B5D3F8044E8CB1503882
:10C00000C2B280212046FDF7D9F8002280212046C7
:10C01000FDF7D4F820461022BDE810408021FDF73E
:10C02000CDB810BD386A0020F0B5204C204F203824
:10C0300000EB8000661DD7F8045E85B0044406441A
:10C04000E5B12B792278012B1DD0022B0AD1AB68E8
:10C0500013F0010F4FF04001284604BF402128464D
:10C06000FAF77AFE0134B442EAD155B100224021F8
:10C07000284605B0BDE8F040FDF7A0B80134B44251
:10C08000F0D105B0F0BD8DF80F20AA6895F9100029
:10C09000697C02F0010201920DF10F020092402230
:10C0A000F7F7A4FFD7F8045EDCE700BF948E07081B
:10C0B000386A00202DE9F041734ED6F8045E84B052
:10C0C000002D00F09680D42280212846FDF776F8D6
:10C0D000802211462846FDF771F8A82280212846C3
:10C0E000FDF76CF83F2280212846FDF767F8D32240
:10C0F00080212846FDF762F8002280212846FDF7BE
:10C100005DF8402280212846FDF758F88D228021D5
:10C110002846FDF753F8142280212846FDF74EF8F3
:10C12000A12280212846FDF749F8C822802128460F
:10C13000FDF744F8DA2280212846FDF73FF8122265
:10C1400080212846FDF73AF8812280212846FDF714
:10C1500035F8CF2280212846FDF730F8D9228021FA
:10C160002846FDF72BF8F12280212846FDF726F816
:10C17000DB2280212846FDF721F840228021284635
:10C18000FDF71CF8A42280212846FDF717F8A62207
:10C1900080212846FDF712F8AF2280212846FDF7BE
:10C1A0000DF8A62280212846FDF708F8AE2280214E
:10C1B0002846FDF703F8202280212846FCF7FEFFE1
:10C1C000002280212846FCF7F9FFB0228021284672
:10C1D000FCF7F4FF402280212846FCF7EFFF002205
:10C1E00080212846FCF7EAFF102280212846FCF730
:10C1F000E5FF4FF480644FF000080DF10F0755B3D1
:10C200002B79012B2FD0022B0DD1AB6813F001033A
:10C210004FF000024FF04001284602BF1A4640216D
:10C220002846FAF799FD013CA4B2002CE7D175B17C
:10C23000812280212846FCF7C1FFC82280212846A0
:10C24000FCF7BCFFAF2280212846FCF7B7FF012096
:10C2500004B0BDE8F081013CA4B2002CE3D1012080
:10C2600004B0BDE8F081AA6895F91000697C8DF8EA
:10C270000F8002F00102CDE900724022F7F7B6FE0E
:10C28000D6F8045ECFE700BF386A0020FBF70CB891
:10C29000FBF70AB8FBF708B8FBF706B8FBF704B8DA
:10C2A000FBF702B838B50409013C032C1BD8104D2C
:10C2B00005EB440200F00F03B2F8DC1541FA03F27B
:10C2C00012F0010211D001209840013808402C449E
:10C2D0006CF048FA94F8E435064A184400EB400044
:10C2E00002EB800038BD002038BD104638BD00BFCD
:10C2F0005C8B0708742500202DE9F04F542204467A
:10C300000021BF4893B06AF07DFBBE4A611EE01C6D
:10C31000144611F8013F5D1E052D88BF0023884299
:10C3200044F8043BF5D102F11003114651F8040B17
:10C33000012800F07D819942F8D1114651F8040B93
:10C34000022800F053819942F8D1114651F8040BAC
:10C35000032800F077819942F8D152F8041B042990
:10C3600000F03A819A42F8D10520FAF7A1F90620A7
:10C37000FAF79EF9A24DDFF8A892DFF8A8821A26F4
:10C3800000272C7B002C40D02046FFF78BFF95F92F
:10C390000DA08346E0B103689B498BF8076003F169
:10C3A0003F4303F57E039B0A0522C85C8BF80620F9
:10C3B00000238BF8083060F043FF944ABBF8043048
:10C3C0000492DBF80000039303A9F6F777FF2C7BB8
:10C3D0000023302201E019F8332094422ED001339B
:10C3E000102BF8D100200AEB4A0A08EBCA030122FD
:10C3F000D3F8641728618C180720C3F8644729759F
:10C40000A8756A7583F8602717440136F6B2202EA6
:10C4100005F10C05B5D177B17D4CDFF80CA2DFF842
:10C420000C920025237C7BB90135032D04F11804FF
:10C430000AF58C7AF6D113B0BDE8F08F754A02EB9D
:10C44000C303D3F8EC05CEE7607960F0F9FE2079FC
:10C4500060F0F6FEA068F6F79BFE2368A068CDF8B2
:10C4600014A04C3304936369142202FB03F3079373
:10C470000023CDE90E33CDE9103306930893E3682A
:10C4800003934FF480624FF40063CDE909234FF426
:10C4900000514FF48073CDE90B134FF4003303A91F
:10C4A0000D9360F0C1FFA2685B49136843F001037C
:10C4B0001360D9F8043023F4733323F4477323F063
:10C4C000030343F44033C9F80430226863695068B9
:10C4D000012B20F0407020F48070D4BF002601268C
:10C4E00040EA062050609068014041F002019160EE
:10C4F000D16A013B21F47001DBB241EA0353D362FC
:10C500003F4B012103F148074FFA85F802E00C3355
:10C51000BB422ED0587D0028F9D093F90D0040453C
:10C52000F5D1187C9E7D01F1010C09285FFA8CFC85
:10C5300030D800EB400E06FA0EF6D2F810B0019695
:10C54000072606FA0EFE019E2BEA0E0E46EA0E069E
:10C550001661062930D8013901EB81011F26884078
:10C560008E406146D2F834C02CEA06063043506350
:10C57000CDE7936843F400739360936843F480734A
:10C580009360936843F001039360936843F08043A2
:10C59000936049E7A0F10A0E0EEB4E0E4FF0070B29
:10C5A00006FA0EF60BFA0EFED2F80CB02BEA0E0EBF
:10C5B00046EA0E06D660CCE70C294DD8073901EBC8
:10C5C00081011F2688408E406146D2F830C02CEA97
:10C5D0000606304310639AE7104B93F88C2A3021FB
:10C5E000013283F8681A83F88C2ABDE60B4991F86A
:10C5F0008C0A3524013081F8504A81F88C0AA4E66F
:10C600007074002044590020288B070803000100A3
:10C61000B01200205C8B0708FDF7FFC0386A0020CD
:10C6200044910708600B0020C874002000230140DB
:10C63000104991F88C0A3424013081F8444A81F879
:10C640008C0A7AE60B4991F88C0A2024013081F893
:10C650005C4A81F88C0A80E60D3901EB81011F26C6
:10C6600088408E406146D2F82CC02CEA0606304342
:10C67000D0624CE7386A002010B503681A79022AA4
:10C68000044603D000232371236010BD987AFFF77E
:10C6900009FE0028F6D040F61A610022C18002721D
:10C6A0002021FCF7EBFE00232371236010BD00BFA7
:10C6B00070B506461C48336803F13F4303F57E031B
:10C6C0009B0A82B0C05C0C46154660F0B9FDB2888A
:10C6D0000092B2FA82F304F003028DF80420C4F34E
:10C6E000810230688DF80520C3F11F03C4F30012E6
:10C6F00064098DF80740C3F3CC0400EB840403F015
:10C7000007038DF806209B00226A0F269D4006FA3B
:10C7100003F322EA03032362226A15436946256272
:10C72000F6F7CCFD02B070BD288B07082DE9F04F5D
:10C73000AE4CAF4DAC4283B050D21E4602E00C343A
:10C74000AC424BD294F805C08C45F8D194F804C0A3
:10C75000844501D00028F2D194F807C09445EED169
:10C760002568002D3BD000236B60AB60EB602B6134
:10C770006B61AB61EB612C6022792A71A779AF60A4
:10C78000217AE960012A33D0022A27D1E07AFFF723
:10C7900089FD94F90980A861A07A85F81080FFF7D7
:10C7A00081FD6861F8B1934C08EB880A4FEA88096B
:10C7B00054F82A3004EB8A0AABB19AF8123003B36A
:10C7C0000E2200238671C27103720921FCF756FE06
:10C7D0006B6923B11A689B88138300E00025284603
:10C7E00003B0BDE8F08F2846FFF746FF0025F6E7C7
:10C7F000E07AFFF757FD627AA37A6B74A8612A7416
:10C80000EDE79AF8080060F01BFD9AF808104A0955
:10C81000012301F01F01023A8B40032A08D8DFE808
:10C8200002F0B6BCB00274494A6922EA03034B61C4
:10C8300009EB080304EB830308F1010B5879FFF7B8
:10C8400031FD5FFA8BFB824620B140F60A3380F857
:10C8500008B0C38009EB080304EB8303D879FFF722
:10C8600021FD034620B140F60A5280F808B0C2808C
:10C8700009EB080204EB820201939079FFF712FDA5
:10C88000019B20B140F60A4280F808B0C28009EB53
:10C89000080B04EB8B0B17F004079BF8092000F042
:10C8A0008280BAF1000F0AD050464A21FFF700FFFC
:10C8B0009BF80700FFF7F6FC9BF80920034643B1FD
:10C8C00018462A21FFF7F4FE09EB080304EB830363
:10C8D0005A7A019209EB080304EB83039879FFF776
:10C8E000E1FC18B1019A0A21FFF7E2FE09EB080BFF
:10C8F00004EB8B0B9BF804A0BAF1000F40F08A8088
:10C9000009EB08033D4A54F82330934200F0A68017
:10C910003B4A934200F0B8803A4A934200F0A98023
:10C92000394A934200F08F80384A934200F0808069
:10C93000374A934200F0B3801A88002F02F4415125
:10C940000CBF032200220A4342F445721A809A8BDC
:10C9500022F400621204120C9A8307221A821A88A7
:10C9600092B242F040021A80BAF1000F35D1C844A9
:10C97000686904EB88040123A37400283FF425AF01
:10C980001EE71D490A6922EA03030B6150E71A49B1
:10C990004A6A22EA03034B624AE717490A6A22EA13
:10C9A00003030B6244E7BAF1000F0AD050460A2194
:10C9B000FFF77EFE9BF80700FFF774FC9BF8092049
:10C9C0000346002B85D018460A21FFF771FE09EBBC
:10C9D000080304EB83035A7A7BE75046FFF762FCB7
:10C9E0000028C4D0036882881A83C0E718AB0808FF
:10C9F000D4AC08086000002000380240003001403C
:10CA000000380040003C004000340140005001402C
:10CA1000005401405046FFF745FC00283FF470AF3A
:10CA20009BF809200921FFF743FE9BF804A067E764
:10CA300002F56842516A41F480115162516A21F451
:10CA40008011516278E702F58232516A41F4005157
:10CA50005162516A21F4005151626DE702F584324E
:10CA6000516A41F480515162516A21F480515162FE
:10CA700062E702F5FE32116A41F400411162116A67
:10CA800021F40041116257E702F50032116A41F4C6
:10CA900080411162116A21F4804111624CE702F574
:10CAA0006442516A41F400115162516A21F400114B
:10CAB000516241E72DE9F043002383B01A46362145
:10CAC0000120FFF733FEDFF87C900746C9F8080E17
:10CAD00060B34FF00508962604F024F804460D468E
:10CAE00004F020F8031B61EB0501B3F57A7F71F1C7
:10CAF0000003F5D3013EEFD10DF107023146384670
:10CB0000FEF7D0F9044668B9B8F10108E3D199F805
:10CB10000C3ED9F8080E0C2B04BF0223C9F8103EB6
:10CB2000FFF7AAFD204603B0BDE8F08399F80C3E5C
:10CB30000C2B01D00446F5E70123C9F8103E04464A
:10CB4000F0E700BF386A0020074B53F8203021B1CE
:10CB50004BB11A689B8853837047002BFCD01A682E
:10CB60009B881383704770474C8B07081D4B70B52B
:10CB7000D3F8184174B193F8C83D05465BB16268BB
:10CB80005379032B2BD8DFE803F021242702136805
:10CB900040331D6070BDE068666881680A6822F0F5
:10CBA00001020A603168104A767932F816608A8983
:10CBB00092B222EA06028A8123740A8892B242F073
:10CBC00001020A800377FAF767FCD8E71368343369
:10CBD000DFE713683833DCE713683C33D9E7002319
:10CBE0001B60FFDE405900205C8A0708254BD3F804
:10CBF00018219AB193F8C81D81B110B5224C94F850
:10CC0000301E03290BD0022911D0002283F8C82D31
:10CC1000FAF76AFB08B984F8310E10BD7047526804
:10CC20005379032B2AD8DFE803F023201D1852681C
:10CC30005379032B1FD8DFE803F00D0A07021368AE
:10CC4000403300221A6010BD13683C33F9E71368C3
:10CC50003833F6E713683433F3E71368403364225C
:10CC60001A6010BD13683C33F9E713683833F6E7F0
:10CC700013683433F3E700231B60FFDE00231B60DF
:10CC8000FFDE00BF40590020386A00202DE9F04F38
:10CC9000BA4BDFF8F4E293F8349E93F8358E93F8AC
:10CCA000367EDFF8E8A283B0002603F638650196E9
:10CCB0000124AB78E978C3F1FF039BB2002B40F06D
:10CCC00092800B460F468C460A46884689460121CB
:10CCD0000191100240EA0340172240EA0C0006EBE3
:10CCE000020CACEB02032A3304FA02F19BB20142BC
:10CCF0000EEB830314BF02210121013AC3F81C117A
:10CD0000531CEED19E4B04351836AB42B6B2D0D18F
:10CD10009A4A4FF44073A2F8B83E2023A2F8BA3ED4
:10CD2000019B2BB182F8349E82F8358E82F8367ED4
:10CD3000924B93F8313E002B52D0DEF81831002B85
:10CD40004ED0EFF31181102282F31288D8685D680B
:10CD50008468226822F0010222602C68894A6D7979
:10CD600032F81550A28992B222EA0502A281026924
:10CD700044681F2A40F2E080203A202000FA02F2A4
:10CD8000E260CAB282F31188DA68DEF818019268AC
:10CD900040F22B31516011680124214311601C7451
:10CDA00003681A7DA24204BF02221A7593F82C1060
:10CDB0000CBF4FF400720022012904D1022183F834
:10CDC0002C1042F4806293F84410012900F0B980DD
:10CDD00093F85C10012900F0BD80002A40F0BF806C
:10CDE00003B0BDE8F08FB5F800C0C3F1FF03AAFBA4
:10CDF0000CB001FB03F340091B120A46052800F2A0
:10CE0000B980DFE800F0886C53361C03AAFB0C07DE
:10CE10007F09C7EB0717ACEB8707BFB2C81AC7F18A
:10CE20003C0700FB07F7AAFB07075FFA83F808EB4C
:10CE300057178946FFB20121BC46019149E7AAFB79
:10CE40000C025209C2EB0212ACEB820292B2A1EBCD
:10CE5000030902FB09F9AAFB09295FFA83F808EB29
:10CE600059198C465FFA89F90F4601214A4601910A
:10CE70002FE7AAFB0C025209C2EB0212ACEB8208AC
:10CE80001FFA88F8CA1AC8F13C0802FB08F8AAFB86
:10CE900008285FFA83F909EB58188C465FFA88F87E
:10CEA0000F4601211A460191434612E7AAFB0C02E4
:10CEB0005209C2EB0212ACEB820292B2CF1A02FB11
:10CEC00007F7AAFB07275FFA83F909EB57171A46FA
:10CED000FFB20B4688460121BC460191F9E6AAFB48
:10CEE0000C025209C2EB0212ACEB82091FFA89F95B
:10CEF000CA1AC9F13C0902FB09F9AAFB0929DFB2E8
:10CF000007EB59195FFA89F99C4688460B460121BF
:10CF10004A460191DDE6A1EB03080CFB08F8DFB2FD
:10CF2000AAFB080807EB58185FFA88F89C4601230B
:10CF3000019389464346CCE6202000FA02F2A26023
:10CF40001FE7022183F8441093F85C10012942F492
:10CF5000006204D1022183F85C1042F480524368DD
:10CF60001B6800215962998989B20A439A8103B0EA
:10CF7000BDE8F08F43464A46BC46AAE6386A002020
:10CF8000F07800205C8A070840590020898888884A
:10CF90002DE9F041314F00243B461D79212D03F14D
:10CFA000140304D001340C2CF7D1BDE8F08104EB5C
:10CFB000840007EB8000F5F765FDDFF8AC800646DE
:10CFC000C8F818010028F0D02846FFF76BF9244D67
:10CFD000C5F8BC0E58B1142202FB047440F21522AD
:10CFE000C28000220272227A4A21FFF761FB95F883
:10CFF000303E022B29D0032B1FD0FAF775F910B958
:10D0000085F8310ED1E740F6AC421648002169F0B0
:10D01000F9FC95F8303E012B04BFFF23C8F8C43D4E
:10D0200098F8C83D012285F8312E002BBDD1337C04
:10D03000002BBAD1BDE8F04128E6FAF72DFA3046C8
:10D04000F5F73CFF64230360AFE7FAF725FA3046B3
:10D05000F5F734FF00230360A7E700BF0C0A0020A8
:10D06000386A00205C5A0020405900202DE9F04F1A
:10D07000DFF828A2884E0021A7B04FF00A0B0C461B
:10D080000AF56C658FE096F8CC3101965F0618D4EE
:10D0900004F1020C43F04003BCF18C0F86F8CC3154
:10D0A00000F2E38004F198010DEB010904F199010C
:10D0B0000DEB010764464FF0040C09F88CCC07F81F
:10D0C0008C3CA71C8C2F42F0020C00F2CE8004F1A5
:10D0D00098036B444FF0050103F88BCC04F1040C6A
:10D0E000BCF18C0F03F88C1C00F2BF8004F19A0194
:10D0F0000DEB01074FF0060907F88C9C009F03F821
:10D10000897C4FEA880804EB09075FFA88F88C2FBE
:10D11000414600F2AA8004F19C0CEC444FF0070851
:10D120000CF88C8C04F1080CBCF18C0F03F8871CF4
:10D1300000F29B8007F198010DEB01074FF005010C
:10D1400007F88C1C03F8852C04F10A028C2A00F2E3
:10D150008C8004F1A0010DEB010C00990CF88C9C63
:10D1600003F8831C04F10C018C297ED804F1A2027F
:10D1700004F1A3036A446B4402F88C8C0C4603F858
:10D180008CEC410900F01F0755F821300122BA400C
:10D1900023EA0203BBF1010B45F821306FD0411C9B
:10D1A000B1F5F07F6BD23C222846FAF79DF90028B2
:10D1B0005EDB0AEB4003C1B2B3F8FC3E00915907B5
:10D1C000C0F307225FFA83F84FEA132E3FF55BAFF7
:10D1D00096F8CC710196790603D407F0380CC44553
:10D1E00019D027F078073B4304F1020CDBB2BCF105
:10D1F0008C0F86F8CC3138D804F198010DEB01087A
:10D2000004F199010DEB010764464FF0040C08F896
:10D210008CCC07F88C3CA31C8C2B26D804F19801ED
:10D220000DEB010707F88B2C052207F88C2C221D2B
:10D230008C2A1AD804F19A036B444FF0060C04EBC5
:10D240000C0103F88CCC8C29009B07F8893C0CD886
:10D2500004F19C0204F19D036A446B440C460721CF
:10D2600002F88C1C03F88CEC8BE76FF0004488E725
:10D27000204614B927B0BDE8F08F074B0193019BFE
:10D2800003AAD3F8C4010021234662F085FD0120E2
:10D2900027B0BDE8F08F00BF307B0020386A002047
:10D2A000F0B52A4CD4F8C40183B010B194F8CA3157
:10D2B0000BB103B0F0BD0DF107028421012384F806
:10D2C000CA31FDF7EFFD94F8CC21D4F8C40142F047
:10D2D00004020421FBF772FFD4F8C4010DF1070228
:10D2E0008421FDF7DFFD9DF8073013F00406F3D12C
:10D2F000174D184884F8CC3131463C2269F082FB46
:10D3000005F570773146A5F13A0E012635F8023F52
:10D310001A0A22F0200203F0040301F01F00134355
:10D320004FEA511C06FA00F001F1010104D05EF849
:10D330002C3018434EF82C00BD42E7D1FFF796FE83
:10D340000028FBD184F8CA0103B0F0BD307B002077
:10D3500032790020F878002070B5414DD5F8C441ED
:10D3600082B094B395F8C831012B42D0022B2ED154
:10D37000082294F910303B4885F8CB2103EB830356
:10D38000042150F823008DF8052000238DF8043087
:10D39000A3688DF806109A078DF8071042D504236C
:10D3A0000DEB0302002162F0A7FCA3689B0722D5C6
:10D3B0002D483C22FF2169F025FB95F8C93123B99E
:10D3C000FFF76EFF012385F8C93102B070BD0DF182
:10D3D0000302A0212046FDF765FD9DF8033003F010
:10D3E0000503012B37D0002B2FD1D5F8C4410822DB
:10D3F000BFE74822BDE71D4B1D491A681D4B486811
:10D400004FF4FA7606FB02F2A3FB023292094B6854
:10D410001B1A9A42FBD26369002BC9D01A689B88F9
:10D420001383C5E7636913B11A689B8853830F4B55
:10D430000F491A680F4B4E68D200A3FB02329209C3
:10D440004B689B1B9A42FBD2A9E70B4A126840F239
:10D45000DC539A42B9D9D5F8C441482289E700BFC4
:10D46000307B002060000020F87800206824002035
:10D47000001000E0D34D62106C240020F0B52F4B5B
:10D480008BB04FF4005103F5707223F8021F9342E2
:10D49000FBD12B4E2B4C356804F2CB17323502E012
:10D4A00033689D4243D9D4F8C4013A468021FDF740
:10D4B000F9FC0028F4D110220346234E01250AE08E
:10D4C0000EF8242C0132D2B2202A034601F8245C43
:10D4D0000CF1040C12D0981C03F1280703F1290168
:10D4E00022280DEB070E69449C46E9D90132D2B2DD
:10D4F0006FF00043202AB4461846ECD1BCF1220F4D
:10D5000018D800F128020DEB020003F128020121D6
:10D510006A4400F8241C4C21023302F8231CD4F87E
:10D52000C40101AA002162F037FC0BB0F0BD10224B
:10D530000023C2E76FF00043F1E700BF327900201B
:10D540006C240020307B0020010000802DE9F04198
:10D55000334D95F8CA3182B004460E46002BFDD1FA
:10D5600095F8CB21D5F8C401194602F0F702012342
:10D5700085F8CA3185F8CB21FBF720FEE2B20746D9
:10D580000921D5F8C401FBF719FEB4F5807F3FD01F
:10D59000D5F8C401DFF88C8050220821FBF70EFE7D
:10D5A000D5F8C4010DF10702A021FDF77BFC48B9B5
:10D5B000D8F8D830B8F8DC2059690A4214BF5A8329
:10D5C0001A83EDE79DF8074014F02004F0D1E2B291
:10D5D0000A21D5F8C401FBF7F1FD3219D5F8C401D1
:10D5E000C0210134FDF75EFC362CF0D157B995F817
:10D5F000CB21D5F8C40102F0F702394685F8CB21DA
:10D60000FBF7DCFD002385F8CA3102B0BDE8F081EC
:10D61000D5F8C40140220A21FBF7D0FDB8E700BFCE
:10D62000307B0020742500202DE9F04F5F4E96F8E6
:10D63000CA41C3B005460F46002CFDD196F8CB2158
:10D64000D6F8C40102F0F7020123214686F8CB2167
:10D6500086F8CA31FBF7B2FDFF2D4FF009038DF8B4
:10D66000055088BFAD0801AA88BF05F0C008137037
:10D6700098BFA04602234FF0000C4FF00A0B0DF1AB
:10D68000050A4FF00B0914E0B4F5827F02F803B0ED
:10D690000AF8031017F80C3017D80CF1010CBCF184
:10D6A000360F02F8059000F1060002F80E3023460E
:10D6B00014D09D1C48EA0C01B5F5827F03F10404E7
:10D6C0001846C9B203F1030EDED90CF1010C6FF05C
:10D6D0000044BCF1360F36482346EAD1B0F5827FCC
:10D6E00061D8082111550DF10501A020C85402335D
:10D6F000D6F8C4412F4894F9101001EB810150F87D
:10D700002100A168890722D5002162F0F5FAA368FB
:10D710009B0731D5284CD6F8C4010DF10302A02196
:10D72000FDF7C0FB48B9D4F8D830B4F8DC2059690B
:10D730000A4214BF5A831A83EDE79DF8033013F0B1
:10D740002003F0D186F8CA3143B0BDE8F08F61699B
:10D7500011B10D68898869831849194F0D681949F5
:10D76000D7F804C0ED00A1FB0515AD097968A1EB60
:10D770000C018D42FAD2C7E7104B11491A68114BC0
:10D7800048684FF4FA7505FB02F2A3FB02329209D6
:10D790004B681B1A9A42FBD26369002BBAD01A68F5
:10D7A0009B881383B6E76FF00043A1E7307B00202E
:10D7B0000100008060000020742500206824002003
:10D7C000001000E0D34D621010B58379C26B13F0E6
:10D7D000010F0446406B20D013F0200F526814BF95
:10D7E0000221422120B1127AFEF762FFE36B5A68F0
:10D7F000012384F86032A4F85C3250790B4C116834
:10D80000205C0A8C83409BB292B222EA03020A8413
:10D810000A8C92B213430B8410BD13F0200F526890
:10D8200014BF022122210028DDD1E1E75C8B07082B
:10D8300038B54368344A1B68934204462BD002F53E
:10D840008062934227D002F57052934223D002F5B2
:10D85000806293421FD002F5806293421BD02B4B13
:10D860001A6852081346B3FBF1FCBCF5803F15D291
:10D870001FFA8CF12046F5F7A1F923681A6853794D
:10D880000BBB937973B963681A6813889BB243F032
:10D890000103138038BD1D4B1A68E3E7012BE4D95F
:10D8A0005B08E0E75AB2002A1FDB194801218518FE
:10D8B00003F01F03520901FA03F3302185F8001326
:10D8C00040F82230DFE759B2002915DB104D012066
:10D8D00005EB010C03F01F03490900FA03F33020A4
:10D8E0008CF8000345F82130CBE70A4A03F00F0318
:10D8F0001A4430231376C6E7064903F00F03194490
:10D9000030230B76BDE700BF00000140080800206F
:10D9100000E100E0FCEC00E02DE9F04F89B0CDE93A
:10D920000312BA4A9DF848A09DF84C70012805469C
:10D930001E4615BF4FF0360B4FF01B0B4FF037094B
:10D940004FF018091346104600240179494500F1AB
:10D95000140004D001340C2CF7D1002403E004EBB4
:10D96000840403EB840400201179594502F1140268
:10D9700005D001300C28F7D14FF0000803E000EB90
:10D98000800003EB80085846FEF78CFCD945024620
:10D9900032D017F00803029336D11AF0010F00F0CD
:10D9A000EF800592002C00F05181A079430700F12F
:10D9B0004D812046F5F766F8954B01934FF41C7C9A
:10D9C0000CFB0534C4F80C02002800F03F814846E7
:10D9D000FEF768FC691C059AC4F80402C9B220B1BC
:10D9E00040F2046C0172A0F806C01AF0020305931D
:10D9F00040F0188102932DE00AF003000328C8D1FB
:10DA0000082347F008070293B8F1000F00F01E81C9
:10DA100098F8061005924A0700F118814046F5F77C
:10DA200031F87B4B01931A464FF41C7303FB05231B
:10DA3000C3F80C02002800F00981059AC3E981228D
:10DA40006B1CDBB21AB1137240F20473D3800AF07C
:10DA500002030593019BDFF8C8914FF41C7202FB8F
:10DA600005FB03EB0B040BF15C014944C4F8E41122
:10DA70000BF5AE714944039BC4F8E8114FF4807173
:10DA80004FF00008C4E97711C4F8FC316149049BE8
:10DA9000C4F80032D4F80C0284F8D671C4F8D0115E
:10DAA000C4E97B883146C4E97D8884F8D5A1C4F8EF
:10DAB000D86184F83C54C4F83884A4F83084FFF763
:10DAC000B7FE07F00101D4F80C025FF021FC059BC2
:10DAD00009EB0B07002B78D0D4F81002002874D083
:10DAE000D4F80C1249680B684168096899426CD0F7
:10DAF0003146012684F83D64474EFFF799FEC4F88D
:10DB000018620BF14401454ED4F80C02C4F81472AB
:10DB10004944C4E98878C4F81C82C4F82862F5F73F
:10DB200009F80BF15001D4F810024944F5F702F856
:10DB3000029B002B63D1019A4FF41C7303FB052356
:10DB4000D3F81022D3F80802002A00F084800028BD
:10DB500055D0536801211A7AFEF7AAFD019B4FF4B4
:10DB60001C7000FB053494F8D63113F0010FD4F883
:10DB7000083274D1002B42D01A689B8813833EE090
:10DB80001AF002030593224B01933FF463AF4FF465
:10DB90001C7101FB0531C1F80822B8F1000F55D006
:10DBA0004046CDE90612F4F76DFF0699C1F80C0264
:10DBB00000284BD0691C079AC9B2002A3FF44AAF2B
:10DBC00040F204531172D38044E7019A4FF41C735E
:10DBD00003FB0523104AC3F81822104AC3F81C227D
:10DBE0000BF144010022D3F80C02C3F8147283F83D
:10DBF0003D244944F4F79EFF029B002B9BD03846FE
:10DC0000FFF7E2FD384609B0BDE8F08F0C0A0020AE
:10DC1000307B0020C4910708D1DF000889E00008AC
:10DC2000007D00200791019906924FF41C73404635
:10DC300003FB0518C8F80822F4F724FFD8F80C32C3
:10DC4000C8F81002DDE90621002BB6D100273846BE
:10DC500009B0BDE8F08F0121FBF710FC7EE7002B37
:10DC6000CDD01A689B885383C9E700BF437913F06E
:10DC7000010306D0D0E90731C268581A531E184074
:10DC800070471846704700BF437913F0020307D06E
:10DC9000D0E9093200699B1A013820EA0300704775
:10DCA000184670474379024613F0010018D010B4AB
:10DCB000D168146AD369481E1B1B03400CD05369FA
:10DCC0001B5D04F1010CD8B2BCFBF1F301FB13C1E5
:10DCD0005DF8044B1162704718465DF8044B7047BD
:10DCE000704700BF43799B070AD5436A8269D154C4
:10DCF000436A02690133B3FBF2F102FB1133436261
:10DD0000704700BF41717047D0E90920101AB0FA7E
:10DD100080F04009704700BF014B1B685B681847E3
:10DD200008820020024B1B6808309B68184700BF20
:10DD300008820020012070470120704701207047B1
:10DD4000012070470120704731B10C4BD3ED017AAF
:10DD5000F8EEE77AC1ED007A72B1084BDFED086AA0
:10DD60009B68A3F5D543333B07EE903AF8EEE77A8C
:10DD700087EEA67A82ED007A704700BF0882002005
:10DD80000000C8420120704701207047704700BF63
:10DD9000034B03EB8000C3680BB19B6819607047AD
:10DDA00008820020044B03EB8003DB680BB19B6807
:10DDB000196023F065BC00BF08820020044B03EB10
:10DDC000C00040F2FF739942A8BF19468180704796
:10DDD000506700200C4A13787BB10C4B93F84C1021
:10DDE00059B193F84D1059B150680022FA2883F8C0
:10DDF0004D20A8BF4FF0FF3070476FF00100704713
:10DE00006FF00200704700BFF81200200882002067
:10DE10002DE9F041114C04F1500884F851101746D7
:10DE2000002502234246FF21064684F85050FCF7A5
:10DE300007F980B1424630460223FF21FCF778F90A
:10DE400048B194F8502094F8513003EB022328464F
:10DE50003B80BDE8F0816FF00C00FAE708820020FB
:10DE60000B4B93F8502182B193F8512152B10949DB
:10DE700088680022B0F5967F83F85121A8BF4FF043
:10DE8000FF3070476FF0020070476FF0010070477D
:10DE900008820020F8120020024BD3F854315B684E
:10DEA000184700BF08820020024BD3F854319B680A
:10DEB000184700BF08820020024BD3F85431DB68BA
:10DEC000184700BF08820020014BD868704700BF88
:10DED000F8120020044B93F8583113B1034B186922
:10DEE00070476FF00100704708820020F812002090
:10DEF000437A5A1C0344D2B242729972037A934213
:10DF000000D97047002AFCD010B5044604F10A017C
:10DF1000D0E9003098470023637210BD2A4ED6F82E
:10DF20005C51D6F8680108B52EF02AFC28462EF080
:10DF300027FCD6F8680141798B073ED500210846B9
:10DF4000FEF702FE00210120FEF7FEFD1F4CD6F871
:10DF5000680103685B689847D0B92B6828465B68FE
:10DF600098470028F3D0D4F89C202B68B4F8A01070
:10DF7000DB685183284698470146D6F86801026855
:10DF800013689847D4F89C30B4F8A0201A83DEE7D1
:10DF9000D6F86801D4F8D8200368B4F8DC10DB6840
:10DFA000518398472B6801461B6828469847D4F848
:10DFB000D830B4F8DC201A83CFE7036841F00201BF
:10DFC0009B699847BAE700BF0882002074250020AB
:10DFD00038B583681C686379DB0748D5A37994F862
:10DFE0005C2203F001010D461ABB94F85F32012B4D
:10DFF0003ED0002B40D194F85E3294F85DC2634568
:10E000000DD2B4F866224FF0010E0EFA03F0013380
:10E010000243D8B2604592B2F7D3A4F86622012336
:10E0200084F85F32E06B85EA0301BDE838405FF0B9
:10E030006FB9E06B43681A68D36AC3F34E03536247
:10E0400094F86D32012B07D094F8613223B1B4F803
:10E0500068320133A4F8683285F001015FF058F9A5
:10E0600000224FF08073A4F86622C4F85C3238BDF9
:10E0700094F85D3284F85E32002384F85F32E06BFE
:10E08000BDE838405FF044B938B583681C686379EF
:10E09000990745D4D90700D438BD94F85C32002BD9
:10E0A000FAD194F85D320133DBB2092B84F85D328A
:10E0B00000F0AC800A2BEFD194F85F52002D00F0F5
:10E0C000C480B4F86602820500F0010302D4002B7C
:10E0D00040F0C480B4F86A320133A4F86A320123F4
:10E0E0009D42A4F85C32D7D1A179E06B002384F87B
:10E0F0005F3201F001015FF00BF9E36B76485B687A
:10E100005A791968835C0A8C05FA03F39BB292B2C0
:10E1100022EA03020A840A8C92B213430B8438BDAC
:10E1200094F86112002967D1D4E90902904200F005
:10E130009E80501CA569A062AA5C25695200A84275
:10E1400034BF05460D4694F86002A56242F40072A1
:10E150000A254FF0010CA4F8642284F8625284F876
:10E1600061C2002850D0A07905071CD410F04005EA
:10E1700090D009214FEA520CC00702F0010248BFBB
:10E1800082F00102A4F864C2002A57D1A26B12B136
:10E1900010689288428384F86212002D3FF47AAFAF
:10E1A00000292DD076E7E36B4B485D686B792A68D0
:10E1B000C35C606B0CFA03FC138C9BB223EA0C0C5F
:10E1C000A2F820C0138C9BB2138410B12A7AFEF7F8
:10E1D0006FFA236CA06B002284F86022002B64D0BD
:10E1E00020B15B6801211A7AFEF762FAA37913F075
:10E1F000400F63793FF44EAF94F9621200294CD17D
:10E20000002284F8612245E7A079AFE794F85F32F5
:10E21000002B7FF441AF94F85E32082B3FF63CAF01
:10E22000B4F86622012000FA03F101330A43D9B29F
:10E23000082992B2F7D9A4F8662238BDA26B002A49
:10E24000A9D0106892880283A5E7B4F8663243F03B
:10E2500001009B05A4F866023FF53CAFE36A400865
:10E260003BB3216BC0B2984794F85F5237E794F8FC
:10E27000601200297FF40EAFA27912077FF50AAF72
:10E28000236CA06B23B318B15B681A7AFEF710FAFF
:10E290002046FFF799FA6379FCE6A079B4F8642286
:10E2A000013949B200F0400564E70121FBF7E6F8C7
:10E2B0009CE7E3696269C0B2D054E369E26894F80C
:10E2C0005F520133B3FBF2F102FB1133E36106E766
:10E2D0001946FBF7D3F8DBE75C8B07080346C06BF6
:10E2E0009960FFF7A5BA00BF30B5032083B00D4693
:10E2F0001446FBF78BF801909DB107EE900A9FED55
:10E300000B7AF8EE677AF0EE006A67EE877AB8EE7D
:10E31000047AA7EEA67ADFED067A67EE277AC5EDD6
:10E32000007A0CB1034B236003B030BD6740533A11
:10E3300000007A443313904300B500680379012B41
:10E3400085B00DD0022B07D1012303AAFF21FBF7D3
:10E3500099FE05B05DF804FB002005B05DF804FBF4
:10E360008268417C90F9100002F00102019203AA38
:10E370000092FF22F5F76EFE05B05DF804FB00BFCA
:10E3800030B5044600680379012B85B029D0022BF3
:10E390001ED1826812F0010F18BF512103AA08BFD5
:10E3A000D121FBF76FFE98B1BDF80C30194A5BBA6A
:10E3B0009BB2D360D368B3F5C87F0EDC1649174A09
:10E3C000D1F8943115683233AB4218D305B030BD63
:10E3D000104B6FF00102DA60F0E74FF0FF33D360CB
:10E3E000ECE78368417C90F9100003F0010301938E
:10E3F00003AB009351220223F5F72CFED3E701F57E
:10E40000CC72C1F89451206800235121FBF718FE0B
:10E4100005B030BDF8120020088200206C240020D6
:10E4200000B500680379012B85B008D0022B2FD0EE
:10E43000204B002283F8582105B05DF804FB836867
:10E44000417C90F9100003F0010303AACDE90023F9
:10E4500002230022F5F7FEFD164B83F85801002831
:10E46000EAD0BDF80C305BBA9BB2B3F5FA6F1AD2A2
:10E470001149124AA1FB0313DB0807EE903AF8EEAC
:10E48000E77AFDEEE77AC2ED047A05B05DF804FBA9
:10E49000826812F0010F18BF002103AA08BF802173
:10E4A000FBF7F0FDD8E7054B4FF0FF321A6105B0DE
:10E4B0005DF804FB08820020CDCCCCCCF812002003
:10E4C00010B500680379012B84B00C461DD0022BD7
:10E4D00018D1826812F0010F14BF0021802103AA15
:10E4E000FBF7D0FD60B15CB19DF80D309DF90C20BB
:10E4F000DB0903EB830302EB820203EB420323807D
:10E5000004B010BD002004B010BD8368417C90F9B8
:10E51000100003F00103019303AB009300220223D8
:10E52000F5F798FD0028DED1EAE700BFF0B50668F0
:10E53000F56983B00446002D65D000232B700423B9
:10E540000DEB03023046FF21FBF7F2FD10B900206E
:10E5500003B0F0BD206804236A46FF21FBF7E8FD05
:10E560000028F4D09DF804108A09023A012AEED955
:10E570009DF8053003EB012343F6FF74C3F30D034D
:10E58000A342E4D0002BE2D09DF806109DF80720AE
:10E5900002EB012240F2FF71B1EB521F4FEA62160B
:10E5A000D5D0002ED3D09DF800C09DF8012002EBFD
:10E5B0000C22C2F30D02A242C9D0002AC7D09DF896
:10E5C00002709DF8034004EB0724B1EB541F4FEA9F
:10E5D0006417BCD0002FBAD0991A0029B8BF49429D
:10E5E000FF29B4DCF11B0029B8BF4942FF29AEDC8A
:10E5F00013445B10F2195210C5F805300123C5F819
:10E6000001202B70A4E709211420F9F795FEF06191
:10E610000546266891E700BF70B50568E8690C46B5
:10E620001646A0B3D0F80130CCB1D0F805209FED4C
:10E630001B7ADFED1B5ADFED1B6A07EE902AF8EE1E
:10E64000677AB7EE006A77EEC77A77EEA77A87EE39
:10E65000A57A77EE467A67EEE67AC4ED007AAEB137
:10E6600007EE903A9FED107ADFED106A9FED106A89
:10E67000F8EEE77A67EE877A87EEA67ADFED0D6A25
:10E6800077EE467A77EEA67AC6ED007A70BD09215C
:10E690001420F9F751FEE861C4E700BF9AC9CC44E1
:10E6A0009AC94C460E76D7450000484300E0FF4427
:10E6B000000048423393884370B50668F46982B01D
:10E6C0000CB30025042325700DEB03023046FF2117
:10E6D000FBF72EFDA8B19DF804108B091CD19DF805
:10E6E00005209DF806509DF8073002EB012292B2FA
:10E6F00003EB0523C4F805205B1101222270C4F846
:10E70000013002B070BD054609211420F9F714FE4E
:10E71000F06104462E68D4E7034A04210320F9F788
:10E7200011FD284602B070BDC42B080870B50668FC
:10E73000F06982B00D461446002848D0D0F8053064
:10E74000DFED266A9FED267A07EE903AF8EE677ABB
:10E7500077EEE67AF3EE096A67EE877AB2EE047A2C
:10E7600067EEA67AF4EEC77AF1EE10FA22DCBAEE82
:10E77000047AF4EEC77AF1EE10FA1BD4D0F8013027
:10E780002DB19FED187A67EE877AC5ED007A7CB1DE
:10E7900007EE903A9FED146ADFED146AB8EE677ADF
:10E7A000DFED137AE7EE067A77EEA67AC4ED007A0B
:10E7B00002B070BD17EE900A61F0A0FD0D4ACDE9E0
:10E7C000000104210320F9F7BDFC02B070BD09214E
:10E7D0001420F9F7B1FDF061B0E700BF000000467A
:10E7E000000080380AD778430319C83D3393884323
:10E7F000000048C2E82B080830B52DED028B574CBD
:10E8000094F8B431022B85B019D0DFED557A79B187
:10E810009FED547A9FED546ADFED546A67EEA77A54
:10E8200067EE877A87EE867A77EE267AC1ED007AF0
:10E830000AB14F4B136005B0BDEC028B30BD94F8AC
:10E8400058326BBB4B4B1B689B072DD5B4F93C3240
:10E8500000EE103AB4F93A32B8EEC00A07EE103AB8
:10E8600020EE000AB8EEC77AB4F93E32A7EE070AE6
:10E8700007EE903AF8EEE77AA7EEA70AB5EEC00ADF
:10E88000F1EE10FAC1DBB5EE400AF1EE10FA5BD4FE
:10E89000F1EEC07AF4EE677AF1EE10FAB7D7B4E78A
:10E8A000344B1B68980704D4D4F85432D3ED347A2F
:10E8B000ADE7314D0DF10E00CDE9001228F02CFE30
:10E8C000BDF80E30D5F8EC03DFED2C5ADFED2C6AE5
:10E8D0009FED2C7A1B1A07EE903AF8EEE77AB0EE2D
:10E8E000408A87EEA56ADDE90012A6EE267AFDEEE3
:10E8F000C77AB0EE470A17EE903A2033402B20D863
:10E90000F9F7ACF9DDE900121F4BD4ED867A6C7C87
:10E91000A3F144001D462C3B002C08BF034695ED97
:10E92000007AD3ED056AA8EE407A37EEA60A20EE0B
:10E93000000AA7EE070AB5EEC00AF1EE10FAA2DA55
:10E9400063E79FED070ADFE7CDE9001263F0BEF948
:10E95000DDE90012F0EE407A9CE700BF088200205B
:10E9600000000000CDCC9C3F00409C4682E6C5479D
:10E9700033139043A000001018D400200000C842B8
:10E9800035FA8E3CDB0FC93F18D8002030B50C4D4E
:10E9900083B055F83030019183B107EE901A93EDB2
:10E9A000047A93ED030AF8EEE77A0446A7EE870AA5
:10E9B00063F07EF855F834309B68186003B030BDC2
:10E9C00050670020F0B54D4E96F84C3083B03BB107
:10E9D00096F85952012D04465ED0022D3ED00DB15D
:10E9E00003B0F0BD012280210068454FFAF7E6FB35
:10E9F00001223870FF212068FAF7E0FB2A463870C0
:10EA000029462068FAF7DAFB96F85A2238709121E5
:10EA10002068FAF7D3FB2946387001222068FAF7FC
:10EA2000CDFB2A463870FF212068FAF7C7FB2A463B
:10EA3000387080212068FAF7C1FB2946034601227D
:10EA400020683B70FAF7BAFB2E4A38701268C6F895
:10EA50005C22012386F8593203B0F0BD0068284FCC
:10EA600001AA1321FCF71EFA9DF8043038705B07E9
:10EA700025D1D6F86032002BB2D0224AD6F85C12EB
:10EA8000126892B2521A9342AAD24FF0FF32002378
:10EA90007A6086F85932A3E701AA0068184F00216E
:10EAA000FCF700FA9DF804303870DA07E1D4154A13
:10EAB00002231268C6F85C2286F8593290E7206873
:10EAC0002B4601AA1E21FBF733FBBDF8043002469A
:10EAD0000B2120683A7001225CBAFAF76FFB0A4BEF
:10EAE0003870A4B2A3FB0434E408012200237C6044
:10EAF00086F84D2086F8593272E700BF0882002060
:10EB0000F81200206C240020CDCCCCCCF0B541F024
:10EB1000010285B000212A4F2A4D2B4E0446FAF7F8
:10EB20004DFB3B68C6F85C32287016E0A368DB0733
:10EB30000DF10F024FF0130120465EBF0DF10F02E1
:10EB400093212046FCF75AF99DF80F30287013F0F6
:10EB500007030ED1D6F860224ABB2379012B18D0C7
:10EB6000022BE3D09DF80F30002013F0070328702C
:10EB7000F0D001220B212046FAF720FB00220346A9
:10EB8000114620462B70FAF719FB2870012005B0BA
:10EB9000F0BDA268617C94F9100002F001020192BC
:10EBA0000DF10F0200921322F5F754FACCE7396801
:10EBB000D6F85C0289B2091A8A42CED21846E6E734
:10EBC0006C240020F81200200882002010B5174C99
:10EBD00084F85110017984F8522001294FF0000285
:10EBE00082B084F8502012D002290CD1032304F102
:10EBF0005002FF21FBF7CEF9002814BF00206FF070
:10EC00000C0002B010BD6FF00C0002B010BD8268A5
:10EC1000417C90F91000503402F00102CDE900422D
:10EC20000323FF22F5F7E2F9E6E700BF08820020A0
:10EC300000680379012B0BD0022B08D183680F4A9F
:10EC400013F0010316D000235121FBF7A3B970473D
:10EC500000B58368094A417C90F9100083B003F045
:10EC60000103CDE9002300235122F5F7BFF903B0DA
:10EC70005DF804FBD121FBF78DB900BFA083002014
:10EC800030B5184D95F8503183B00BB903B030BD95
:10EC900004460DF10501006860F00EF89DF805309E
:10ECA00073B901212068104A85F852104FF40644C8
:10ECB0000323FF21A5F85040FBF7C2F903B030BD94
:10ECC0000DF1060296212068FFF7A2F8074ABDF869
:10ECD00006300749A2FB0323DB0801228B6085F87D
:10ECE0005121DEE70882002058820020CDCCCCCC18
:10ECF000F81200202DE9F843DFF8648004460F463F
:10ED00001646002540F634092046202168F0D9FD3A
:10ED10000446D0B103461C4613F8010B2028FAD054
:10ED20002046F9F7A9FF4845A8BF4846B0F5617FDE
:10ED3000B8BF4FF46170A0F56170A8FB0030C00847
:10ED40004DB178703378013333700DB90125DBE7AD
:10ED50002046BDE8F8833870337801333370F4E728
:10ED60001F85EB5130B583B005460846019161F02F
:10ED700059F90199044602462846F9F72FFC20B9B3
:10ED80002A5DA2F13001092902D8002003B030BD6C
:10ED900022F02002413A192AF8D90134281903B087
:10EDA00030BD00BF002ABCBF80185242002B30B5D6
:10EDB0003BDB5D180028B7BF121A841814460020E8
:10EDC000A4F11D0C0029BCBF2B460021BCF1000F93
:10EDD000C8BFA2EB0C04A5F10F02C8BF2418002A7B
:10EDE000C4BF9B1A5D1884421EDBC1F1010C114A9D
:10EDF000C1EB0113AC4400EB4303CCEB0C1C01341E
:10EE00004FEA4C0C02EB43024FF0200E8D42A8BF9C
:10EE1000002304DB22F813E01E339C45FAD10130B5
:10EE2000A04202F10202F1D130BD5C180D465B42F6
:10EE30002146BFE7347900201B4B1C48196C1C4A43
:10EE400010B441F080510124196404625321FF245D
:10EE5000CA205462506251625B6FDB0085B013D4EC
:10EE60000023144902930291029A13480432029239
:10EE7000029A136003930391039B0393039B18600F
:10EE800005B05DF8044B70470A4B002201920193D4
:10EE9000019B0193019A084B12689A42E0D105B098
:10EEA0005DF8044B704700BF0038024000000E427E
:10EEB000002800405028004076614E6970B4694CCB
:10EEC0000023224692F90410012902F10C021ED0FF
:10EED0000133062BF6D1002394F90420032A04F110
:10EEE0000C042AD00133062BF6D15F4B5D686A060D
:10EEF00047D55E4900230E460A461479372C02F1A5
:10EF000014024ED001330C2BF7D100234DE0584AA8
:10EF100003EB430302EB8303D3F86432002BDBD013
:10EF2000544B93F83D2093F83C5003799A4201D01A
:10EF3000AB42D0D1012070BC70474D4A03EB430374
:10EF400002EB8303D3F86432002BCED04A4B027914
:10EF500093F83D1093F83C309142EBD09A42E9D0BF
:10EF6000414B5D686A060CD5C3E7002B75D0196864
:10EF700003689942DED002EB820256F822209A42C0
:10EF8000D8D0EB0351D40179A1F13403012BD1D9AD
:10EF900001F0EF01A1F12000B0FA80F0400970BC4F
:10EFA000704703EB830306EB8303304C002294F895
:10EFB00004C0BCF1360F04F1140409D001320C2A4C
:10EFC000F5D1002B4BD01A6803689A420BD1B1E7F8
:10EFD00002EB8202920093B11C6803689C42A9D0A4
:10EFE00092599A42A6D0214A00231479182C02F192
:10EFF000140206D001330C2BF7D1002305E003687F
:10F00000EEE703EB830306EB830300220C791B2C52
:10F0100001F11401A9D001320C2AF7D1002BB0D094
:10F020001A6803689A42ACD184E7104E3246002336
:10F030001179212902F1140207D001330C2BA2D03F
:10F040001179212902F11402F7D103EB830302683D
:10F0500056F823309A4296D16CE703688BE7034A4F
:10F06000C3E700BF6C840020A00000100C0A002041
:10F070000882002070030020BC0500200D4B10B555
:10F0800003F1F00C4FF0000E02E014339C450FD05A
:10F090001A688242F9D1DA688A4218BFD9600EF143
:10F0A000010403F1140318BF5FFA84FE9C45EFD1FD
:10F0B000704610BD0C0A00202DE9F04F3D4EDFF8E0
:10F0C0000091DFF800813C4D83B04FF0000B0190C0
:10F0D000B2465F46DAF800404046002101E055F8AC
:10F0E0003100844203D001310E29F8D1FF21494477
:10F0F00091F8B012012944D0022909D1DAF80C1094
:10F10000480705D521F0040141F00801CAF80C10A8
:10F110005046FFF7D3FE48B9264B0BEB8B0103EBB0
:10F120008101C96801F00C00042835D00BF1010BF6
:10F13000BBF10C0F0AF1140ACCD1204C3046FFF77A
:10F14000BDFEC0B9F368590703F00C0213D5042AB9
:10F1500011D07A1CD5B2019A23F0080040F00400C7
:10F16000BA42014623F004031ED9F0603068FFF76D
:10F1700085FF2844C7B21436B442DFD103B0BDE8DE
:10F18000F08FDAF80C100B07C2D521F0080141F01E
:10F190000401CAF80C10BBE72046FFF76FFF0137E8
:10F1A000FFB20744FFB2C1E73068F3601946FFF7CA
:10F1B00065FFE0E70C0A0020B88A0708FC0A002077
:10F1C000088200200000014038B50446BDF8105008
:10F1D0002160084619B11946F3F7F0FC206829466A
:10F1E000F3F768FD236859680B68B3F844206FEAA9
:10F1F00042426FEA524292B2A3F844201A8892B275
:10F2000042F001021A804A79032A17D8DFE802F097
:10F21000110C070240330022A3601A6038BD3C3352
:10F220000022A3601A6038BD38330022A3601A6040
:10F2300038BD34330022A3601A6038BD0023A360B8
:10F240001B60FFDE2DE9F04F85B00646BDF838A003
:10F250009DF83CB0894617469846F3F713FC0546DF
:10F26000002842D0274A92F8BE42092C38D804EB35
:10F27000440302EB43130021C3F8C01283F8C41205
:10F28000631CDBB282F8BE3204EB440402F5307238
:10F290003079039302EB4414FDF704F850B3039B59
:10F2A00080F8069002210372C1710390BBF1000F38
:10F2B00012D11121FAF7E2F8039A136892885A835F
:10F2C0002046CDF800A043463A462946FFF77CFF8A
:10F2D000204605B0BDE8F08F327AFDF7E9F9EFE797
:10F2E000094A00210420F8F72DFF0024204605B02C
:10F2F000BDE8F08FBBF1000FE2D11121FAF7BEF8A3
:10F30000DEE700BF088200200C2C08082DE9F0473A
:10F310003E4D95F8803682B03BB93D4A022104202B
:10F3200002B0BDE8F047F8F70DBF95F8817695F883
:10F3300082360137FF1A102F0DDD102302210093B2
:10F3400085F88316334A3B4600210420F8F7FAFE7D
:10F3500002B0BDE8F08795F88C36012B064611D037
:10F36000022B0BD15FF09AF92B4BC5F8903695F82C
:10F370008C1611F0FD040BD0284ACFE7284BC5F8B6
:10F380009036F4E75FF08AF9264BC5F89036EEE741
:10F390007368BB422FDB002FDADDDFF89880DFF8DF
:10F3A00098A0DFF884902C3604E00134BC4248F881
:10F3B000040BCDD0DAF80430B5F884160091C3F30D
:10F3C00000720192B5F88636174AB9FBF3F356F886
:10F3D000040F9BB20321FFF735FF0028E5D1134A44
:10F3E000052601462346042085F8836602B0BDE861
:10F3F000F047F8F7A7BE042000930D4A85F883066E
:10F400003B462146F8F79EFEA2E700BF0882002097
:10F41000482C0808642C0808A5DD0008F02C080812
:10F4200091DD00088116030840420F00C82C08082F
:10F43000902C080814820020A000001030B503684A
:10F440002C4C2DED028BA34283B0F0EE408AB0EE3F
:10F45000608A13D004F58064A3420FD004F5705481
:10F46000A3420BD004F58064A34207D004F5806466
:10F47000A34203D0204B1C68640801E01E4B1C68AB
:10F480000192B4FBF1F202F57F420023FF32120C2D
:10F490000093B4FBF2F4B4FBF1F52246ABB20221C7
:10F4A000FFF7D0FEC0B1B5EE408AF1EE10FA17D0EA
:10F4B00007EE904AF8EE677A27EE888A9FED0F7A7A
:10F4C000C8EE076A0123037127EE667AC0ED046A6D
:10F4D000A8EEA77A80ED037A03B0BDEC028B30BDB5
:10F4E00007EE905AB8EE678A07EE904AF8EE677A10
:10F4F000E4E700BF000001400808002000007A4453
:10F500002DE9F04F2DED028BAA4B1F780C2F9BB0ED
:10F5100000F31581A84BA94D9B792B70032B22D9A1
:10F520001A1F022A00F20481052B00F03581062BF8
:10F530000CBF4FF47A544FF47A64A14AA149DFF822
:10F54000D8C203921646A04AC6F894264FF0000887
:10F5500000224FF000094A60CCE900899B4AB2FBC7
:10F56000F4F20A6005E0964A03921146984AC1F8FF
:10F570009426984A12F81330002B00F0108103688B
:10F58000BB42C0F26F81002F00F0A380DFF88C92A5
:10F59000DFF88CA29FED908A00F1040B4FF0000879
:10F5A000D9F804202B785BF8046FC2F30072062BA5
:10F5B00000F2E080DFE803F0AEA0927704040400DC
:10F5C000052B00F0D58085498548062B08BF0146EC
:10F5D0000024019200940A46142302213046FFF7CA
:10F5E00031FE0290002800F0C0807E4B31681A780E
:10F5F0007D4E22B9B0E00134944200F0AD80230189
:10F60000F3589942F7D1E2B2130104930298774C70
:10F61000016806914FF4907303FB02420B68D1F826
:10F6200004E05C6E049BC265F318DEF800000792EC
:10F6300005949A60002C00F0F580B0F844306C4AD4
:10F640006FEA43436FEA53439BB2A0F84430038808
:10F650009BB243F0800303809EF8063013F0040F42
:10F660009EF80530D15C028C14BF042301238B402B
:10F670009BB292B222EA03020284028C92B213433A
:10F68000038403889BB243F001030380059B002B96
:10F6900000F0FF80029A01231371029B4AF8383070
:10F6A0004FEAC8030CE0444BDFED520A9988B0EEF4
:10F6B000600A3046FFF7C2FE4AF838004FEAC80336
:10F6C0005AF80330002B58D008F1010847457FF461
:10F6D00067AF1BB0BDEC028BBDE8F08FDFED460AD3
:10F6E0009FED460A30464FF4FA61FFF7A7FE4FEA56
:10F6F000C8034AF83800E3E7DFED410A3046B0EED0
:10F70000600A4FF47A71FFF799FE4FEAC8034AF88E
:10F710003800D5E79FED300AF0EE480A30464FF446
:10F72000C871FFF78BFE4FEAC8034AF83800C7E7F5
:10F73000234A03921146334AC1F8942619E7204917
:10F74000314A0C230120009381F883063B460021B7
:10F750000420F8F7F7FCBCE713010493F1502149AA
:10F76000531C072A0B707FF651AF0023029394E7D6
:10F7700026492DE700234AF83830039C244A052007
:10F7800084F883064346002104201BB0BDEC028BA5
:10F79000BDE8F04FF8F7D6BC4FF4FA54CDE61D4A59
:10F7A000022104201BB0BDEC028BBDE8F04FF8F73E
:10F7B000C9BC00BF9800001018690020096700202C
:10F7C0000882002010670020BDDD000840420F00C5
:10F7D0008DE90008808B07086F12833AC0C62D00A0
:10F7E000001BB700B0670020B4670020A08800208D
:10F7F0005C8B070800000000ACC5A737ACC5A73676
:10F800006F1203398DDD00082C2D0808808D5B00F8
:10F81000B42D0808582D080818670020A000001013
:10F8200050670020DEF810304A4C059A190B1B0A6D
:10F83000CDE908E008469E46530104EB421CE3581C
:10F8400080EA13318EEA132301F0030103F00F0362
:10F850000B4302F1010211D0102AEDD1069A0023C8
:10F86000D3601AE703980093032180F883163A4A7D
:10F870003B4600210420F8F765FC2AE7069BC3F805
:10F880000CC09CF81C30DDE908E0002B3FF4D5AE3D
:10F8900003E7069B314AD8684368934252D0304A06
:10F8A000136B43F480031363069C07232146838371
:10F8B0005DF094FCE3689868F3F76AFCE3686268BB
:10F8C00098680799036823F0010303601368127CAA
:10F8D0000D914C330C93234B53F822300B930023A0
:10F8E000CDE91633CDE918331093149312230F93F7
:10F8F0004FF4806311934FF4804C4FF48053CDE963
:10F90000123C40230E930BA94FF4003315935DF086
:10F910008BFD2246E4680499A3681068069231447E
:10F9200056681A6842F010021A60446674790E4AEA
:10F9300032F81420A0F868208A81069A4B600123CF
:10F940001374A7E6A2F52052136B43F4001313635C
:10F95000AAE700BF0C080020782D080800600240CC
:10F9600000380240608B07085C8A070810B5104C0D
:10F97000D4E90423A16882B002FB03F38B428DF823
:10F98000070012D06368E0680DF10701184464F0C5
:10F990009BFE63682269A16813446269B3FBF1F0BE
:10F9A000013201FB10336360626102B010BD00BF21
:10F9B0002867002010B51420FCF774FC90B10446B1
:10F9C00001214FF40873C3800172F9F757FD2168D4
:10F9D000114BA0884883002283F89C2FC3F8984FCE
:10F9E00083F89D2F2520FCF75DFC044690B14FF471
:10F9F00008720223C28003720121F9F73FFD2168DA
:10FA0000054BA0884883002283F8A42FC3F8A04F99
:10FA100083F8A52F10BD00BF0882002010B5037920
:10FA2000012B84B00C4621D0022B1DD18368DB074B
:10FA30000DF10F024CBF01218121FBF7DFF99DF889
:10FA40000F30114A1070C3F3C002C3F3001CC3F39C
:10FA50008001A270C3F38012DB0984F800C06170DA
:10FA6000E270237104B010BD0020E8E782680DF158
:10FA70000F0102F00102CDE900121A46417C90F913
:10FA80001000F4F7E7FADAE7F81200202DE9F04366
:10FA900083B014460F4601AA50210546FBF702FA2F
:10FAA0009DF804303C4EDFF8F490307001335B0079
:10FAB000DBB201AA238046212846FBF7F3F923781D
:10FAC000DFF8DC80307009FB03F303F5FA73A8FB61
:10FAD00003239DF8042099090132DB0902FB01335D
:10FAE000A280A8FB03239B0901AAE3605121022302
:10FAF0002846FAF71DFB2378BDF80410307009FB87
:10FB000003F349BA03F5FA73A8FB0323CAB2C1F39E
:10FB100007218A40013292B29909DB0902FB0133C5
:10FB2000E280A8FB03239B09238201AA70212846B7
:10FB3000FBF7B8F99DF80430307001335B00DBB29D
:10FB400001AA6380712102232846FAF7F1FABDF871
:10FB50000420F978307052BAD3B2C2F3072293402E
:10FB600001339AB2228119B1E388D31A9AB2228161
:10FB7000A1780A4B0A4803FB01F101F5FA71A0FBD9
:10FB800001139909DB0902FB0133A0FB03239B0945
:10FB9000638203B0BDE8F083F8120020002F3A0022
:10FBA000D34D62102DE9F043A84FA94CDFF8A48291
:10FBB0008FB006464FF000094FF4FA7309AA892165
:10FBC0000068C7F8603287F84C90FBF76BF99DF836
:10FBD0002420207042F0010289213068F9F7EEFA02
:10FBE0004A46207088213068F9F7E8FA012220702F
:10FBF00080213068F9F7E2FA01222070FF21306895
:10FC0000F9F7DCFA4A46207049463068F9F7D6FA27
:10FC100009AA207091213068FBF744F99DF824303F
:10FC2000207001224946306887F85A32F9F7C6FA3F
:10FC30004A462070FF213068F9F7C0FA4A46207022
:10FC400080213068F9F7BAFA09AA2070602130687B
:10FC5000FBF728F99DF82420207042F01202602161
:10FC60003068F9F7ABFA20250223207009AA442155
:10FC700030688DF825508DF82490FAF7E1F9FF22CD
:10FC8000207001213068F9F799FA35682070012257
:10FC900080212846F9F792FA01222070FF21284698
:10FCA000F9F78CFA4A46207049462846F9F786FA51
:10FCB00006222070FF212846F9F780FA09AA207051
:10FCC00083212846FBF7EEF89DF82420207042F0AF
:10FCD000040283212846F9F771FA07222070FF21D8
:10FCE0002846F9F76BFA0122207081212846F9F79E
:10FCF00065FA0122207080212846F9F75FFA6B220D
:10FD0000207094212846F9F759FA4A462070832139
:10FD10002846F9F753FAD8F800302070C7F85C325B
:10FD200014E0AB68DB0709AA4FF0830128465EBFE9
:10FD300009AA83212846FBF761F89DF8243020703A
:10FD400083B9D7F86032002B40F00F832B79012B59
:10FD500000F0FE82022BE4D09DF8243000202070B9
:10FD6000002BEED0012283212846F9F727FA09AAB1
:10FD7000207092212846FBF795F8002220708121FF
:10FD800028469DF82490F9F719FA06222070FF21E1
:10FD90002846F9F713FA09AA207083212846FBF7B1
:10FDA00081F89DF82420207002F0FB028321284670
:10FDB000F9F704FA01222070FF212846F9F7FEF92D
:10FDC0000122207000212846F9F7F8F9002220705E
:10FDD000FF212846F9F7F2F90022207080212846F9
:10FDE000F9F7ECF90623207007AAB0213068FAF77A
:10FDF0009FF901222070FF213068F9F7DFF9002216
:10FE000020704F213068F9F7D9F92C2220704E214B
:10FE10003068F9F7D3F900222070FF213068F9F734
:10FE2000CDF9B4222070B6213068F9F7C7F94FEA4E
:10FE3000D918B8F1000F4FF00005207018BF4FF02F
:10FE40000C0809F07F0EAC46012017E00882002064
:10FE5000F81200206C240020F44503F0070317D0AB
:10FE600011F81C2C42FA03F3DB070CF1010105F138
:10FE7000010548BF5FFA81FC302D12D0EBB20EAA0B
:10FE800002EBD301984503F0070200FA02F2E3D92E
:10FE900011F81C3C013523EA0202302D01F81C2C1C
:10FEA000ECD1062307AAB0213068FAF7C9F801227D
:10FEB0002070FF213068F9F781F900221146207087
:10FEC0003068F9F77BF900222070FF213068F9F7DC
:10FED00075F90022207009213068F9F76FF90022C6
:10FEE000207010213068F9F769F900222070112183
:10FEF0003068F9F763F90122207024213068F9F79E
:10FF00005DF9FF22207025213068F9F757F90022AA
:10FF1000207075213068F9F751F901222070FF2116
:10FF20003068F9F74BF92C2220704E213068F9F730
:10FF300045F90022207048213068F9F73FF9294639
:10FF4000207020223068F9F739F900222070FF2153
:10FF50003068F9F733F92946207009223068F9F73B
:10FF60002DF90022207054213068F9F727F9042276
:10FF7000207031213068F9F721F9032220703221F5
:10FF80003068F9F71BF98322207040213068F9F7B7
:10FF900015F92522207046213068F9F70FF9002263
:10FFA000207060213068F9F709F9002220702721BC
:10FFB0003068F9F703F90622207050213068F9F70C
:10FFC000FDF80022207051213068F9F7F7F89622E9
:10FFD000207052213068F9F7F1F80822207056217C
:10FFE0003068F9F7EBF82A46207057213068F9F7A6
:10FFF000E5F80022207061213068F9F7DFF800226F
:020000040801F1
:10000000207062213068F9F7D9F80022207064214D
:100010003068F9F7D3F80022207065213068F9F7CD
:10002000CDF8A022207066213068F9F7C7F80122C8
:100030002070FF213068F9F7C1F8322220702221A8
:100040003068F9F7BBF81422207047213068F9F7BF
:10005000B5F8FF22207049213068F9F7AFF8002287
:1000600020704A213068F9F7A9F800222070FF219A
:100070003068F9F7A3F80A2220707A213068F9F77E
:100080009DF8002220707B213068F9F797F8212233
:10009000207078213068F9F791F801222070FF2153
:1000A0003068F9F78BF83422207023213068F9F793
:1000B00085F80022207042213068F9F77FF8FF228E
:1000C000207044213068F9F779F826222070452104
:1000D0003068F9F773F80522207046213068F9F787
:1000E0006DF84022114620703068F9F767F8062253
:1000F00020700E213068F9F761F81A222070202153
:100100003068F9F75BF84022207043213068F9F736
:1001100055F800222070FF213068F9F74FF80322CC
:10012000207034213068F9F749F8442220703521D5
:100130003068F9F743F801222070FF213068F9F7A1
:100140003DF80422207031213068F9F737F8092290
:1001500020704B213068F9F731F8052220704C21CE
:100160003068F9F72BF8042220704D213068F9F738
:1001700025F800222070FF213068F9F71FF80022CF
:10018000207044213068F9F719F8202220704521A9
:100190003068F9F713F80822207047213068F9F722
:1001A0000DF82822207048213068F9F707F800225E
:1001B000207067213068F9F701F80422207070215F
:1001C0003068F8F7FBFF0122207071213068F8F7E2
:1001D000F5FFFE22207072213068F8F7EFFF002251
:1001E000207076213068F8F7E9FF0022207077212F
:1001F0003068F8F7E3FF01222070FF213068F8F73C
:10020000DDFF012220700D213068F8F7D7FF0022B2
:100210002070FF213068F8F7D1FF01222070802183
:100220003068F8F7CBFFF822207001213068F8F72A
:10023000C5FF01222070FF213068F8F7BFFF0122BF
:1002400020708E213068F8F7B9FF0122207000215C
:100250003068F8F7B3FF00222070FF213068F8F70C
:10026000ADFF0022207080213068F8F7A7FF04223C
:1002700020700A213068F8F7A1FF3568207009AABC
:1002800084212846FAF70EFE9DF82420207002F003
:10029000EF0284212846F8F791FF012220700B21FC
:1002A0003068F8F78BFF05A9207030680390FFF7DE
:1002B000B5FB039809AA05A9FFF7E8FB9DF81430E0
:1002C000002B65D00C9B03F684539DF81620002A62
:1002D00055D00C9A02F2B22203EB42039DF817208C
:1002E00022B1BDF8342002F5257213449DF8182080
:1002F00022B1BDF8362002F22622134401213068D3
:10030000C7F8B83FE822F8F759FFD7F8B81F2070B0
:1003100044F61F639942306802D95EF007FD3068E9
:1003200001221146F8F74AFF402120703068FEF79D
:10033000EDFB50B1012130680222F8F73FFF0021A8
:1003400020703068FEF7E2FB28BB0FB0BDE8F083F9
:10035000AA68697C95F9100002F00102019209AACD
:1003600000928322F3F776FEE7E4D8F80020D7F86E
:100370005C1292B2521A9342BFF4E8ACE5E79DF8E2
:100380001520002AAAD00C9A02F525721344A5E77D
:1003900040F6363399E7E82201213068F8F70EFF7E
:1003A000002502234FF0200C09AA20704421306858
:1003B0008DF825C08DF82450F9F742FED6F800805C
:1003C000207005A94046FFF729FB09AA05A9404668
:1003D000FFF75CFB502257214046F8F7EFFE08225A
:1003E000207056214046F8F7E9FE0822207050217F
:1003F0004046F8F7E3FEBDF8342020704FF47A71E0
:1004000048F20E6301FB02337C4A934240F2F280D1
:100410007B4AA2FB03231B0C5A1E32F0FF0309D0B8
:100420002B465208013322F0FF019BB20029F8D17C
:100430001B029BB21343C3F30722DBB28DF81020DB
:100440008DF8113004AA022351214046F9F7F8FD36
:100450000C9A20704FF47A7148F20E6301FB02335C
:10046000684A934200F2C480654AA2FB0332120C30
:10047000013AD2B246214046F8F7A0FED7F8B81F9D
:10048000207044F61F63994202D940465EF04EFC4C
:1004900004AA01214046FAF705FD0222207001213D
:1004A00040469DF81050F8F789FE00212070404624
:1004B000FEF72CFB2A4601214046F8F77FFE3568FF
:1004C000207005A92846FFF7A9FA09AA05A9284618
:1004D000FFF7DCFA482211462846F8F76FFE08229B
:1004E000207047212846F8F769FE03222070322148
:1004F0002846F8F763FE0722207030212846F8F7D7
:100500005DFE01222070FF212846F8F757FE2022C9
:10051000207030212846F8F751FE00222070FF217C
:100520002846F8F74BFE0622207070212846F8F77F
:1005300045FEBDF83610344A207046F644034FF4A9
:100540007A7000FB0133A2FB03239DF817201B0BDD
:100550001AB1BDF82A2013449BB2002B46D05A1E74
:1005600032F0FF0309D000235208013322F0FF01CB
:100570009BB20029F8D11B029BB21343C3F307229D
:10058000DBB28DF810208DF811307121022304AAFE
:100590002846F9F755FDD7F8B81F207044F61F63B9
:1005A000994202D928465EF0C1FB04AA01212846DF
:1005B000FAF778FC02222070012128469DF810608D
:1005C000F8F7FCFD002120702846FEF79FFA32461E
:1005D00001212846F8F7F2FD642201232070C7F8B4
:1005E000602287F84C300FB0BDE8F0831A46C8E7A8
:1005F000FF223FE72B462A4620E700BF1B0C0100E5
:10060000950370F41B280D014963A41310B5174C12
:1006100084F85110017952BAA4F8522001294FF000
:10062000000282B084F8502012D002290CD1042399
:1006300004F15002FF21F9F7ADFC002814BF00209F
:100640006FF00C0002B010BD6FF00C0002B010BDD6
:100650008268417C90F91000503402F00102CDE92B
:1006600000420423FF22F3F7C1FCE6E708820020E2
:100670002DE9F04FA24FA34D066800213C4685B0FE
:10068000834685F850115A37C4F12D0905F1500AF7
:10069000884615E0022A0FD1B26812F0010F4FF020
:1006A000030352464FF0FF01304601BF0323524679
:1006B000FF213046F9F76EFCBC421AD014F8011F36
:1006C000327985F8521009EB0403012A85F850802D
:1006D00085F85130DED1B368717C96F9100003F0D3
:1006E0000103CDE900A3FF220323F3F77FFCBC4203
:1006F000E4D14FF40743A5F85030402385F8523039
:1007000052460323FF213046F9F79AFC00238DF867
:100710000E300DF10E0130465EF0CEFA9DF80E302F
:10072000002BF6D04FF40640A5F850000120764A81
:1007300085F852000323FF213046F9F781FC4FF47E
:100740000740714AA5F8500000240323FF213046DA
:1007500085F85240F9F774FC4FF40060A5F850009A
:100760000920694A85F852000323FF213046F9F732
:1007700067FC4FF43063A5F85030634A85F8524067
:1007800030460323FF21F9F75BFC00287FD0DBF81C
:1007900000600DF10E025E213046FDF739FBBDF819
:1007A0000E30B3F5D77F00F0A38079D8512B75D0E8
:1007B00040F29480AD2B00F09B80D62B40F08A80D5
:1007C000212408BB0A224B213046FEF7FFF90F22F5
:1007D00060213046FEF7FAF90D2263213046FEF71C
:1007E000F5F9B82269213046FEF7F0F940F60D72AE
:1007F00078213046FFF70AFF40F60E627A21304634
:10080000FFF704FF002875D0DBF8000021215EF01F
:10081000A3F9DBF800400DF10E02DE212046FDF7C2
:10082000F7FABDF80E309FED397AC3F30903ADF83E
:100830000E3003EB8303DB0007EE903AF8EEE77A25
:10084000204667EE877A0623FCEEE77A4FF4D84419
:1008500017EE902A110E85F85210110C52BA85F835
:100860005310A5F85420FF215246A5F85040F9F73F
:10087000E7FB4FF407414023DBF80000A5F85010D8
:1008800085F8523052460323FF21F9F7D9FB85F84A
:10089000500105B0BDE8F08F1E2BB5D1142490E7B0
:1008A00040F2E132934221D00AD940F28F42934282
:1008B00003D040F291529342A6D14FF4FA7480E7EC
:1008C00040F2D922934211D040F2E122934209D161
:1008D000642476E7602B3FF473AF95E71D2BDBD1E3
:1008E0000F246EE7B3F5E67FF2D08DE7C82468E702
:1008F000322466E7214630465EF02EF984E700BFD9
:100900004C92070808820020588200209A99893F5B
:1009100003682DE9F041DF691FB13B46BDE8F041B6
:100920001847002A164611DD04460D460E4400E025
:1009300023689B68204698470028F9D0236815F85B
:10094000011B1B6820469847AE42F1D1BDE8F081FB
:10095000DEE700BF224B1B6813F0100F214B03D0C2
:10096000B3F8BC2F520717D493F8D62F02BB93F8D5
:10097000E42FD3F8E03F52B143B120B11A689B880D
:10098000138370474BB31A689B885383704780F07A
:100990000100002BF1D1F9E793F8D62FB2B993F803
:1009A000E42FD3F8E03F002AECD1002BE6D17047CA
:1009B000D3F8D82F002AE9D058B19268B3F8DC1FD9
:1009C000094BB3FBF1F35B1013607047D3F8D82FDA
:1009D00022B1936800221A6070477047704700BFC9
:1009E0009C0000100882002040420F00BFF34F8F90
:1009F0000549064BCA6802F4E0621343CB60BFF3BB
:100A00004F8F00BFFDE700BF00ED00E00400FA05D6
:100A100008B572B600224FF0FF31930003F1604336
:100A200003F561430132082AC3F88010C3F880112E
:100A3000F3D1FFF7DBFF00BF012108B50846F3F74C
:100A400069FCFFF7E5FF00BF00B583B00D49002248
:100A500000920091009B04330093009B1B68012BC4
:100A600002D003B05DF804FB01920191019B06499D
:100A700004330193019B1A600B6883F308884B6869
:100A80009847FEE7502800400000FF1F10B4EFF326
:100A90001183102282F31288094C0A4822684FF011
:100AA000E021013222608A69C0F8E82F0022C0F8F4
:100AB000EC2F0A69DBB283F311885DF8044B7047B1
:100AC0006C2400200882002030B4EFF31182102340
:100AD00083F312884FF0E023D2B29969186910F4B9
:100AE000803F0D481EBF0121C0F8EC1F99690B4BD8
:100AF0001D68D0F8EC3F82F31188094804684FF470
:100B00007A7202FB04F02B44401A0021B0FBF4F08F
:100B100030BCE3FB02017047088200206C240020F7
:100B200068240020124B5B68C3F30803FBB9EFF3A2
:100B30001183E3B930B40F4A0F4C4FF0E02C116829
:100B4000DCF8180013688B42F9D1D4F8E81F814211
:100B5000F5D30A4A15684FF47A7404FB05F20021B4
:100B6000101AB0FBF5F0E3FB040130BC7047ABE7B3
:100B700000ED00E06C2400200882002068240020A2
:100B800090B170B5461EFFF7CDFF04460D46FFF746
:100B9000C9FF031B61EB0502B3F57A7F72F1000315
:100BA000F5D3013EEFD270BD704700BF70B500684D
:100BB00001220921F8F702FB6426FFF7B3FF044680
:100BC0000D46FFF7AFFF031B61EB0502B3F57A7F1C
:100BD00072F10003F5D3013EEFD170BD2DE98048DD
:100BE00083B0431C0193DFF83C810A230093D8F8BB
:100BF0009C10D8F8D830B8F8A000B8F8DC20DDF8A0
:100C000004B048834FF0320A1A834FF005094C694B
:100C1000204214BF4883088359690A4214BF5A838B
:100C20001A830120FFF796FE56465746FFF77AFFD4
:100C300004460D46FFF776FF001B61EB0501B0F59A
:100C40007A7F71F10003F5D3013FEFD1D8F89C30E2
:100C5000B8F8A02059690A4214BF5A831A83D8F8F9
:100C6000D830B8F8DC2059690A4214BF5A831A8375
:100C70000020FFF76FFEFFF755FF04460D46FFF714
:100C800051FF001B61EB0501B0F57A7F71F10003A4
:100C9000F5D3013EEFD1B9F1000F0BD0B9F1010945
:100CA00010D0B8F8A000D8F89C10B8F8DC20D8F81C
:100CB000D830ACE70BF1FF3BBBF1000F19D04FF080
:100CC0000009EEE74FF4FA76FFF72CFF04460D46D5
:100CD000FFF728FF001B61EB0501B0F57A7F71F18A
:100CE0000003F5D3013EEFD14FF0FA0ABBF1000F3C
:100CF000E5D14FF47A76FFF715FF04460D46FFF76E
:100D000011FF031B61EB0501B3F57A7F71F100035D
:100D1000F5D3013EEFD1009B013B00937FF467AF19
:100D2000FFF78AFE7425002018B103681B6A03B11F
:100D300018470020704700BF10B50C4620B103686B
:100D4000DB6A0BB1984768B9074B0020C4E9000083
:100D5000C4E90200C4E906332D2130222061217547
:100D600084F8202010BD00BF488208080178F9B13E
:100D7000F8B5104F0546002602E015F8011FB1B185
:100D8000D7F8F04F637A5A1C2344D2B26272997238
:100D9000237A9342F1D8002AEFD004F10A01D4E972
:100DA00000309847667215F8011F0029E8D1F8BD98
:100DB000704700BF0882002070B504460F48FFF757
:100DC000D5FF2046FFF7D2FF0D48FFF7CFFF0D4BB1
:100DD000B3F8F46F16B970BD013EFCD0FFF7A2FE68
:100DE00004460D46FFF79EFE031B61EB0502B3F5BB
:100DF0007A7F72F10003F5D3EEE700BFDC2D08081F
:100E0000708D08080882002030B583B00F4C019027
:100E10000F480091FFF7AAFFDDE900320D49D4F831
:100E2000F00F5CF0A7FBD4F8F05F6A7A32B12B6860
:100E3000686805F10A01984700236B7294F8F63F41
:100E400013B1012384F8F73F03B030BD08820020BE
:100E5000E42D0808F1DE00080FB470B582B006A9D1
:100E600051F8040B0191FFF7CFFF0E48FFF77EFF0B
:100E70000D4BB3F8F46F36B902B0BDE8704004B062
:100E80007047013EF8D0FFF74DFE04460D46FFF7D0
:100E900049FE031B61EB0502B3F57A7F72F1000393
:100EA000F5D3EEE7708D08080882002000283DD0B9
:100EB0000378002B3AD02DE9F04F87B05A4905AAA4
:100EC00064F010FC0446002800F0A2804FF0000BF4
:100ED000DFF88091DFF88081DFF880A15D465F4612
:100EE0004FF0FF360BE0BBF1000F26D04E4905AAAC
:100EF000002064F0F7FB0BF1010B044610B3BBF1CB
:100F0000010F15D0BBF1020FEDD14946204666F026
:100F100032FD00286ED045F001054146204666F0BE
:100F20002AFD00285FD045F00205DFE73F4893E740
:100F30002046F7F7A1FE0746D8E72046F7F79CFEC4
:100F40000646D3E770B23A4A002392F90010814274
:100F500025D00133062B02F10C02F6D1002F50D020
:100F6000002D08BF03250023EDB2CDE90153009702
:100F70001A4619462BF056FB044600284ED02D4841
:100F8000DFF8DC803A463146F7F7A6F831462A48C2
:100F9000F7F7A2F8D8F85C0121465AF07FF8DFF89D
:100FA000C08003EB430308EB8303D3F8FC4F002C12
:100FB000D4D022483146F7F78FF85DB16179A94264
:100FC00008D01F482A46F7F787F82368E9B29B69DB
:100FD00020469847E36A002BD8D01A48F7F77CF8E8
:100FE0000023E362D2E72046514666F0C4FC0028A5
:100FF00099D17BE71449204666F0BDFC00288AD1D0
:101000008BE712483146F7F767F807B0BDE8F08F75
:101010004FF0FF3025462746064694E731460C48F8
:10102000F7F75AF8F1E700BFD0830808E42E080864
:1010300000920020442E0808B42E0808642E0808E8
:101040007C2E08089C2E08082C460808FC2D080851
:10105000242E0808F02D0808F42D0808F82D08089B
:1010600008820020002868D02DE9F04F90F800C0D9
:1010700085B00446BCF1000F2AD000F100475A4E5B
:101080008646023F01466346722207E0984526D114
:10109000B94212D011F8013F16F8012FA3F1410512
:1010A000192DA2F1410098BF2033192802F1200820
:1010B000ECD99A4213D1002AEAD14C4C0023C4F84F
:1010C0001C3E84F8233EA4F8243E05B0BDE8F08F12
:1010D0000021012005B0BDE8F04F5AF039B8444E68
:1010E000214663466C2207E098452AD1B94212D0C6
:1010F00011F8013F16F8012FA3F14105192DA2F1B6
:10110000410098BF2033192802F12008ECD99A42F7
:1011100017D1002AEAD1374B1B685B07D5D4334C73
:1011200094F9223E002BD0D194F91D3E002BC5DC52
:1011300005B0BDE8F04F52F023B8002101205AF06D
:1011400007B82D48732307E065455BD1774513D079
:101150001EF801CF10F8013FACF141011929A3F1AC
:10116000410298BF0CF1200C192A03F12005EBD99C
:10117000634547D1002BE9D11C4B002293F9230E84
:1011800083F81C2E1C46164693F8CE140129A1F1B3
:10119000030509D0052D07D90EB184F8230E174891
:1011A00005B0BDE8F04F57E693F8CF14A52903F139
:1011B000140303D00132782AE6D1EDE7012803D0E9
:1011C000013840B20126F5E70D4984F81C0E0023D2
:1011D000013284F81D2E01F8B83C84F8233E05B096
:1011E000BDE8F04F4FF0B6BDF02E080818D400202F
:1011F000F82E08089C000010C83D0808E42E0808D6
:1012000000930020DFF880A22046F7F735FD1AF999
:10121000B87C07FA80F5772D064600F2D18020468B
:10122000202166F04EFB8046002800F01C8103461A
:10123000984613F8012B202AFAD04046F7F71CFDF8
:1012400001245FFA80F94046202166F03AFB80468F
:10125000002800F00D810346984613F8012B202A40
:10126000FAD04046F7F708FD01340090E4B240465A
:10127000202166F026FB8046002800F0F780034618
:10128000984613F8012B202AFAD04046F7F7F4FCD1
:1012900001340190E4B24046202166F012FB804602
:1012A000002800F0BF800346984613F8012B202A3F
:1012B000FAD04046F7F7E0FC01340290E4B2404631
:1012C000202166F0FEFA8046002800F0A98003463F
:1012D000984613F8012B202AFAD04046F7F7CCFCA9
:1012E00001340FFA80FBE4B24046202166F0E9FAAF
:1012F0000246002800F0B58003461A4613F8011B89
:101300002029FAD010460392F7F7B6FC0134039A6D
:101310000FFA80F8E4B21046202166F0D2FA0028D5
:1013200056D003461A46013311782029FAD01046C8
:101330000392F7F7A1FC039A03461BB21046202143
:10134000039366F0BEFA039B002800F093800246E8
:101350001046013201782029FAD00393F7F78CFC6C
:1013600004F0FD04042C039B08BFC2B27FF417AF46
:10137000B9F1010F04D9A9F1030105293FF60FAF17
:1013800022B1A52A2FD0482A7FF409AF3DB33B49AB
:1013900005EB850501EB850181F8CE940098C1F835
:1013A000BC040198C1F8C0040298C1F8C404A1F8B3
:1013B000C8B4A1F8CA84A1F8CC3481F8CF2484E65B
:1013C0002F4930487723002205B0BDE8F04F43E5B0
:1013D0005FFA88F203468046062CC9D0DFE627492B
:1013E00081F8235ED8E7FDB9244C0099C4F8BC14F9
:1013F0000199C4F8C0140299A4F8CC3484F8CE94AE
:10140000C4F8C414A4F8C8B4A4F8CA8484F8CF24D7
:10141000012301373E440AF8B86C84F8233E54E6B1
:10142000834661E702904AE7144C009805EB850576
:1014300004EB8501A1F8CC3494F8233EC1F8BC0438
:101440000198C1F8C0040133029881F8CE94C1F824
:10145000C404A1F8C8B4A1F8CA8481F8CF245BB24F
:10146000D7E7804657E704468146ECE6019012E74D
:101470000090FCE60134E4B20246ADE718D4002047
:10148000002F08080C2F0808009300202DE9F047D2
:1014900082B03E4901AA64F025F9002872D04FF0CD
:1014A000000A4FF0FF34394DD1465646D046274604
:1014B000BAF1040F09D8DFE80AF0443E380E030001
:1014C0000378482B46D0562B41D03148FFF7C4FC57
:1014D00002B0BDE8F087F7F7CFFB3F280646F4D807
:1014E000002001AA294664F0FDF80AF1010A00284B
:1014F000DED1BAF1040F3AD02FDDBAF1050FE4D1F5
:10150000244AB30103F47C6308F03F0843EA08036C
:10151000B9F1000F01D043F40053932101FB0744BC
:1015200002EB440424F8B43CD2E7F7F7A5FB3F28CC
:101530008046D5D9C9E7F7F79FFB92280446CFD953
:10154000C3E7F7F799FB03280746C9D9BDE74FF072
:101550000109C5E74FF00009C2E7BAF1020FB4DC98
:101560000D4923463A46012059F078FEB0E7094A72
:10157000932303FB074302EB430333F8B49CC9F303
:101580004039BEE74FF0FF373C46E9E7D083080813
:10159000E42E0808009300204C92002080B51948E2
:1015A000194DFFF7E3FB1948FFF7E0FBD5F8F04FC3
:1015B000627A32B12146606851F80A3B98470023AD
:1015C0006372D5F85C713B6838465B699847B0B97F
:1015D0000A26FFF7A7FA04460D46FFF7A3FA031BF6
:1015E00061EB0502B3F57A7F72F10003F5D3013E9A
:1015F000EFD13B6838465B6998470028E8D0012066
:1016000007F014FB2C2F080808820020482F080838
:1016100030B42F4C94F8E433012B86B002D006B0DE
:1016200030BC704794F8E9330A2B04D0294806B03F
:1016300030BCFFF79BBB41218DF8011026490023E8
:101640001520097D8DF80200CDE90333EB20CDE9AB
:101650000133A6228DF803008DF80410B220032177
:101660008DF805008DF814308DF800208DF80610E7
:10167000EC460DF1120541F2210083EA0223082213
:1016800013F4004F80EA43010ABF5B008BB29BB2A8
:10169000013AF5D1654502D01CF8012FEDE7C3F3FF
:1016A00007228DF814308DF81320EC461523C4F86A
:1016B0005434BCE80F00094D0FC59CE8030045F801
:1016C000040B0748297006B030BCFFF74FBB00BFC2
:1016D00000930020542F0808F812002004970020DF
:1016E000642F0808F8B52F482F4FFFF73FFB2F480E
:1016F000FFF73CFBB7F8F46F002E44D1D7F8F04F5A
:10170000627A32B12146606851F80A3B984700235B
:101710006372274B002583F85854C3F8985483F814
:101720009C5422F0FFF82348FFF720FBD7F8F04F36
:10173000627A2AB12146606851F80A3B984765727F
:10174000D7F85C713B6838465B699847B0B90A26A0
:10175000FFF7E8F904460D46FFF7E4F9031B61EBD8
:101760000502B3F57A7F72F10003F5D3013EEFD1A4
:101770003B6838465B6998470028E8D0002007F0AE
:1017800055FA013EBAD0FFF7CDF904460D46FFF7F2
:10179000C9F9031B61EB0502B3F57A7F72F100030F
:1017A000F5D3EEE7802F080808820020708D080826
:1017B00000930020482F0808F8B530490522044658
:1017C00066F094F818BB2E4E96F8F63F23B9012226
:1017D00086F8F62F86F8F73F2A48FFF7C7FA2A4817
:1017E000FFF7C4FAB6F8F46F16B9F8BD013EFCD0A5
:1017F000FFF798F904460D46FFF794F9031B61EBD8
:101800000502B3F57A7F72F10003F5D3EEE71F49C5
:101810000322204666F06AF850BB194E96F8F63F50
:1018200013B196F8F73FFBB91948FFF79FFA16482E
:10183000FFF79CFAB6F8F47F3FB9002386F8F63F2D
:1018400086F8F73FF8BD013FF7D0FFF76BF9044684
:101850000D46FFF767F9031B61EB0502B3F57A7FCD
:1018600072F10003F5D3EEE70A48FFF7F5FAE4E773
:10187000BDE8F8400848FFF7EFBA00BFAC2F0808F2
:1018800008820020B42F0808708D0808EC4E080864
:1018900004300808CC2F080818300808F8B52C4C7C
:1018A00094F8F63F1BB194F8F73F002B44D1294D33
:1018B00029480126FFF75AFA85F8A36485F8D86409
:1018C000F7F77AFA254B85F8CE641B682448C5F8EB
:1018D000B034002685F8D86485F8A364FFF746FA8B
:1018E000D4F8F05F6A7A02BBD4F85C713B68384682
:1018F0005B699847B0B90A24FFF714F905460E460C
:10190000FFF710F9401B61EB0601B0F57A7F71F12A
:101910000003F5D3013CEFD13B6838465B6998473B
:101920000028E8D0002007F081F9D5E9003005F162
:101930000A0198476E72D7E70A48FFF78DFA0A48FE
:10194000FFF78AFA002384F8F63F84F8F73FF8BDE2
:101950000882002000930020483008086C240020F2
:10196000482F0808CC2F080828300808F8B5284C5C
:10197000284F012605462848FFF7F8F905F00CFF27
:1019800084F8A36484F8D864F7F716FA234A244944
:10199000126884F8CE6400232846C4F8B02484F882
:1019A000D83484F8A33487F8F73FFDF7DBF900B1AA
:1019B000F8BD04461B48FFF7D9F9D7F8F05F6A7AFB
:1019C0002AB1D5E9003005F10A0198476C72D7F8C1
:1019D0005C713B6838465B699847B0B90A26FFF7E7
:1019E000A1F804460D46FFF79DF8031B61EB0502C5
:1019F000B3F57A7F72F10003F5D3013EEFD13B6876
:101A000038465B6998470028E8D0002007F00EF9B7
:101A10000093002008820020503008086C24002029
:101A200068300808482F080870B50C48FFF79EF981
:101A30000B4BB3F8F46F16B970BD013EFCD0FFF745
:101A400071F804460D46FFF76DF8031B61EB0502C4
:101A5000B3F57A7F72F10003F5D3EEE7708D0808D5
:101A600008820020800601D5002933D10CB470B55E
:101A7000194C1A49D4F8F00F82B007AB069A0193BB
:101A80005BF078FDD4F8F05F6A7A32B12B68686851
:101A900005F10A01984700236B721148FFF766F9B8
:101AA000B4F8F46F3EB9012002B0BDE8704002B056
:101AB0007047013EF7D0FFF735F804460D46FFF7B3
:101AC00031F8031B61EB0502B3F57A7F72F1000375
:101AD000F5D3EEE70020704708820020F1DE000811
:101AE000708D0808F0B5044683B070B302785AB31D
:101AF00000F10040434D21460238722307E097422F
:101B000037D1884214D011F8012F15F8013FA2F106
:101B1000410EBEF1190FA3F1410C98BF2032BCF168
:101B2000190F03F12007EAD9934222D1002BE8D103
:101B3000354B364AC3F8DC24C3F8E024C3F8E42468
:101B4000C3F8E82403B0F0BD1446314D314E35F8EA
:101B5000241005EB840332465888CDE9001001209B
:101B6000234600210444FFF77DFF042CEFD103B08E
:101B7000F0BD2046F7F780F8032805462FD8204609
:101B8000202165F09EFE0446002839D003461C46FD
:101B900013F8012B202AFAD02046F7F76DF8012719
:101BA00006462021204665F08CFE034688B1184683
:101BB00001330278202AFAD0F7F75EF84FB1A6F287
:101BC000EE2240F2DC539A4203D8A0F2EE229A426F
:101BD0000ED9114803B0BDE8F040FFF73DB90F49F9
:101BE0000F480323002203B0BDE8F040FFF734B9EB
:101BF000054B03EB8505A5F8DC64A5F8DE04A1E739
:101C00000746CEE7F02E080800930020E803D0072F
